Component: ARM Compiler 5.06 update 6 (build 750) Tool: armlink [4d35ed]

==============================================================================

Section Cross References

    main.o(i.TIMER2_IRQHandler) refers to main.o(i.saadc_start) for saadc_start
    main.o(i.TIMER2_IRQHandler) refers to printf1.o(i.__0sprintf$1) for __2sprintf
    main.o(i.TIMER2_IRQHandler) refers to strlen.o(.text) for strlen
    main.o(i.TIMER2_IRQHandler) refers to main.o(.data) for .data
    main.o(i.TIMER2_IRQHandler) refers to main.o(.bss) for .bss
    main.o(i.ble_evt_handler) refers to nrf_log_frontend.o(i.nrf_log_frontend_std_0) for nrf_log_frontend_std_0
    main.o(i.ble_evt_handler) refers to bsp.o(i.bsp_indication_set) for bsp_indication_set
    main.o(i.ble_evt_handler) refers to app_error.o(i.app_error_handler_bare) for app_error_handler_bare
    main.o(i.ble_evt_handler) refers to nrf_ble_qwr.o(i.nrf_ble_qwr_conn_handle_assign) for nrf_ble_qwr_conn_handle_assign
    main.o(i.ble_evt_handler) refers to main.o(.data) for .data
    main.o(i.ble_evt_handler) refers to nrf_log_frontend.o(log_const_data) for m_nrf_log_app_logs_data_const
    main.o(i.ble_evt_handler) refers to main.o(.bss) for .bss
    main.o(i.conn_params_error_handler) refers to app_error.o(i.app_error_handler_bare) for app_error_handler_bare
    main.o(i.fatfs_example) refers to diskio_blkdev.o(i.diskio_blockdev_register) for diskio_blockdev_register
    main.o(i.fatfs_example) refers to nrf_log_frontend.o(i.nrf_log_frontend_std_0) for nrf_log_frontend_std_0
    main.o(i.fatfs_example) refers to diskio_blkdev.o(i.disk_initialize) for disk_initialize
    main.o(i.fatfs_example) refers to nrf_log_frontend.o(i.nrf_log_frontend_std_1) for nrf_log_frontend_std_1
    main.o(i.fatfs_example) refers to ff.o(i.f_mount) for f_mount
==============================================================================

Removing Unused input sections from the image.

    Removing main.o(.rev16_text), (4 bytes).
    Removing main.o(.revsh_text), (4 bytes).
    Removing main.o(.rrx_text), (6 bytes).
    Removing main.o(.data), (6 bytes).
    Removing main.o(.data), (4 bytes).
    Removing main.o(.data), (2 bytes).
    Removing boards.o(.rev16_text), (4 bytes).
    Removing boards.o(.revsh_text), (4 bytes).
    Removing boards.o(.rrx_text), (6 bytes).
    Removing boards.o(i.bsp_board_button_state_get), (32 bytes).
    Removing boards.o(i.bsp_board_init), (84 bytes).
    Removing boards.o(i.bsp_board_led_idx_to_pin), (12 bytes).
    Removing boards.o(i.bsp_board_pin_to_led_idx), (36 bytes).
    Removing boards.o(i.nrf_gpio_cfg), (36 bytes).
    Removing bsp.o(.rev16_text), (4 bytes).
    Removing bsp.o(.revsh_text), (4 bytes).
    Removing bsp.o(.rrx_text), (6 bytes).
    Removing bsp.o(i.alert_timer_handler), (6 bytes).
==============================================================================

Image Symbol Table

    Local Symbols

    Symbol Name                              Value     Ov Type        Size  Object(Section)

    ../clib/../cmprslib/zerorunl2.c          0x00000000   Number         0  __dczerorl2.o ABSOLUTE
    ../clib/microlib/ctype/ctype.c           0x00000000   Number         0  ctype_o.o ABSOLUTE
    ../clib/microlib/ctype/ctype.c           0x00000000   Number         0  isalnum_o.o ABSOLUTE
    ../clib/microlib/ctype/ctype.c           0x00000000   Number         0  isalpha_o.o ABSOLUTE
    ../clib/microlib/ctype/ctype.c           0x00000000   Number         0  isblank_o.o ABSOLUTE
    ../clib/microlib/ctype/ctype.c           0x00000000   Number         0  isspace_o.o ABSOLUTE
    ../clib/microlib/ctype/ctype.c           0x00000000   Number         0  isupper_o.o ABSOLUTE
    ../clib/microlib/ctype/ctype.c           0x00000000   Number         0  isxdigit_o.o ABSOLUTE
    ../clib/microlib/ctype/ctype.c           0x00000000   Number         0  iscntrl_o.o ABSOLUTE
    ../clib/microlib/ctype/ctype.c           0x00000000   Number         0  isgraph_o.o ABSOLUTE
    ../clib/microlib/ctype/ctype.c           0x00000000   Number         0  islower_o.o ABSOLUTE
    ../clib/microlib/ctype/ctype.c           0x00000000   Number         0  isprint_o.o ABSOLUTE
    ../clib/microlib/ctype/ctype.c           0x00000000   Number         0  ispunct_o.o ABSOLUTE
    ../clib/microlib/ctype/ctype.c           0x00000000   Number         0  isdigit_o.o ABSOLUTE
    ../clib/microlib/division.c              0x00000000   Number         0  uldiv.o ABSOLUTE
    ../clib/microlib/division.c              0x00000000   Number         0  uidiv.o ABSOLUTE
    ../clib/microlib/init/entry.s            0x00000000   Number         0  entry5.o ABSOLUTE
    ../clib/microlib/init/entry.s            0x00000000   Number         0  entry7a.o ABSOLUTE
    ../clib/microlib/init/entry.s            0x00000000   Number         0  entry.o ABSOLUTE
    ../clib/microlib/init/entry.s            0x00000000   Number         0  entry2.o ABSOLUTE
    ../clib/microlib/init/entry.s            0x00000000   Number         0  entry11b.o ABSOLUTE
    ../clib/microlib/init/entry.s            0x00000000   Number         0  entry11a.o ABSOLUTE
    ../clib/microlib/init/entry.s            0x00000000   Number         0  entry10b.o ABSOLUTE
    ../clib/microlib/init/entry.s            0x00000000   Number         0  entry10a.o ABSOLUTE
    ../clib/microlib/init/entry.s            0x00000000   Number         0  entry9b.o ABSOLUTE
    ../clib/microlib/init/entry.s            0x00000000   Number         0  entry9a.o ABSOLUTE
    ../clib/microlib/init/entry.s            0x00000000   Number         0  entry8b.o ABSOLUTE
    ../clib/microlib/init/entry.s            0x00000000   Number         0  entry8a.o ABSOLUTE
    ../clib/microlib/init/entry.s            0x00000000   Number         0  entry7b.o ABSOLUTE
    ../clib/microlib/longlong.c              0x00000000   Number         0  llshl.o ABSOLUTE
    ../clib/microlib/longlong.c              0x00000000   Number         0  llsshr.o ABSOLUTE
    ../clib/microlib/longlong.c              0x00000000   Number         0  llushr.o ABSOLUTE
    ../clib/microlib/printf/printf.c         0x00000000   Number         0  printf1.o ABSOLUTE
    ../clib/microlib/printf/printf.c         0x00000000   Number         0  printf0.o ABSOLUTE
    ../clib/microlib/printf/printf.c         0x00000000   Number         0  printfb.o ABSOLUTE
    ../clib/microlib/printf/printf.c         0x00000000   Number         0  printf2.o ABSOLUTE
    ../clib/microlib/printf/printf.c         0x00000000   Number         0  printfa.o ABSOLUTE
    ../clib/microlib/printf/printf.c         0x00000000   Number         0  printf8.o ABSOLUTE
    ../clib/microlib/printf/printf.c         0x00000000   Number         0  printf7.o ABSOLUTE
    ../clib/microlib/printf/printf.c         0x00000000   Number         0  printf6.o ABSOLUTE
    ../clib/microlib/printf/printf.c         0x00000000   Number         0  printf5.o ABSOLUTE
    ../clib/microlib/printf/printf.c         0x00000000   Number         0  printf4.o ABSOLUTE
    ../clib/microlib/printf/printf.c         0x00000000   Number         0  printf3.o ABSOLUTE
    ../clib/microlib/printf/stubs.s          0x00000000   Number         0  stubs.o ABSOLUTE
    ../clib/microlib/string/memcmp.c         0x00000000   Number         0  memcmp.o ABSOLUTE
    ../clib/microlib/string/memcpy.c         0x00000000   Number         0  memcpya.o ABSOLUTE
    ../clib/microlib/string/memcpy.c         0x00000000   Number         0  memcpyb.o ABSOLUTE
    ../clib/microlib/string/memset.c         0x00000000   Number         0  memseta.o ABSOLUTE
    ../clib/microlib/string/strcpy.c         0x00000000   Number         0  strcpy.o ABSOLUTE
    ../clib/microlib/string/strlen.c         0x00000000   Number         0  strlen.o ABSOLUTE
    ../clib/microlib/stubs.s                 0x00000000   Number         0  iusefp.o ABSOLUTE
    ../fplib/microlib/fpadd.c                0x00000000   Number         0  dadd.o ABSOLUTE
    ../fplib/microlib/fpdiv.c                0x00000000   Number         0  ddiv.o ABSOLUTE
    ../fplib/microlib/fpepilogue.c           0x00000000   Number         0  depilogue.o ABSOLUTE
    ../fplib/microlib/fpfix.c                0x00000000   Number         0  dfixul.o ABSOLUTE
    ../fplib/microlib/fpmul.c                0x00000000   Number         0  dmul.o ABSOLUTE
    ..\..\..\..\..\..\components\ble\ble_advertising\ble_advertising.c 0x00000000   Number         0  ble_advertising.o ABSOLUTE
    ..\..\..\..\..\..\components\ble\ble_link_ctx_manager\ble_link_ctx_manager.c 0x00000000   Number         0  ble_link_ctx_manager.o ABSOLUTE
    ..\..\..\..\..\..\components\ble\ble_services\ble_nus\ble_nus.c 0x00000000   Number         0  ble_nus.o ABSOLUTE
    ..\..\..\..\..\..\components\ble\common\ble_advdata.c 0x00000000   Number         0  ble_advdata.o ABSOLUTE
    ..\..\..\..\..\..\components\ble\common\ble_conn_params.c 0x00000000   Number         0  ble_conn_params.o ABSOLUTE
    ..\..\..\..\..\..\components\ble\common\ble_conn_state.c 0x00000000   Number         0  ble_conn_state.o ABSOLUTE
    ..\..\..\..\..\..\components\ble\common\ble_srv_common.c 0x00000000   Number         0  ble_srv_common.o ABSOLUTE
    ..\..\..\..\..\..\components\ble\nrf_ble_gatt\nrf_ble_gatt.c 0x00000000   Number         0  nrf_ble_gatt.o ABSOLUTE
    ..\..\..\..\..\..\components\ble\nrf_ble_qwr\nrf_ble_qwr.c 0x00000000   Number         0  nrf_ble_qwr.o ABSOLUTE
    ..\..\..\..\..\..\components\boards\boards.c 0x00000000   Number         0  boards.o ABSOLUTE
    ..\..\..\..\..\..\components\libraries\atomic\nrf_atomic.c 0x00000000   Number         0  nrf_atomic.o ABSOLUTE
    ..\..\..\..\..\..\components\libraries\atomic_fifo\nrf_atfifo.c 0x00000000   Number         0  nrf_atfifo.o ABSOLUTE
    ..\..\..\..\..\..\components\libraries\atomic_flags\nrf_atflags.c 0x00000000   Number         0  nrf_atflags.o ABSOLUTE
    ..\..\..\..\..\..\components\libraries\balloc\nrf_balloc.c 0x00000000   Number         0  nrf_balloc.o ABSOLUTE
    ..\..\..\..\..\..\components\libraries\block_dev\sdc\nrf_block_dev_sdc.c 0x00000000   Number         0  nrf_block_dev_sdc.o ABSOLUTE
    ..\..\..\..\..\..\components\libraries\bsp\bsp.c 0x00000000   Number         0  bsp.o ABSOLUTE
    ..\..\..\..\..\..\components\libraries\bsp\bsp_btn_ble.c 0x00000000   Number         0  bsp_btn_ble.o ABSOLUTE
    ..\..\..\..\..\..\components\libraries\button\app_button.c 0x00000000   Number         0  app_button.o ABSOLUTE
    ..\..\..\..\..\..\components\libraries\experimental_section_vars\nrf_section_iter.c 0x00000000   Number         0  nrf_section_iter.o ABSOLUTE
    ..\..\..\..\..\..\components\libraries\fifo\app_fifo.c 0x00000000   Number         0  app_fifo.o ABSOLUTE
    ..\..\..\..\..\..\components\libraries\hardfault\hardfault_implementation.c 0x00000000   Number         0  hardfault_implementation.o ABSOLUTE
    ..\..\..\..\..\..\components\libraries\log\src\nrf_log_backend_rtt.c 0x00000000   Number         0  nrf_log_backend_rtt.o ABSOLUTE
    ..\..\..\..\..\..\components\libraries\log\src\nrf_log_backend_serial.c 0x00000000   Number         0  nrf_log_backend_serial.o ABSOLUTE
    ..\..\..\..\..\..\components\libraries\log\src\nrf_log_backend_uart.c 0x00000000   Number         0  nrf_log_backend_uart.o ABSOLUTE
    ..\..\..\..\..\..\components\libraries\log\src\nrf_log_default_backends.c 0x00000000   Number         0  nrf_log_default_backends.o ABSOLUTE
    ..\..\..\..\..\..\components\libraries\log\src\nrf_log_frontend.c 0x00000000   Number         0  nrf_log_frontend.o ABSOLUTE
    ..\..\..\..\..\..\components\libraries\log\src\nrf_log_str_formatter.c 0x00000000   Number         0  nrf_log_str_formatter.o ABSOLUTE
    ..\..\..\..\..\..\components\libraries\memobj\nrf_memobj.c 0x00000000   Number         0  nrf_memobj.o ABSOLUTE
    ..\..\..\..\..\..\components\libraries\pwr_mgmt\nrf_pwr_mgmt.c 0x00000000   Number         0  nrf_pwr_mgmt.o ABSOLUTE
    ..\..\..\..\..\..\components\libraries\ringbuf\nrf_ringbuf.c 0x00000000   Number         0  nrf_ringbuf.o ABSOLUTE
    ..\..\..\..\..\..\components\libraries\scheduler\app_scheduler.c 0x00000000   Number         0  app_scheduler.o ABSOLUTE
    ..\..\..\..\..\..\components\libraries\sdcard\app_sdcard.c 0x00000000   Number         0  app_sdcard.o ABSOLUTE
    ..\..\..\..\..\..\components\libraries\sortlist\nrf_sortlist.c 0x00000000   Number         0  nrf_sortlist.o ABSOLUTE
    ..\..\..\..\..\..\components\libraries\strerror\nrf_strerror.c 0x00000000   Number         0  nrf_strerror.o ABSOLUTE
    ..\..\..\..\..\..\components\libraries\timer\app_timer2.c 0x00000000   Number         0  app_timer2.o ABSOLUTE
    ..\..\..\..\..\..\components\libraries\timer\drv_rtc.c 0x00000000   Number         0  drv_rtc.o ABSOLUTE
    ..\..\..\..\..\..\components\libraries\uart\app_uart_fifo.c 0x00000000   Number         0  app_uart_fifo.o ABSOLUTE
    ..\..\..\..\..\..\components\libraries\uart\retarget.c 0x00000000   Number         0  retarget.o ABSOLUTE
    ..\..\..\..\..\..\components\libraries\util\app_error.c 0x00000000   Number         0  app_error.o ABSOLUTE
    ..\..\..\..\..\..\components\libraries\util\app_error_handler_keil.c 0x00000000   Number         0  app_error_handler_keil.o ABSOLUTE
    ..\..\..\..\..\..\components\libraries\util\app_error_weak.c 0x00000000   Number         0  app_error_weak.o ABSOLUTE
    ..\..\..\..\..\..\components\libraries\util\app_util_platform.c 0x00000000   Number         0  app_util_platform.o ABSOLUTE
    ..\..\..\..\..\..\components\libraries\util\nrf_assert.c 0x00000000   Number         0  nrf_assert.o ABSOLUTE
    ..\..\..\..\..\..\components\softdevice\common\nrf_sdh.c 0x00000000   Number         0  nrf_sdh.o ABSOLUTE
    ..\..\..\..\..\..\components\softdevice\common\nrf_sdh_ble.c 0x00000000   Number         0  nrf_sdh_ble.o ABSOLUTE
    ..\..\..\..\..\..\components\softdevice\common\nrf_sdh_soc.c 0x00000000   Number         0  nrf_sdh_soc.o ABSOLUTE
    ..\..\..\..\..\..\external\fatfs\port\diskio_blkdev.c 0x00000000   Number         0  diskio_blkdev.o ABSOLUTE
    ..\..\..\..\..\..\external\fatfs\src\ff.c 0x00000000   Number         0  ff.o ABSOLUTE
    ..\..\..\..\..\..\external\fprintf\nrf_fprintf.c 0x00000000   Number         0  nrf_fprintf.o ABSOLUTE
    ..\..\..\..\..\..\external\fprintf\nrf_fprintf_format.c 0x00000000   Number         0  nrf_fprintf_format.o ABSOLUTE
    ..\..\..\..\..\..\external\segger_rtt\SEGGER_RTT.c 0x00000000   Number         0  segger_rtt.o ABSOLUTE
    ..\..\..\..\..\..\external\segger_rtt\SEGGER_RTT_Syscalls_KEIL.c 0x00000000   Number         0  segger_rtt_syscalls_keil.o ABSOLUTE
    ..\..\..\..\..\..\external\segger_rtt\SEGGER_RTT_printf.c 0x00000000   Number         0  segger_rtt_printf.o ABSOLUTE
    ..\..\..\..\..\..\external\utf_converter\utf.c 0x00000000   Number         0  utf.o ABSOLUTE
    ..\..\..\..\..\..\integration\nrfx\legacy\nrf_drv_clock.c 0x00000000   Number         0  nrf_drv_clock.o ABSOLUTE
    ..\..\..\..\..\..\integration\nrfx\legacy\nrf_drv_spi.c 0x00000000   Number         0  nrf_drv_spi.o ABSOLUTE
    ..\..\..\..\..\..\integration\nrfx\legacy\nrf_drv_uart.c 0x00000000   Number         0  nrf_drv_uart.o ABSOLUTE
    ..\..\..\..\..\..\modules\nrfx\drivers\src\nrfx_clock.c 0x00000000   Number         0  nrfx_clock.o ABSOLUTE
    ..\..\..\..\..\..\modules\nrfx\drivers\src\nrfx_gpiote.c 0x00000000   Number         0  nrfx_gpiote.o ABSOLUTE
    ..\..\..\..\..\..\modules\nrfx\drivers\src\nrfx_spi.c 0x00000000   Number         0  nrfx_spi.o ABSOLUTE
    ..\..\..\..\..\..\modules\nrfx\drivers\src\nrfx_spim.c 0x00000000   Number         0  nrfx_spim.o ABSOLUTE
    ..\..\..\..\..\..\modules\nrfx\drivers\src\nrfx_uart.c 0x00000000   Number         0  nrfx_uart.o ABSOLUTE
    ..\..\..\..\..\..\modules\nrfx\drivers\src\nrfx_uarte.c 0x00000000   Number         0  nrfx_uarte.o ABSOLUTE
    ..\..\..\..\..\..\modules\nrfx\drivers\src\prs\nrfx_prs.c 0x00000000   Number         0  nrfx_prs.o ABSOLUTE
    ..\..\..\..\..\..\modules\nrfx\soc\nrfx_atomic.c 0x00000000   Number         0  nrfx_atomic.o ABSOLUTE
    ..\..\..\main.c                          0x00000000   Number         0  main.o ABSOLUTE
    ..\\..\\..\\..\\..\\..\\components\\ble\\ble_advertising\\ble_advertising.c 0x00000000   Number         0  ble_advertising.o ABSOLUTE
    ..\\..\\..\\..\\..\\..\\components\\ble\\ble_link_ctx_manager\\ble_link_ctx_manager.c 0x00000000   Number         0  ble_link_ctx_manager.o ABSOLUTE
    ..\\..\\..\\..\\..\\..\\components\\ble\\ble_services\\ble_nus\\ble_nus.c 0x00000000   Number         0  ble_nus.o ABSOLUTE
    ..\\..\\..\\..\\..\\..\\components\\ble\\common\\ble_advdata.c 0x00000000   Number         0  ble_advdata.o ABSOLUTE
    ..\\..\\..\\..\\..\\..\\components\\ble\\common\\ble_conn_params.c 0x00000000   Number         0  ble_conn_params.o ABSOLUTE
    ..\\..\\..\\..\\..\\..\\components\\ble\\common\\ble_conn_state.c 0x00000000   Number         0  ble_conn_state.o ABSOLUTE
    ..\\..\\..\\..\\..\\..\\components\\ble\\common\\ble_srv_common.c 0x00000000   Number         0  ble_srv_common.o ABSOLUTE
    ..\\..\\..\\..\\..\\..\\components\\ble\\nrf_ble_gatt\\nrf_ble_gatt.c 0x00000000   Number         0  nrf_ble_gatt.o ABSOLUTE
    ..\\..\\..\\..\\..\\..\\components\\ble\\nrf_ble_qwr\\nrf_ble_qwr.c 0x00000000   Number         0  nrf_ble_qwr.o ABSOLUTE
    ..\\..\\..\\..\\..\\..\\components\\boards\\boards.c 0x00000000   Number         0  boards.o ABSOLUTE
    ..\\..\\..\\..\\..\\..\\components\\libraries\\atomic\\nrf_atomic.c 0x00000000   Number         0  nrf_atomic.o ABSOLUTE
    ..\\..\\..\\..\\..\\..\\components\\libraries\\atomic_fifo\\nrf_atfifo.c 0x00000000   Number         0  nrf_atfifo.o ABSOLUTE
    ..\\..\\..\\..\\..\\..\\components\\libraries\\atomic_flags\\nrf_atflags.c 0x00000000   Number         0  nrf_atflags.o ABSOLUTE
    ..\\..\\..\\..\\..\\..\\components\\libraries\\balloc\\nrf_balloc.c 0x00000000   Number         0  nrf_balloc.o ABSOLUTE
    ..\\..\\..\\..\\..\\..\\components\\libraries\\block_dev\\sdc\\nrf_block_dev_sdc.c 0x00000000   Number         0  nrf_block_dev_sdc.o ABSOLUTE
    ..\\..\\..\\..\\..\\..\\components\\libraries\\bsp\\bsp.c 0x00000000   Number         0  bsp.o ABSOLUTE
    ..\\..\\..\\..\\..\\..\\components\\libraries\\bsp\\bsp_btn_ble.c 0x00000000   Number         0  bsp_btn_ble.o ABSOLUTE
    ..\\..\\..\\..\\..\\..\\components\\libraries\\button\\app_button.c 0x00000000   Number         0  app_button.o ABSOLUTE
    ..\\..\\..\\..\\..\\..\\components\\libraries\\experimental_section_vars\\nrf_section_iter.c 0x00000000   Number         0  nrf_section_iter.o ABSOLUTE
    ..\\..\\..\\..\\..\\..\\components\\libraries\\fifo\\app_fifo.c 0x00000000   Number         0  app_fifo.o ABSOLUTE
    ..\\..\\..\\..\\..\\..\\components\\libraries\\hardfault\\hardfault_implementation.c 0x00000000   Number         0  hardfault_implementation.o ABSOLUTE
    ..\\..\\..\\..\\..\\..\\components\\libraries\\log\\src\\nrf_log_backend_rtt.c 0x00000000   Number         0  nrf_log_backend_rtt.o ABSOLUTE
    ..\\..\\..\\..\\..\\..\\components\\libraries\\log\\src\\nrf_log_backend_serial.c 0x00000000   Number         0  nrf_log_backend_serial.o ABSOLUTE
    ..\\..\\..\\..\\..\\..\\components\\libraries\\log\\src\\nrf_log_backend_uart.c 0x00000000   Number         0  nrf_log_backend_uart.o ABSOLUTE
    ..\\..\\..\\..\\..\\..\\components\\libraries\\log\\src\\nrf_log_default_backends.c 0x00000000   Number         0  nrf_log_default_backends.o ABSOLUTE
    ..\\..\\..\\..\\..\\..\\components\\libraries\\log\\src\\nrf_log_frontend.c 0x00000000   Number         0  nrf_log_frontend.o ABSOLUTE
    ..\\..\\..\\..\\..\\..\\components\\libraries\\log\\src\\nrf_log_str_formatter.c 0x00000000   Number         0  nrf_log_str_formatter.o ABSOLUTE
    ..\\..\\..\\..\\..\\..\\components\\libraries\\memobj\\nrf_memobj.c 0x00000000   Number         0  nrf_memobj.o ABSOLUTE
    ..\\..\\..\\..\\..\\..\\components\\libraries\\pwr_mgmt\\nrf_pwr_mgmt.c 0x00000000   Number         0  nrf_pwr_mgmt.o ABSOLUTE
    ..\\..\\..\\..\\..\\..\\components\\libraries\\ringbuf\\nrf_ringbuf.c 0x00000000   Number         0  nrf_ringbuf.o ABSOLUTE
    ..\\..\\..\\..\\..\\..\\components\\libraries\\scheduler\\app_scheduler.c 0x00000000   Number         0  app_scheduler.o ABSOLUTE
    ..\\..\\..\\..\\..\\..\\components\\libraries\\sdcard\\app_sdcard.c 0x00000000   Number         0  app_sdcard.o ABSOLUTE
    ..\\..\\..\\..\\..\\..\\components\\libraries\\sortlist\\nrf_sortlist.c 0x00000000   Number         0  nrf_sortlist.o ABSOLUTE
    ..\\..\\..\\..\\..\\..\\components\\libraries\\strerror\\nrf_strerror.c 0x00000000   Number         0  nrf_strerror.o ABSOLUTE
    ..\\..\\..\\..\\..\\..\\components\\libraries\\timer\\app_timer2.c 0x00000000   Number         0  app_timer2.o ABSOLUTE
    ..\\..\\..\\..\\..\\..\\components\\libraries\\timer\\drv_rtc.c 0x00000000   Number         0  drv_rtc.o ABSOLUTE
    ..\\..\\..\\..\\..\\..\\components\\libraries\\uart\\app_uart_fifo.c 0x00000000   Number         0  app_uart_fifo.o ABSOLUTE
    ..\\..\\..\\..\\..\\..\\components\\libraries\\uart\\retarget.c 0x00000000   Number         0  retarget.o ABSOLUTE
    ..\\..\\..\\..\\..\\..\\components\\libraries\\util\\app_error.c 0x00000000   Number         0  app_error.o ABSOLUTE
    ..\\..\\..\\..\\..\\..\\components\\libraries\\util\\app_error_handler_keil.c 0x00000000   Number         0  app_error_handler_keil.o ABSOLUTE
    ..\\..\\..\\..\\..\\..\\components\\libraries\\util\\app_error_weak.c 0x00000000   Number         0  app_error_weak.o ABSOLUTE
    ..\\..\\..\\..\\..\\..\\components\\libraries\\util\\app_util_platform.c 0x00000000   Number         0  app_util_platform.o ABSOLUTE
    ..\\..\\..\\..\\..\\..\\components\\libraries\\util\\nrf_assert.c 0x00000000   Number         0  nrf_assert.o ABSOLUTE
    ..\\..\\..\\..\\..\\..\\components\\softdevice\\common\\nrf_sdh.c 0x00000000   Number         0  nrf_sdh.o ABSOLUTE
    ..\\..\\..\\..\\..\\..\\components\\softdevice\\common\\nrf_sdh_ble.c 0x00000000   Number         0  nrf_sdh_ble.o ABSOLUTE
    ..\\..\\..\\..\\..\\..\\components\\softdevice\\common\\nrf_sdh_soc.c 0x00000000   Number         0  nrf_sdh_soc.o ABSOLUTE
    ..\\..\\..\\..\\..\\..\\external\\fatfs\\port\\diskio_blkdev.c 0x00000000   Number         0  diskio_blkdev.o ABSOLUTE
    ..\\..\\..\\..\\..\\..\\external\\fprintf\\nrf_fprintf.c 0x00000000   Number         0  nrf_fprintf.o ABSOLUTE
    ..\\..\\..\\..\\..\\..\\external\\fprintf\\nrf_fprintf_format.c 0x00000000   Number         0  nrf_fprintf_format.o ABSOLUTE
    ..\\..\\..\\..\\..\\..\\external\\segger_rtt\\SEGGER_RTT.c 0x00000000   Number         0  segger_rtt.o ABSOLUTE
    ..\\..\\..\\..\\..\\..\\external\\segger_rtt\\SEGGER_RTT_printf.c 0x00000000   Number         0  segger_rtt_printf.o ABSOLUTE
    ..\\..\\..\\..\\..\\..\\integration\\nrfx\\legacy\\nrf_drv_clock.c 0x00000000   Number         0  nrf_drv_clock.o ABSOLUTE
    ..\\..\\..\\..\\..\\..\\integration\\nrfx\\legacy\\nrf_drv_spi.c 0x00000000   Number         0  nrf_drv_spi.o ABSOLUTE
    ..\\..\\..\\..\\..\\..\\integration\\nrfx\\legacy\\nrf_drv_uart.c 0x00000000   Number         0  nrf_drv_uart.o ABSOLUTE
    ..\\..\\..\\..\\..\\..\\modules\\nrfx\\drivers\\src\\nrfx_clock.c 0x00000000   Number         0  nrfx_clock.o ABSOLUTE
    ..\\..\\..\\..\\..\\..\\modules\\nrfx\\drivers\\src\\nrfx_gpiote.c 0x00000000   Number         0  nrfx_gpiote.o ABSOLUTE
    ..\\..\\..\\..\\..\\..\\modules\\nrfx\\drivers\\src\\nrfx_spi.c 0x00000000   Number         0  nrfx_spi.o ABSOLUTE
    ..\\..\\..\\..\\..\\..\\modules\\nrfx\\drivers\\src\\nrfx_spim.c 0x00000000   Number         0  nrfx_spim.o ABSOLUTE
    ..\\..\\..\\..\\..\\..\\modules\\nrfx\\drivers\\src\\nrfx_uart.c 0x00000000   Number         0  nrfx_uart.o ABSOLUTE
    ..\\..\\..\\..\\..\\..\\modules\\nrfx\\drivers\\src\\nrfx_uarte.c 0x00000000   Number         0  nrfx_uarte.o ABSOLUTE
    ..\\..\\..\\..\\..\\..\\modules\\nrfx\\drivers\\src\\prs\\nrfx_prs.c 0x00000000   Number         0  nrfx_prs.o ABSOLUTE
    ..\\..\\..\\..\\..\\..\\modules\\nrfx\\soc\\nrfx_atomic.c 0x00000000   Number         0  nrfx_atomic.o ABSOLUTE
    ..\\..\\..\\main.c                       0x00000000   Number         0  main.o ABSOLUTE
    RTE\Device\nRF52832_xxAA\arm_startup_nrf52.s 0x00000000   Number         0  arm_startup_nrf52.o ABSOLUTE
    RTE\Device\nRF52832_xxAA\system_nrf52.c  0x00000000   Number         0  system_nrf52.o ABSOLUTE
    RTE\\Device\\nRF52832_xxAA\\system_nrf52.c 0x00000000   Number         0  system_nrf52.o ABSOLUTE
    cdrcmple.s                               0x00000000   Number         0  cdrcmple.o ABSOLUTE
    dc.s                                     0x00000000   Number         0  dc.o ABSOLUTE
    handlers.s                               0x00000000   Number         0  handlers.o ABSOLUTE
    init.s                                   0x00000000   Number         0  init.o ABSOLUTE
    RESET                                    0x00026000   Section      512  arm_startup_nrf52.o(RESET)
    .ARM.Collect$$$$00000000                 0x00026200   Section        0  entry.o(.ARM.Collect$$$$00000000)
    .ARM.Collect$$$$00000001                 0x00026200   Section        4  entry2.o(.ARM.Collect$$$$00000001)
    .ARM.Collect$$$$00000004                 0x00026204   Section        4  entry5.o(.ARM.Collect$$$$00000004)
    .ARM.Collect$$$$00000008                 0x00026208   Section        0  entry7b.o(.ARM.Collect$$$$00000008)
    .ARM.Collect$$$$0000000A                 0x00026208   Section        0  entry8b.o(.ARM.Collect$$$$0000000A)
    .ARM.Collect$$$$0000000B                 0x00026208   Section        8  entry9a.o(.ARM.Collect$$$$0000000B)
    .ARM.Collect$$$$0000000D                 0x00026210   Section        0  entry10a.o(.ARM.Collect$$$$0000000D)
    .ARM.Collect$$$$0000000F                 0x00026210   Section        0  entry11a.o(.ARM.Collect$$$$0000000F)
    .ARM.Collect$$$$00002712                 0x00026210   Section        4  entry2.o(.ARM.Collect$$$$00002712)
    __lit__00000000                          0x00026210   Data           4  entry2.o(.ARM.Collect$$$$00002712)
    .emb_text                                0x00026214   Section      200  nrf_atfifo.o(.emb_text)
    $v0                                      0x00026214   Number         0  nrf_atfifo.o(.emb_text)
    .emb_text                                0x000262dc   Section      226  nrf_atomic.o(.emb_text)
    $v0                                      0x000262dc   Number         0  nrf_atomic.o(.emb_text)
    .text                                    0x000263c0   Section       36  arm_startup_nrf52.o(.text)
    $v0                                      0x000263c0   Number         0  arm_startup_nrf52.o(.text)
    .text                                    0x000263e4   Section        0  uldiv.o(.text)
    .text                                    0x00026446   Section        0  llshl.o(.text)
    .text                                    0x00026464   Section        0  ctype_o.o(.text)
    .text                                    0x0002646c   Section        0  memcpya.o(.text)
    .text                                    0x00026490   Section        0  memseta.o(.text)
    .text                                    0x000264b4   Section        0  strlen.o(.text)
    .text                                    0x000264c2   Section        0  strcpy.o(.text)
    .text                                    0x000264d4   Section        0  uidiv.o(.text)
    .text                                    0x00026500   Section        0  llushr.o(.text)
    .text                                    0x00026520   Section       36  init.o(.text)
    .text                                    0x00026544   Section        0  __dczerorl2.o(.text)
    i.GPIOTE_IRQHandler                      0x0002659c   Section        0  nrfx_gpiote.o(i.GPIOTE_IRQHandler)
    i.POWER_CLOCK_IRQHandler                 0x00026640   Section        0  nrfx_clock.o(i.POWER_CLOCK_IRQHandler)
    i.RTC1_IRQHandler                        0x00026698   Section        0  drv_rtc.o(i.RTC1_IRQHandler)
    i.SEGGER_RTT_Init                        0x000266a8   Section        0  segger_rtt.o(i.SEGGER_RTT_Init)
    i.SEGGER_RTT_WriteNoLock                 0x000266ac   Section        0  segger_rtt.o(i.SEGGER_RTT_WriteNoLock)
    i.SPIM0_SPIS0_TWIM0_TWIS0_SPI0_TWI0_IRQHandler 0x00026708   Section        0  nrfx_spim.o(i.SPIM0_SPIS0_TWIM0_TWIS0_SPI0_TWI0_IRQHandler)
    i.SWI2_EGU2_IRQHandler                   0x0002675c   Section        0  nrf_sdh.o(i.SWI2_EGU2_IRQHandler)
    i.SystemInit                             0x00026760   Section        0  system_nrf52.o(i.SystemInit)
    i.TIMER2_IRQHandler                      0x000267e4   Section        0  main.o(i.TIMER2_IRQHandler)
    i.UARTE0_UART0_IRQHandler                0x00026874   Section        0  nrfx_prs.o(i.UARTE0_UART0_IRQHandler)
    i._DoInit                                0x00026880   Section        0  segger_rtt.o(i._DoInit)
    _DoInit                                  0x00026881   Thumb Code    76  segger_rtt.o(i._DoInit)
    i._GetAvailWriteSpace                    0x000268e8   Section        0  segger_rtt.o(i._GetAvailWriteSpace)
    _GetAvailWriteSpace                      0x000268e9   Thumb Code    22  segger_rtt.o(i._GetAvailWriteSpace)
    i._WriteBlocking                         0x000268fe   Section        0  segger_rtt.o(i._WriteBlocking)
    _WriteBlocking                           0x000268ff   Thumb Code    90  segger_rtt.o(i._WriteBlocking)
    i._WriteNoCheck                          0x00026958   Section        0  segger_rtt.o(i._WriteNoCheck)
    _WriteNoCheck                            0x00026959   Thumb Code    66  segger_rtt.o(i._WriteNoCheck)
    i.__0sprintf$1                           0x0002699c   Section        0  printf1.o(i.__0sprintf$1)
    i.__scatterload_copy                     0x000269c4   Section       14  handlers.o(i.__scatterload_copy)
    i.__scatterload_null                     0x000269d2   Section        2  handlers.o(i.__scatterload_null)
    i.__scatterload_zeroinit                 0x000269d4   Section       14  handlers.o(i.__scatterload_zeroinit)
    i.__sd_nvic_app_accessible_irq           0x000269e4   Section        0  nrf_sdh.o(i.__sd_nvic_app_accessible_irq)
    __sd_nvic_app_accessible_irq             0x000269e5   Thumb Code    32  nrf_sdh.o(i.__sd_nvic_app_accessible_irq)
    i._printf_core                           0x00026a08   Section        0  printf1.o(i._printf_core)
    _printf_core                             0x00026a09   Thumb Code   336  printf1.o(i._printf_core)
    i._sputc                                 0x00026b5c   Section        0  printf1.o(i._sputc)
    _sputc                                   0x00026b5d   Thumb Code    10  printf1.o(i._sputc)
    i.adv_set_data_size_max_get              0x00026b66   Section        0  ble_advertising.o(i.adv_set_data_size_max_get)
    adv_set_data_size_max_get                0x00026b67   Thumb Code    16  ble_advertising.o(i.adv_set_data_size_max_get)
    i.advertising_buttons_configure          0x00026b76   Section        0  bsp_btn_ble.o(i.advertising_buttons_configure)
    advertising_buttons_configure            0x00026b77   Thumb Code    54  bsp_btn_ble.o(i.advertising_buttons_configure)
    i.app_error_fault_handler                0x00026bac   Section        0  app_error_weak.o(i.app_error_fault_handler)
    i.app_error_handler_bare                 0x00026c30   Section        0  app_error.o(i.app_error_handler_bare)
    i.app_fifo_get                           0x00026c46   Section        0  app_fifo.o(i.app_fifo_get)
    i.app_fifo_put                           0x00026c5c   Section        0  app_fifo.o(i.app_fifo_put)
    i.app_sdc_block_read                     0x00026c78   Section        0  app_sdcard.o(i.app_sdc_block_read)
    i.app_sdc_block_write                    0x00026cd0   Section        0  app_sdcard.o(i.app_sdc_block_write)
    i.app_sdc_busy_check                     0x00026d3c   Section        0  app_sdcard.o(i.app_sdc_busy_check)
    i.app_sdc_info_get                       0x00026d58   Section        0  app_sdcard.o(i.app_sdc_info_get)
    i.app_sdc_init                           0x00026d70   Section        0  app_sdcard.o(i.app_sdc_init)
    i.app_sdc_uninit                         0x00026e3c   Section        0  app_sdcard.o(i.app_sdc_uninit)
    i.app_timer_create                       0x00026e84   Section        0  app_timer2.o(i.app_timer_create)
    i.app_timer_start                        0x00026e9a   Section        0  app_timer2.o(i.app_timer_start)
    i.app_timer_stop                         0x00026eca   Section        0  app_timer2.o(i.app_timer_stop)
    i.app_uart_put                           0x00026ed8   Section        0  app_uart_fifo.o(i.app_uart_put)
    i.app_util_critical_region_enter         0x00026f2c   Section        0  app_util_platform.o(i.app_util_critical_region_enter)
    i.app_util_critical_region_exit          0x00026f74   Section        0  app_util_platform.o(i.app_util_critical_region_exit)
    i.apply_config                           0x00026fa8   Section        0  nrfx_uart.o(i.apply_config)
    apply_config                             0x00026fa9   Thumb Code   136  nrfx_uart.o(i.apply_config)
    i.apply_config                           0x00027030   Section        0  nrfx_uarte.o(i.apply_config)
    apply_config                             0x00027031   Thumb Code   136  nrfx_uarte.o(i.apply_config)
    i.blcm_link_ctx_get                      0x000270b8   Section        0  ble_link_ctx_manager.o(i.blcm_link_ctx_get)
    i.ble_advdata_encode                     0x00027100   Section        0  ble_advdata.o(i.ble_advdata_encode)
    i.ble_advdata_parse                      0x00027282   Section        0  ble_advdata.o(i.ble_advdata_parse)
    i.ble_advdata_search                     0x000272a2   Section        0  ble_advdata.o(i.ble_advdata_search)
    i.ble_advertising_conn_cfg_tag_set       0x000272e8   Section        0  ble_advertising.o(i.ble_advertising_conn_cfg_tag_set)
    i.ble_advertising_init                   0x000272ee   Section        0  ble_advertising.o(i.ble_advertising_init)
    i.ble_advertising_on_ble_evt             0x000273e6   Section        0  ble_advertising.o(i.ble_advertising_on_ble_evt)
    i.ble_advertising_start                  0x00027450   Section        0  ble_advertising.o(i.ble_advertising_start)
    i.ble_conn_params_init                   0x00027680   Section        0  ble_conn_params.o(i.ble_conn_params_init)
    i.ble_conn_state_conn_idx                0x000276e8   Section        0  ble_conn_state.o(i.ble_conn_state_conn_idx)
    i.ble_conn_state_valid                   0x000276fc   Section        0  ble_conn_state.o(i.ble_conn_state_valid)
    i.ble_device_addr_encode                 0x00027710   Section        0  ble_advdata.o(i.ble_device_addr_encode)
    ble_device_addr_encode                   0x00027711   Thumb Code    96  ble_advdata.o(i.ble_device_addr_encode)
    i.ble_evt_handler                        0x00027770   Section        0  main.o(i.ble_evt_handler)
    ble_evt_handler                          0x00027771   Thumb Code   174  main.o(i.ble_evt_handler)
    i.ble_evt_handler                        0x0002784c   Section        0  bsp_btn_ble.o(i.ble_evt_handler)
    ble_evt_handler                          0x0002784d   Thumb Code   106  bsp_btn_ble.o(i.ble_evt_handler)
    i.ble_evt_handler                        0x000278bc   Section        0  ble_conn_params.o(i.ble_evt_handler)
    ble_evt_handler                          0x000278bd   Thumb Code   242  ble_conn_params.o(i.ble_evt_handler)
    i.ble_evt_handler                        0x000279b8   Section        0  ble_conn_state.o(i.ble_evt_handler)
    ble_evt_handler                          0x000279b9   Thumb Code   274  ble_conn_state.o(i.ble_evt_handler)
    i.ble_nus_init                           0x00027ad0   Section        0  ble_nus.o(i.ble_nus_init)
    i.ble_nus_on_ble_evt                     0x00027ba4   Section        0  ble_nus.o(i.ble_nus_on_ble_evt)
    i.ble_srv_is_notification_enabled        0x00027c1a   Section        0  ble_srv_common.o(i.ble_srv_is_notification_enabled)
    i.block_dev_handler                      0x00027c24   Section        0  diskio_blkdev.o(i.block_dev_handler)
    block_dev_handler                        0x00027c25   Thumb Code    40  diskio_blkdev.o(i.block_dev_handler)
    i.block_dev_sdc_geometry                 0x00027c50   Section        0  nrf_block_dev_sdc.o(i.block_dev_sdc_geometry)
    block_dev_sdc_geometry                   0x00027c51   Thumb Code     4  nrf_block_dev_sdc.o(i.block_dev_sdc_geometry)
    i.block_dev_sdc_init                     0x00027c54   Section        0  nrf_block_dev_sdc.o(i.block_dev_sdc_init)
    block_dev_sdc_init                       0x00027c55   Thumb Code   104  nrf_block_dev_sdc.o(i.block_dev_sdc_init)
    i.block_dev_sdc_ioctl                    0x00027cc8   Section        0  nrf_block_dev_sdc.o(i.block_dev_sdc_ioctl)
    block_dev_sdc_ioctl                      0x00027cc9   Thumb Code    32  nrf_block_dev_sdc.o(i.block_dev_sdc_ioctl)
    i.block_dev_sdc_read_req                 0x00027ce8   Section        0  nrf_block_dev_sdc.o(i.block_dev_sdc_read_req)
    block_dev_sdc_read_req                   0x00027ce9   Thumb Code   116  nrf_block_dev_sdc.o(i.block_dev_sdc_read_req)
    i.block_dev_sdc_uninit                   0x00027d64   Section        0  nrf_block_dev_sdc.o(i.block_dev_sdc_uninit)
    block_dev_sdc_uninit                     0x00027d65   Thumb Code    74  nrf_block_dev_sdc.o(i.block_dev_sdc_uninit)
    i.block_dev_sdc_write_req                0x00027db8   Section        0  nrf_block_dev_sdc.o(i.block_dev_sdc_write_req)
    block_dev_sdc_write_req                  0x00027db9   Thumb Code   116  nrf_block_dev_sdc.o(i.block_dev_sdc_write_req)
    i.bsp_board_button_idx_to_pin            0x00027e34   Section        0  boards.o(i.bsp_board_button_idx_to_pin)
    i.bsp_board_led_invert                   0x00027e40   Section        0  boards.o(i.bsp_board_led_invert)
    i.bsp_board_led_off                      0x00027e64   Section        0  boards.o(i.bsp_board_led_off)
    i.bsp_board_led_on                       0x00027e74   Section        0  boards.o(i.bsp_board_led_on)
    i.bsp_board_led_state_get                0x00027e84   Section        0  boards.o(i.bsp_board_led_state_get)
    i.bsp_board_leds_off                     0x00027ea4   Section        0  boards.o(i.bsp_board_leds_off)
    i.bsp_board_leds_on                      0x00027eb6   Section        0  boards.o(i.bsp_board_leds_on)
    i.bsp_board_pin_to_button_idx            0x00027ec8   Section        0  boards.o(i.bsp_board_pin_to_button_idx)
    i.bsp_btn_ble_sleep_mode_prepare         0x00027eec   Section        0  bsp_btn_ble.o(i.bsp_btn_ble_sleep_mode_prepare)
    i.bsp_button_event_handler               0x00027f0c   Section        0  bsp.o(i.bsp_button_event_handler)
    bsp_button_event_handler                 0x00027f0d   Thumb Code   132  bsp.o(i.bsp_button_event_handler)
    i.bsp_event_to_button_action_assign      0x00027f9c   Section        0  bsp.o(i.bsp_event_to_button_action_assign)
    i.bsp_indication_set                     0x00027fe0   Section        0  bsp.o(i.bsp_indication_set)
    i.bsp_led_indication                     0x00027ff8   Section        0  bsp.o(i.bsp_led_indication)
    bsp_led_indication                       0x00027ff9   Thumb Code   446  bsp.o(i.bsp_led_indication)
    i.bsp_wakeup_button_enable               0x000281c0   Section        0  bsp.o(i.bsp_wakeup_button_enable)
    i.buf_prealloc                           0x000281c8   Section        0  nrf_log_frontend.o(i.buf_prealloc)
    buf_prealloc                             0x000281c9   Thumb Code   140  nrf_log_frontend.o(i.buf_prealloc)
    i.buffer_add                             0x0002825c   Section        0  nrf_fprintf_format.o(i.buffer_add)
    buffer_add                               0x0002825d   Thumb Code    46  nrf_fprintf_format.o(i.buffer_add)
    i.buffer_is_empty                        0x0002828c   Section        0  nrf_log_frontend.o(i.buffer_is_empty)
    i.channel_port_get                       0x000282a4   Section        0  nrfx_gpiote.o(i.channel_port_get)
    channel_port_get                         0x000282a5   Thumb Code    10  nrfx_gpiote.o(i.channel_port_get)
    i.characteristic_add                     0x000282b4   Section        0  ble_srv_common.o(i.characteristic_add)
    i.check_fs                               0x00028444   Section        0  ff.o(i.check_fs)
    check_fs                                 0x00028445   Thumb Code   102  ff.o(i.check_fs)
    i.clock_clk_started_notify               0x000284b4   Section        0  nrf_drv_clock.o(i.clock_clk_started_notify)
    clock_clk_started_notify                 0x000284b5   Thumb Code    34  nrf_drv_clock.o(i.clock_clk_started_notify)
    i.clock_irq_handler                      0x000284dc   Section        0  nrf_drv_clock.o(i.clock_irq_handler)
    clock_irq_handler                        0x000284dd   Thumb Code    24  nrf_drv_clock.o(i.clock_irq_handler)
    i.clust2sect                             0x000284f8   Section        0  ff.o(i.clust2sect)
    clust2sect                               0x000284f9   Thumb Code    24  ff.o(i.clust2sect)
    i.compare_func                           0x00028510   Section        0  app_timer2.o(i.compare_func)
    compare_func                             0x00028511   Thumb Code    24  app_timer2.o(i.compare_func)
    i.conn_handle_list_get                   0x00028528   Section        0  ble_conn_state.o(i.conn_handle_list_get)
    i.conn_int_encode                        0x00028566   Section        0  ble_advdata.o(i.conn_int_encode)
    conn_int_encode                          0x00028567   Thumb Code   136  ble_advdata.o(i.conn_int_encode)
    i.conn_params_error_handler              0x000285ee   Section        0  main.o(i.conn_params_error_handler)
    conn_params_error_handler                0x000285ef   Thumb Code     4  main.o(i.conn_params_error_handler)
    i.conn_params_negotiation                0x000285f4   Section        0  ble_conn_params.o(i.conn_params_negotiation)
    conn_params_negotiation                  0x000285f5   Thumb Code    68  ble_conn_params.o(i.conn_params_negotiation)
    i.create_chain                           0x0002863c   Section        0  ff.o(i.create_chain)
    create_chain                             0x0002863d   Thumb Code   164  ff.o(i.create_chain)
    i.create_name                            0x000286e0   Section        0  ff.o(i.create_name)
    create_name                              0x000286e1   Thumb Code   210  ff.o(i.create_name)
    i.data_length_update                     0x000287c4   Section        0  nrf_ble_gatt.o(i.data_length_update)
    data_length_update                       0x000287c5   Thumb Code   110  nrf_ble_gatt.o(i.data_length_update)
    i.default_wait_func                      0x00028884   Section        0  diskio_blkdev.o(i.default_wait_func)
    default_wait_func                        0x00028885   Thumb Code     4  diskio_blkdev.o(i.default_wait_func)
    i.dir_find                               0x00028888   Section        0  ff.o(i.dir_find)
    dir_find                                 0x00028889   Thumb Code   100  ff.o(i.dir_find)
    i.dir_next                               0x000288ec   Section        0  ff.o(i.dir_next)
    dir_next                                 0x000288ed   Thumb Code   244  ff.o(i.dir_next)
    i.dir_read                               0x000289e0   Section        0  ff.o(i.dir_read)
    dir_read                                 0x000289e1   Thumb Code    96  ff.o(i.dir_read)
    i.dir_register                           0x00028a40   Section        0  ff.o(i.dir_register)
    dir_register                             0x00028a41   Thumb Code   102  ff.o(i.dir_register)
    i.dir_sdi                                0x00028aa6   Section        0  ff.o(i.dir_sdi)
    dir_sdi                                  0x00028aa7   Thumb Code   130  ff.o(i.dir_sdi)
    i.disk_initialize                        0x00028b28   Section        0  diskio_blkdev.o(i.disk_initialize)
    i.disk_ioctl                             0x00028ba8   Section        0  diskio_blkdev.o(i.disk_ioctl)
    i.disk_read                              0x00028c24   Section        0  diskio_blkdev.o(i.disk_read)
    i.disk_status                            0x00028ca0   Section        0  diskio_blkdev.o(i.disk_status)
    i.disk_write                             0x00028cc0   Section        0  diskio_blkdev.o(i.disk_write)
    i.diskio_blockdev_register               0x00028d48   Section        0  diskio_blkdev.o(i.diskio_blockdev_register)
    i.dropped_sat16_get                      0x00028d54   Section        0  nrf_log_frontend.o(i.dropped_sat16_get)
    dropped_sat16_get                        0x00028d55   Thumb Code    16  nrf_log_frontend.o(i.dropped_sat16_get)
    i.drv_rtc_counter_get                    0x00028d68   Section        0  drv_rtc.o(i.drv_rtc_counter_get)
    i.drv_rtc_irq_trigger                    0x00028d70   Section        0  drv_rtc.o(i.drv_rtc_irq_trigger)
    i.f_close                                0x00028d8e   Section        0  ff.o(i.f_close)
    i.f_mount                                0x00028dac   Section        0  ff.o(i.f_mount)
    i.f_open                                 0x00028df8   Section        0  ff.o(i.f_open)
    i.f_opendir                              0x00028fac   Section        0  ff.o(i.f_opendir)
    i.f_readdir                              0x0002900e   Section        0  ff.o(i.f_readdir)
    i.f_sync                                 0x00029050   Section        0  ff.o(i.f_sync)
    i.f_write                                0x000290e0   Section        0  ff.o(i.f_write)
    i.fatfs_example                          0x00029260   Section        0  main.o(i.fatfs_example)
    fatfs_example                            0x00029261   Thumb Code   374  main.o(i.fatfs_example)
    i.fifo_get                               0x0002958c   Section        0  app_fifo.o(i.fifo_get)
    fifo_get                                 0x0002958d   Thumb Code    20  app_fifo.o(i.fifo_get)
    i.fifo_put                               0x000295a0   Section        0  app_fifo.o(i.fifo_put)
    fifo_put                                 0x000295a1   Thumb Code    18  app_fifo.o(i.fifo_put)
    i.find_volume                            0x000295b4   Section        0  ff.o(i.find_volume)
    find_volume                              0x000295b5   Thumb Code   576  ff.o(i.find_volume)
    i.flag_toggle                            0x00029800   Section        0  ble_conn_state.o(i.flag_toggle)
    flag_toggle                              0x00029801   Thumb Code    10  ble_conn_state.o(i.flag_toggle)
    i.flags_set                              0x0002980a   Section        0  ble_advertising.o(i.flags_set)
    flags_set                                0x0002980b   Thumb Code    40  ble_advertising.o(i.flags_set)
    i.follow_path                            0x00029832   Section        0  ff.o(i.follow_path)
    follow_path                              0x00029833   Thumb Code   116  ff.o(i.follow_path)
    i.gatt_evt_handler                       0x000298a8   Section        0  main.o(i.gatt_evt_handler)
    i.gatt_init                              0x00029904   Section        0  main.o(i.gatt_init)
    i.get_fat                                0x00029934   Section        0  ff.o(i.get_fat)
    get_fat                                  0x00029935   Thumb Code   190  ff.o(i.get_fat)
    i.get_fileinfo                           0x000299f2   Section        0  ff.o(i.get_fileinfo)
    get_fileinfo                             0x000299f3   Thumb Code    98  ff.o(i.get_fileinfo)
    i.get_ldnumber                           0x00029a54   Section        0  ff.o(i.get_ldnumber)
    get_ldnumber                             0x00029a55   Thumb Code    60  ff.o(i.get_ldnumber)
    i.get_now                                0x00029a90   Section        0  app_timer2.o(i.get_now)
    get_now                                  0x00029a91   Thumb Code    46  app_timer2.o(i.get_now)
    i.instance_get                           0x00029ac4   Section        0  ble_conn_params.o(i.instance_get)
    instance_get                             0x00029ac5   Thumb Code    14  ble_conn_params.o(i.instance_get)
    i.int_print                              0x00029ad8   Section        0  nrf_fprintf_format.o(i.int_print)
    int_print                                0x00029ad9   Thumb Code   166  nrf_fprintf_format.o(i.int_print)
    i.interrupts_enable                      0x00029b80   Section        0  nrfx_uarte.o(i.interrupts_enable)
    interrupts_enable                        0x00029b81   Thumb Code   132  nrfx_uarte.o(i.interrupts_enable)
    i.invalid_packets_omit                   0x00029c08   Section        0  nrf_log_frontend.o(i.invalid_packets_omit)
    invalid_packets_omit                     0x00029c09   Thumb Code    52  nrf_log_frontend.o(i.invalid_packets_omit)
    i.is_conn_params_ok                      0x00029c3c   Section        0  ble_conn_params.o(i.is_conn_params_ok)
    is_conn_params_ok                        0x00029c3d   Thumb Code    68  ble_conn_params.o(i.is_conn_params_ok)
    i.ld_clust                               0x00029c80   Section        0  ff.o(i.ld_clust)
    ld_clust                                 0x00029c81   Thumb Code    38  ff.o(i.ld_clust)
    i.ld_dword                               0x00029ca6   Section        0  ff.o(i.ld_dword)
    ld_dword                                 0x00029ca7   Thumb Code    22  ff.o(i.ld_dword)
    i.ld_word                                0x00029cbc   Section        0  ff.o(i.ld_word)
    ld_word                                  0x00029cbd   Thumb Code    10  ff.o(i.ld_word)
    i.leds_off                               0x00029cc8   Section        0  bsp.o(i.leds_off)
    leds_off                                 0x00029cc9   Thumb Code    42  bsp.o(i.leds_off)
    i.link_init                              0x00029cf8   Section        0  nrf_ble_gatt.o(i.link_init)
    link_init                                0x00029cf9   Thumb Code    24  nrf_ble_gatt.o(i.link_init)
    i.log_skip                               0x00029d10   Section        0  nrf_log_frontend.o(i.log_skip)
    log_skip                                 0x00029d11   Thumb Code   150  nrf_log_frontend.o(i.log_skip)
    i.main                                   0x00029db4   Section        0  main.o(i.main)
    i.manuf_specific_data_encode             0x00029f94   Section        0  ble_advdata.o(i.manuf_specific_data_encode)
    manuf_specific_data_encode               0x00029f95   Thumb Code   100  ble_advdata.o(i.manuf_specific_data_encode)
    i.mem_cpy                                0x00029ff8   Section        0  ff.o(i.mem_cpy)
    mem_cpy                                  0x00029ff9   Thumb Code    18  ff.o(i.mem_cpy)
    i.mem_set                                0x0002a00c   Section        0  ff.o(i.mem_set)
    mem_set                                  0x0002a00d   Thumb Code    14  ff.o(i.mem_set)
    i.memobj_op                              0x0002a01a   Section        0  nrf_memobj.o(i.memobj_op)
    memobj_op                                0x0002a01b   Thumb Code   126  nrf_memobj.o(i.memobj_op)
    i.module_idx_get                         0x0002a098   Section        0  nrf_log_frontend.o(i.module_idx_get)
    module_idx_get                           0x0002a099   Thumb Code    42  nrf_log_frontend.o(i.module_idx_get)
    i.move_window                            0x0002a0c8   Section        0  ff.o(i.move_window)
    move_window                              0x0002a0c9   Thumb Code    50  ff.o(i.move_window)
    i.name_encode                            0x0002a0fa   Section        0  ble_advdata.o(i.name_encode)
    name_encode                              0x0002a0fb   Thumb Code   166  ble_advdata.o(i.name_encode)
    i.nrf_atfifo_item_alloc                  0x0002a1a0   Section        0  nrf_atfifo.o(i.nrf_atfifo_item_alloc)
    i.nrf_atfifo_item_put                    0x0002a1b6   Section        0  nrf_atfifo.o(i.nrf_atfifo_item_put)
    i.nrf_atflags_clear                      0x0002a1cc   Section        0  nrf_atflags.o(i.nrf_atflags_clear)
    i.nrf_atflags_get                        0x0002a1e2   Section        0  nrf_atflags.o(i.nrf_atflags_get)
    i.nrf_atflags_set                        0x0002a1f8   Section        0  nrf_atflags.o(i.nrf_atflags_set)
    i.nrf_atomic_flag_clear_fetch            0x0002a20c   Section        0  nrf_atomic.o(i.nrf_atomic_flag_clear_fetch)
    i.nrf_atomic_flag_set                    0x0002a212   Section        0  nrf_atomic.o(i.nrf_atomic_flag_set)
    i.nrf_atomic_u32_add                     0x0002a218   Section        0  nrf_atomic.o(i.nrf_atomic_u32_add)
    i.nrf_atomic_u32_and                     0x0002a224   Section        0  nrf_atomic.o(i.nrf_atomic_u32_and)
    i.nrf_atomic_u32_fetch_and               0x0002a230   Section        0  nrf_atomic.o(i.nrf_atomic_u32_fetch_and)
    i.nrf_atomic_u32_fetch_store             0x0002a23a   Section        0  nrf_atomic.o(i.nrf_atomic_u32_fetch_store)
    i.nrf_atomic_u32_or                      0x0002a244   Section        0  nrf_atomic.o(i.nrf_atomic_u32_or)
    i.nrf_atomic_u32_sub                     0x0002a250   Section        0  nrf_atomic.o(i.nrf_atomic_u32_sub)
    i.nrf_balloc_alloc                       0x0002a25c   Section        0  nrf_balloc.o(i.nrf_balloc_alloc)
    i.nrf_balloc_free                        0x0002a2a0   Section        0  nrf_balloc.o(i.nrf_balloc_free)
    i.nrf_balloc_init                        0x0002a2d0   Section        0  nrf_balloc.o(i.nrf_balloc_init)
    i.nrf_bitmask_bit_is_set                 0x0002a300   Section        0  nrfx_gpiote.o(i.nrf_bitmask_bit_is_set)
    nrf_bitmask_bit_is_set                   0x0002a301   Thumb Code    16  nrfx_gpiote.o(i.nrf_bitmask_bit_is_set)
    i.nrf_ble_gatt_att_mtu_periph_set        0x0002a310   Section        0  nrf_ble_gatt.o(i.nrf_ble_gatt_att_mtu_periph_set)
    i.nrf_ble_gatt_init                      0x0002a328   Section        0  nrf_ble_gatt.o(i.nrf_ble_gatt_init)
    i.nrf_ble_gatt_on_ble_evt                0x0002a34c   Section        0  nrf_ble_gatt.o(i.nrf_ble_gatt_on_ble_evt)
    i.nrf_ble_qwr_conn_handle_assign         0x0002a49c   Section        0  nrf_ble_qwr.o(i.nrf_ble_qwr_conn_handle_assign)
    i.nrf_ble_qwr_init                       0x0002a4b2   Section        0  nrf_ble_qwr.o(i.nrf_ble_qwr_init)
    i.nrf_ble_qwr_on_ble_evt                 0x0002a4d6   Section        0  nrf_ble_qwr.o(i.nrf_ble_qwr_on_ble_evt)
    i.nrf_blk_dev_ioctl                      0x0002a58c   Section        0  diskio_blkdev.o(i.nrf_blk_dev_ioctl)
    nrf_blk_dev_ioctl                        0x0002a58d   Thumb Code     6  diskio_blkdev.o(i.nrf_blk_dev_ioctl)
    i.nrf_clock_event_check                  0x0002a592   Section        0  nrfx_clock.o(i.nrf_clock_event_check)
    nrf_clock_event_check                    0x0002a593   Thumb Code    14  nrfx_clock.o(i.nrf_clock_event_check)
    i.nrf_clock_event_clear                  0x0002a5a0   Section        0  nrfx_clock.o(i.nrf_clock_event_clear)
    nrf_clock_event_clear                    0x0002a5a1   Thumb Code    16  nrfx_clock.o(i.nrf_clock_event_clear)
    i.nrf_drv_clock_init                     0x0002a5b0   Section        0  nrf_drv_clock.o(i.nrf_drv_clock_init)
    i.nrf_drv_clock_lfclk_release            0x0002a5f0   Section        0  nrf_drv_clock.o(i.nrf_drv_clock_lfclk_release)
    i.nrf_drv_spi_init                       0x0002a624   Section        0  nrf_drv_spi.o(i.nrf_drv_spi_init)
    i.nrf_drv_spi_transfer                   0x0002a694   Section        0  app_sdcard.o(i.nrf_drv_spi_transfer)
    nrf_drv_spi_transfer                     0x0002a695   Thumb Code    22  app_sdcard.o(i.nrf_drv_spi_transfer)
    i.nrf_drv_uart_init                      0x0002a6ac   Section        0  nrf_drv_uart.o(i.nrf_drv_uart_init)
    i.nrf_drv_uart_tx                        0x0002a714   Section        0  app_uart_fifo.o(i.nrf_drv_uart_tx)
    nrf_drv_uart_tx                          0x0002a715   Thumb Code    26  app_uart_fifo.o(i.nrf_drv_uart_tx)
    i.nrf_fprintf                            0x0002a734   Section        0  nrf_fprintf.o(i.nrf_fprintf)
    i.nrf_fprintf_buffer_flush               0x0002a74e   Section        0  nrf_fprintf.o(i.nrf_fprintf_buffer_flush)
    i.nrf_fprintf_fmt                        0x0002a766   Section        0  nrf_fprintf_format.o(i.nrf_fprintf_fmt)
    i.nrf_gpio_cfg                           0x0002a940   Section        0  nrfx_uart.o(i.nrf_gpio_cfg)
    nrf_gpio_cfg                             0x0002a941   Thumb Code    36  nrfx_uart.o(i.nrf_gpio_cfg)
    i.nrf_gpio_cfg                           0x0002a964   Section        0  nrfx_uarte.o(i.nrf_gpio_cfg)
    nrf_gpio_cfg                             0x0002a965   Thumb Code    36  nrfx_uarte.o(i.nrf_gpio_cfg)
    i.nrf_gpio_cfg                           0x0002a988   Section        0  nrfx_spim.o(i.nrf_gpio_cfg)
    nrf_gpio_cfg                             0x0002a989   Thumb Code    36  nrfx_spim.o(i.nrf_gpio_cfg)
    i.nrf_gpio_cfg                           0x0002a9ac   Section        0  app_sdcard.o(i.nrf_gpio_cfg)
    nrf_gpio_cfg                             0x0002a9ad   Thumb Code    36  app_sdcard.o(i.nrf_gpio_cfg)
    i.nrf_gpio_cfg_default                   0x0002a9d0   Section        0  nrfx_uart.o(i.nrf_gpio_cfg_default)
    nrf_gpio_cfg_default                     0x0002a9d1   Thumb Code    18  nrfx_uart.o(i.nrf_gpio_cfg_default)
    i.nrf_gpio_cfg_default                   0x0002a9e2   Section        0  nrfx_uarte.o(i.nrf_gpio_cfg_default)
    nrf_gpio_cfg_default                     0x0002a9e3   Thumb Code    18  nrfx_uarte.o(i.nrf_gpio_cfg_default)
    i.nrf_gpio_cfg_input                     0x0002a9f4   Section        0  nrfx_uart.o(i.nrf_gpio_cfg_input)
    nrf_gpio_cfg_input                       0x0002a9f5   Thumb Code    18  nrfx_uart.o(i.nrf_gpio_cfg_input)
    i.nrf_gpio_cfg_input                     0x0002aa06   Section        0  nrfx_uarte.o(i.nrf_gpio_cfg_input)
    nrf_gpio_cfg_input                       0x0002aa07   Thumb Code    18  nrfx_uarte.o(i.nrf_gpio_cfg_input)
    i.nrf_gpio_cfg_output                    0x0002aa18   Section        0  nrfx_uart.o(i.nrf_gpio_cfg_output)
    nrf_gpio_cfg_output                      0x0002aa19   Thumb Code    20  nrfx_uart.o(i.nrf_gpio_cfg_output)
    i.nrf_gpio_cfg_output                    0x0002aa2c   Section        0  nrfx_uarte.o(i.nrf_gpio_cfg_output)
    nrf_gpio_cfg_output                      0x0002aa2d   Thumb Code    20  nrfx_uarte.o(i.nrf_gpio_cfg_output)
    i.nrf_gpio_cfg_output                    0x0002aa40   Section        0  nrfx_spim.o(i.nrf_gpio_cfg_output)
    nrf_gpio_cfg_output                      0x0002aa41   Thumb Code    20  nrfx_spim.o(i.nrf_gpio_cfg_output)
    i.nrf_gpio_cfg_sense_set                 0x0002aa54   Section        0  nrfx_gpiote.o(i.nrf_gpio_cfg_sense_set)
    nrf_gpio_cfg_sense_set                   0x0002aa55   Thumb Code    34  nrfx_gpiote.o(i.nrf_gpio_cfg_sense_set)
    i.nrf_gpio_latches_read_and_clear        0x0002aa78   Section        0  nrfx_gpiote.o(i.nrf_gpio_latches_read_and_clear)
    nrf_gpio_latches_read_and_clear          0x0002aa79   Thumb Code    38  nrfx_gpiote.o(i.nrf_gpio_latches_read_and_clear)
    i.nrf_gpio_pin_clear                     0x0002aaa4   Section        0  nrfx_spim.o(i.nrf_gpio_pin_clear)
    nrf_gpio_pin_clear                       0x0002aaa5   Thumb Code    14  nrfx_spim.o(i.nrf_gpio_pin_clear)
    i.nrf_gpio_pin_set                       0x0002aab2   Section        0  nrfx_spim.o(i.nrf_gpio_pin_set)
    nrf_gpio_pin_set                         0x0002aab3   Thumb Code    14  nrfx_spim.o(i.nrf_gpio_pin_set)
    i.nrf_gpio_pin_set                       0x0002aac0   Section        0  app_sdcard.o(i.nrf_gpio_pin_set)
    nrf_gpio_pin_set                         0x0002aac1   Thumb Code    14  app_sdcard.o(i.nrf_gpio_pin_set)
    i.nrf_gpio_pin_write                     0x0002aace   Section        0  boards.o(i.nrf_gpio_pin_write)
    nrf_gpio_pin_write                       0x0002aacf   Thumb Code    22  boards.o(i.nrf_gpio_pin_write)
    i.nrf_gpiote_event_clear                 0x0002aae4   Section        0  nrfx_gpiote.o(i.nrf_gpiote_event_clear)
    nrf_gpiote_event_clear                   0x0002aae5   Thumb Code    16  nrfx_gpiote.o(i.nrf_gpiote_event_clear)
    i.nrf_gpiote_event_is_set                0x0002aaf8   Section        0  nrfx_gpiote.o(i.nrf_gpiote_event_is_set)
    nrf_gpiote_event_is_set                  0x0002aaf9   Thumb Code    12  nrfx_gpiote.o(i.nrf_gpiote_event_is_set)
    i.nrf_log_backend_add                    0x0002ab08   Section        0  nrf_log_frontend.o(i.nrf_log_backend_add)
    i.nrf_log_backend_rtt_flush              0x0002ab64   Section        0  nrf_log_backend_rtt.o(i.nrf_log_backend_rtt_flush)
    nrf_log_backend_rtt_flush                0x0002ab65   Thumb Code     2  nrf_log_backend_rtt.o(i.nrf_log_backend_rtt_flush)
    i.nrf_log_backend_rtt_init               0x0002ab66   Section        0  nrf_log_backend_rtt.o(i.nrf_log_backend_rtt_init)
    i.nrf_log_backend_rtt_panic_set          0x0002ab6a   Section        0  nrf_log_backend_rtt.o(i.nrf_log_backend_rtt_panic_set)
    nrf_log_backend_rtt_panic_set            0x0002ab6b   Thumb Code     2  nrf_log_backend_rtt.o(i.nrf_log_backend_rtt_panic_set)
    i.nrf_log_backend_rtt_put                0x0002ab6c   Section        0  nrf_log_backend_rtt.o(i.nrf_log_backend_rtt_put)
    nrf_log_backend_rtt_put                  0x0002ab6d   Thumb Code    16  nrf_log_backend_rtt.o(i.nrf_log_backend_rtt_put)
    i.nrf_log_backend_serial_put             0x0002ab84   Section        0  nrf_log_backend_serial.o(i.nrf_log_backend_serial_put)
    i.nrf_log_backend_uart_flush             0x0002ac4c   Section        0  nrf_log_backend_uart.o(i.nrf_log_backend_uart_flush)
    nrf_log_backend_uart_flush               0x0002ac4d   Thumb Code     2  nrf_log_backend_uart.o(i.nrf_log_backend_uart_flush)
    i.nrf_log_backend_uart_init              0x0002ac4e   Section        0  nrf_log_backend_uart.o(i.nrf_log_backend_uart_init)
    i.nrf_log_backend_uart_panic_set         0x0002ac54   Section        0  nrf_log_backend_uart.o(i.nrf_log_backend_uart_panic_set)
    nrf_log_backend_uart_panic_set           0x0002ac55   Thumb Code    36  nrf_log_backend_uart.o(i.nrf_log_backend_uart_panic_set)
    i.nrf_log_backend_uart_put               0x0002ac80   Section        0  nrf_log_backend_uart.o(i.nrf_log_backend_uart_put)
    nrf_log_backend_uart_put                 0x0002ac81   Thumb Code    16  nrf_log_backend_uart.o(i.nrf_log_backend_uart_put)
    i.nrf_log_color_id_get                   0x0002ac98   Section        0  nrf_log_frontend.o(i.nrf_log_color_id_get)
    i.nrf_log_default_backends_init          0x0002acc8   Section        0  nrf_log_default_backends.o(i.nrf_log_default_backends_init)
    i.nrf_log_frontend_dequeue               0x0002acfc   Section        0  nrf_log_frontend.o(i.nrf_log_frontend_dequeue)
    i.nrf_log_frontend_std_0                 0x0002af34   Section        0  nrf_log_frontend.o(i.nrf_log_frontend_std_0)
    i.nrf_log_frontend_std_1                 0x0002af3c   Section        0  nrf_log_frontend.o(i.nrf_log_frontend_std_1)
    i.nrf_log_frontend_std_2                 0x0002af4a   Section        0  nrf_log_frontend.o(i.nrf_log_frontend_std_2)
    i.nrf_log_hexdump_entry_process          0x0002af5c   Section        0  nrf_log_str_formatter.o(i.nrf_log_hexdump_entry_process)
    i.nrf_log_init                           0x0002b00c   Section        0  nrf_log_frontend.o(i.nrf_log_init)
    i.nrf_log_module_cnt_get                 0x0002b034   Section        0  nrf_log_frontend.o(i.nrf_log_module_cnt_get)
    i.nrf_log_module_name_get                0x0002b048   Section        0  nrf_log_frontend.o(i.nrf_log_module_name_get)
    i.nrf_log_panic                          0x0002b064   Section        0  nrf_log_frontend.o(i.nrf_log_panic)
    i.nrf_log_std_entry_process              0x0002b08c   Section        0  nrf_log_str_formatter.o(i.nrf_log_std_entry_process)
    i.nrf_memobj_alloc                       0x0002b142   Section        0  nrf_memobj.o(i.nrf_memobj_alloc)
    i.nrf_memobj_free                        0x0002b1a2   Section        0  nrf_memobj.o(i.nrf_memobj_free)
    i.nrf_memobj_get                         0x0002b1d4   Section        0  nrf_memobj.o(i.nrf_memobj_get)
    i.nrf_memobj_pool_init                   0x0002b1dc   Section        0  nrf_memobj.o(i.nrf_memobj_pool_init)
    i.nrf_memobj_put                         0x0002b1e0   Section        0  nrf_memobj.o(i.nrf_memobj_put)
    i.nrf_memobj_read                        0x0002b1fe   Section        0  nrf_memobj.o(i.nrf_memobj_read)
    i.nrf_memobj_write                       0x0002b20e   Section        0  nrf_memobj.o(i.nrf_memobj_write)
    i.nrf_pwr_mgmt_init                      0x0002b220   Section        0  nrf_pwr_mgmt.o(i.nrf_pwr_mgmt_init)
    i.nrf_qwr_error_handler                  0x0002b248   Section        0  main.o(i.nrf_qwr_error_handler)
    nrf_qwr_error_handler                    0x0002b249   Thumb Code     4  main.o(i.nrf_qwr_error_handler)
    i.nrf_ringbuf_init                       0x0002b24c   Section        0  nrf_ringbuf.o(i.nrf_ringbuf_init)
    i.nrf_sdh_ble_app_ram_start_get          0x0002b268   Section        0  nrf_sdh_ble.o(i.nrf_sdh_ble_app_ram_start_get)
    i.nrf_sdh_ble_default_cfg_set            0x0002b27c   Section        0  nrf_sdh_ble.o(i.nrf_sdh_ble_default_cfg_set)
    i.nrf_sdh_ble_enable                     0x0002b3ac   Section        0  nrf_sdh_ble.o(i.nrf_sdh_ble_enable)
    i.nrf_sdh_ble_evts_poll                  0x0002b4dc   Section        0  nrf_sdh_ble.o(i.nrf_sdh_ble_evts_poll)
    nrf_sdh_ble_evts_poll                    0x0002b4dd   Thumb Code    88  nrf_sdh_ble.o(i.nrf_sdh_ble_evts_poll)
    i.nrf_sdh_enable_request                 0x0002b53c   Section        0  nrf_sdh.o(i.nrf_sdh_enable_request)
    i.nrf_sdh_evts_poll                      0x0002b5b0   Section        0  nrf_sdh.o(i.nrf_sdh_evts_poll)
    i.nrf_sdh_is_enabled                     0x0002b5d4   Section        0  nrf_sdh.o(i.nrf_sdh_is_enabled)
    i.nrf_sdh_soc_evts_poll                  0x0002b5e0   Section        0  nrf_sdh_soc.o(i.nrf_sdh_soc_evts_poll)
    nrf_sdh_soc_evts_poll                    0x0002b5e1   Thumb Code    56  nrf_sdh_soc.o(i.nrf_sdh_soc_evts_poll)
    i.nrf_section_iter_init                  0x0002b61c   Section        0  nrf_section_iter.o(i.nrf_section_iter_init)
    i.nrf_section_iter_item_set              0x0002b626   Section        0  nrf_section_iter.o(i.nrf_section_iter_item_set)
    nrf_section_iter_item_set                0x0002b627   Thumb Code    36  nrf_section_iter.o(i.nrf_section_iter_item_set)
    i.nrf_section_iter_next                  0x0002b64a   Section        0  nrf_section_iter.o(i.nrf_section_iter_next)
    i.nrf_spim_event_check                   0x0002b66a   Section        0  nrfx_spim.o(i.nrf_spim_event_check)
    nrf_spim_event_check                     0x0002b66b   Thumb Code    10  nrfx_spim.o(i.nrf_spim_event_check)
    i.nrf_strerror_find                      0x0002b674   Section        0  nrf_strerror.o(i.nrf_strerror_find)
    i.nrf_strerror_get                       0x0002b6ac   Section        0  nrf_strerror.o(i.nrf_strerror_get)
    i.nrf_uart_event_check                   0x0002b6c0   Section        0  nrfx_uart.o(i.nrf_uart_event_check)
    nrf_uart_event_check                     0x0002b6c1   Thumb Code    10  nrfx_uart.o(i.nrf_uart_event_check)
    i.nrf_uart_event_clear                   0x0002b6ca   Section        0  nrfx_uart.o(i.nrf_uart_event_clear)
    nrf_uart_event_clear                     0x0002b6cb   Thumb Code    12  nrfx_uart.o(i.nrf_uart_event_clear)
    i.nrf_uart_int_enable_check              0x0002b6d6   Section        0  nrfx_uart.o(i.nrf_uart_int_enable_check)
    nrf_uart_int_enable_check                0x0002b6d7   Thumb Code    12  nrfx_uart.o(i.nrf_uart_int_enable_check)
    i.nrf_uarte_event_check                  0x0002b6e2   Section        0  nrfx_uarte.o(i.nrf_uarte_event_check)
    nrf_uarte_event_check                    0x0002b6e3   Thumb Code    10  nrfx_uarte.o(i.nrf_uarte_event_check)
    i.nrf_uarte_event_clear                  0x0002b6ec   Section        0  nrfx_uarte.o(i.nrf_uarte_event_clear)
    nrf_uarte_event_clear                    0x0002b6ed   Thumb Code    12  nrfx_uarte.o(i.nrf_uarte_event_clear)
    i.nrf_wdt_started                        0x0002b6f8   Section        0  nrf_drv_clock.o(i.nrf_wdt_started)
    nrf_wdt_started                          0x0002b6f9   Thumb Code    12  nrf_drv_clock.o(i.nrf_wdt_started)
    i.nrfx_clock_enable                      0x0002b708   Section        0  nrfx_clock.o(i.nrfx_clock_enable)
    i.nrfx_clock_init                        0x0002b734   Section        0  nrfx_clock.o(i.nrfx_clock_init)
    i.nrfx_clock_lfclk_stop                  0x0002b754   Section        0  nrfx_clock.o(i.nrfx_clock_lfclk_stop)
    i.nrfx_is_in_ram                         0x0002b784   Section        0  nrfx_uarte.o(i.nrfx_is_in_ram)
    nrfx_is_in_ram                           0x0002b785   Thumb Code    16  nrfx_uarte.o(i.nrfx_is_in_ram)
    i.nrfx_is_in_ram                         0x0002b794   Section        0  nrfx_spim.o(i.nrfx_is_in_ram)
    nrfx_is_in_ram                           0x0002b795   Thumb Code    16  nrfx_spim.o(i.nrfx_is_in_ram)
    i.nrfx_prs_acquire                       0x0002b7a4   Section        0  nrfx_prs.o(i.nrfx_prs_acquire)
    i.nrfx_prs_release                       0x0002b7de   Section        0  nrfx_prs.o(i.nrfx_prs_release)
    i.nrfx_spim_init                         0x0002b7f0   Section        0  nrfx_spim.o(i.nrfx_spim_init)
    i.nrfx_spim_uninit                       0x0002b95c   Section        0  nrfx_spim.o(i.nrfx_spim_uninit)
    i.nrfx_spim_xfer                         0x0002b9f0   Section        0  nrfx_spim.o(i.nrfx_spim_xfer)
    i.nrfx_uart_0_irq_handler                0x0002ba54   Section        0  nrfx_uart.o(i.nrfx_uart_0_irq_handler)
    i.nrfx_uart_init                         0x0002ba64   Section        0  nrfx_uart.o(i.nrfx_uart_init)
    i.nrfx_uart_tx                           0x0002bb38   Section        0  nrfx_uart.o(i.nrfx_uart_tx)
    i.nrfx_uart_tx_in_progress               0x0002bbe0   Section        0  nrfx_uart.o(i.nrfx_uart_tx_in_progress)
    i.nrfx_uart_uninit                       0x0002bc00   Section        0  nrfx_uart.o(i.nrfx_uart_uninit)
    i.nrfx_uarte_0_irq_handler               0x0002bcc0   Section        0  nrfx_uarte.o(i.nrfx_uarte_0_irq_handler)
    i.nrfx_uarte_init                        0x0002bcd0   Section        0  nrfx_uarte.o(i.nrfx_uarte_init)
    i.nrfx_uarte_tx                          0x0002bd3c   Section        0  nrfx_uarte.o(i.nrfx_uarte_tx)
    i.nrfx_uarte_tx_in_progress              0x0002bde8   Section        0  nrfx_uarte.o(i.nrfx_uarte_tx_in_progress)
    i.nrfx_uarte_uninit                      0x0002be04   Section        0  nrfx_uarte.o(i.nrfx_uarte_uninit)
    i.nus_data_handler                       0x0002bf0c   Section        0  main.o(i.nus_data_handler)
    nus_data_handler                         0x0002bf0d   Thumb Code    98  main.o(i.nus_data_handler)
    i.nvmc_config                            0x0002bfa4   Section        0  system_nrf52.o(i.nvmc_config)
    i.on_adv_evt                             0x0002bfbc   Section        0  main.o(i.on_adv_evt)
    on_adv_evt                               0x0002bfbd   Thumb Code    54  main.o(i.on_adv_evt)
    i.on_conn_params_evt                     0x0002bff4   Section        0  main.o(i.on_conn_params_evt)
    on_conn_params_evt                       0x0002bff5   Thumb Code    24  main.o(i.on_conn_params_evt)
    i.on_connect                             0x0002c010   Section        0  ble_nus.o(i.on_connect)
    on_connect                               0x0002c011   Thumb Code   106  ble_nus.o(i.on_connect)
    i.on_connected_evt                       0x0002c07c   Section        0  nrf_ble_gatt.o(i.on_connected_evt)
    on_connected_evt                         0x0002c07d   Thumb Code   106  nrf_ble_gatt.o(i.on_connected_evt)
    i.on_exchange_mtu_request_evt            0x0002c124   Section        0  nrf_ble_gatt.o(i.on_exchange_mtu_request_evt)
    on_exchange_mtu_request_evt              0x0002c125   Thumb Code   110  nrf_ble_gatt.o(i.on_exchange_mtu_request_evt)
    i.on_write                               0x0002c1d0   Section        0  ble_nus.o(i.on_write)
    on_write                                 0x0002c1d1   Thumb Code   132  ble_nus.o(i.on_write)
    i.phy_is_valid                           0x0002c254   Section        0  ble_advertising.o(i.phy_is_valid)
    phy_is_valid                             0x0002c255   Thumb Code    18  ble_advertising.o(i.phy_is_valid)
    i.port_event_handle                      0x0002c268   Section        0  nrfx_gpiote.o(i.port_event_handle)
    port_event_handle                        0x0002c269   Thumb Code   176  nrfx_gpiote.o(i.port_event_handle)
    i.port_handler_polarity_get              0x0002c31c   Section        0  nrfx_gpiote.o(i.port_handler_polarity_get)
    port_handler_polarity_get                0x0002c31d   Thumb Code    12  nrfx_gpiote.o(i.port_handler_polarity_get)
    i.postfix_process                        0x0002c32c   Section        0  nrf_log_str_formatter.o(i.postfix_process)
    postfix_process                          0x0002c32d   Thumb Code    48  nrf_log_str_formatter.o(i.postfix_process)
    i.prefix_process                         0x0002c368   Section        0  nrf_log_str_formatter.o(i.prefix_process)
    prefix_process                           0x0002c369   Thumb Code    90  nrf_log_str_formatter.o(i.prefix_process)
    i.prs_box_get                            0x0002c400   Section        0  nrfx_prs.o(i.prs_box_get)
    prs_box_get                              0x0002c401   Thumb Code    14  nrfx_prs.o(i.prs_box_get)
    i.put_fat                                0x0002c418   Section        0  ff.o(i.put_fat)
    put_fat                                  0x0002c419   Thumb Code   234  ff.o(i.put_fat)
    i.remove_chain                           0x0002c502   Section        0  ff.o(i.remove_chain)
    remove_chain                             0x0002c503   Thumb Code   116  ff.o(i.remove_chain)
    i.rx_byte                                0x0002c576   Section        0  nrfx_uart.o(i.rx_byte)
    rx_byte                                  0x0002c577   Thumb Code    50  nrfx_uart.o(i.rx_byte)
    i.rx_done_event                          0x0002c5a8   Section        0  nrfx_uart.o(i.rx_done_event)
    rx_done_event                            0x0002c5a9   Thumb Code    22  nrfx_uart.o(i.rx_done_event)
    i.rx_done_event                          0x0002c5be   Section        0  nrfx_uarte.o(i.rx_done_event)
    rx_done_event                            0x0002c5bf   Thumb Code    22  nrfx_uarte.o(i.rx_done_event)
    i.saadc_init                             0x0002c5d4   Section        0  main.o(i.saadc_init)
    i.saadc_start                            0x0002c618   Section        0  main.o(i.saadc_start)
    i.sd_state_evt_handler                   0x0002c640   Section        0  nrf_drv_clock.o(i.sd_state_evt_handler)
    sd_state_evt_handler                     0x0002c641   Thumb Code    84  nrf_drv_clock.o(i.sd_state_evt_handler)
    i.sdc_cmd                                0x0002c698   Section        0  app_sdcard.o(i.sdc_cmd)
    sdc_cmd                                  0x0002c699   Thumb Code   178  app_sdcard.o(i.sdc_cmd)
    i.sdc_handler                            0x0002c750   Section        0  nrf_block_dev_sdc.o(i.sdc_handler)
    sdc_handler                              0x0002c751   Thumb Code   148  nrf_block_dev_sdc.o(i.sdc_handler)
    i.sdc_pt_identification                  0x0002c7ec   Section        0  app_sdcard.o(i.sdc_pt_identification)
    sdc_pt_identification                    0x0002c7ed   Thumb Code   662  app_sdcard.o(i.sdc_pt_identification)
    i.sdc_pt_read                            0x0002ca88   Section        0  app_sdcard.o(i.sdc_pt_read)
    sdc_pt_read                              0x0002ca89   Thumb Code   122  app_sdcard.o(i.sdc_pt_read)
    i.sdc_pt_sub_data_read                   0x0002cb08   Section        0  app_sdcard.o(i.sdc_pt_sub_data_read)
    sdc_pt_sub_data_read                     0x0002cb09   Thumb Code   348  app_sdcard.o(i.sdc_pt_sub_data_read)
    i.sdc_pt_write                           0x0002cc68   Section        0  app_sdcard.o(i.sdc_pt_write)
    sdc_pt_write                             0x0002cc69   Thumb Code   516  app_sdcard.o(i.sdc_pt_write)
    i.sdc_spi_transfer                       0x0002ce70   Section        0  app_sdcard.o(i.sdc_spi_transfer)
    sdc_spi_transfer                         0x0002ce71   Thumb Code    50  app_sdcard.o(i.sdc_spi_transfer)
    i.sdh_request_observer_notify            0x0002ceac   Section        0  nrf_sdh.o(i.sdh_request_observer_notify)
    sdh_request_observer_notify              0x0002cead   Thumb Code    44  nrf_sdh.o(i.sdh_request_observer_notify)
    i.sdh_state_observer_notify              0x0002cedc   Section        0  nrf_sdh.o(i.sdh_state_observer_notify)
    sdh_state_observer_notify                0x0002cedd   Thumb Code    38  nrf_sdh.o(i.sdh_state_observer_notify)
    i.send_error_evt                         0x0002cf08   Section        0  ble_conn_params.o(i.send_error_evt)
    send_error_evt                           0x0002cf09   Thumb Code    12  ble_conn_params.o(i.send_error_evt)
    i.serial_tx                              0x0002cf18   Section        0  nrf_log_backend_rtt.o(i.serial_tx)
    serial_tx                                0x0002cf19   Thumb Code    70  nrf_log_backend_rtt.o(i.serial_tx)
    i.serial_tx                              0x0002cf68   Section        0  nrf_log_backend_uart.o(i.serial_tx)
    serial_tx                                0x0002cf69   Thumb Code    54  nrf_log_backend_uart.o(i.serial_tx)
    i.service_data_encode                    0x0002cfa8   Section        0  ble_advdata.o(i.service_data_encode)
    service_data_encode                      0x0002cfa9   Thumb Code   136  ble_advdata.o(i.service_data_encode)
    i.set_security_req                       0x0002d030   Section        0  ble_srv_common.o(i.set_security_req)
    set_security_req                         0x0002d031   Thumb Code    48  ble_srv_common.o(i.set_security_req)
    i.soc_evt_handler                        0x0002d060   Section        0  nrf_drv_clock.o(i.soc_evt_handler)
    soc_evt_handler                          0x0002d061   Thumb Code    18  nrf_drv_clock.o(i.soc_evt_handler)
    i.softdevices_evt_irq_enable             0x0002d078   Section        0  nrf_sdh.o(i.softdevices_evt_irq_enable)
    softdevices_evt_irq_enable               0x0002d079   Thumb Code    80  nrf_sdh.o(i.softdevices_evt_irq_enable)
    i.spi_handler                            0x0002d0d0   Section        0  app_sdcard.o(i.spi_handler)
    spi_handler                              0x0002d0d1   Thumb Code   434  app_sdcard.o(i.spi_handler)
    i.spim_evt_handler                       0x0002d28c   Section        0  nrf_drv_spi.o(i.spim_evt_handler)
    spim_evt_handler                         0x0002d28d   Thumb Code    52  nrf_drv_spi.o(i.spim_evt_handler)
    i.spim_xfer                              0x0002d2c4   Section        0  nrfx_spim.o(i.spim_xfer)
    spim_xfer                                0x0002d2c5   Thumb Code   188  nrfx_spim.o(i.spim_xfer)
    i.st_clust                               0x0002d380   Section        0  ff.o(i.st_clust)
    st_clust                                 0x0002d381   Thumb Code    40  ff.o(i.st_clust)
    i.st_dword                               0x0002d3a8   Section        0  ff.o(i.st_dword)
    st_dword                                 0x0002d3a9   Thumb Code    16  ff.o(i.st_dword)
    i.st_word                                0x0002d3b8   Section        0  ff.o(i.st_word)
    st_word                                  0x0002d3b9   Thumb Code     8  ff.o(i.st_word)
    i.std_n                                  0x0002d3c0   Section        0  nrf_log_frontend.o(i.std_n)
    std_n                                    0x0002d3c1   Thumb Code   140  nrf_log_frontend.o(i.std_n)
    i.sync_fs                                0x0002d454   Section        0  ff.o(i.sync_fs)
    sync_fs                                  0x0002d455   Thumb Code   126  ff.o(i.sync_fs)
    i.sync_window                            0x0002d4dc   Section        0  ff.o(i.sync_window)
    sync_window                              0x0002d4dd   Thumb Code    82  ff.o(i.sync_window)
    i.timer_init                             0x0002d530   Section        0  main.o(i.timer_init)
    i.timer_req_schedule                     0x0002d57c   Section        0  app_timer2.o(i.timer_req_schedule)
    timer_req_schedule                       0x0002d57d   Thumb Code    46  app_timer2.o(i.timer_req_schedule)
    i.tx_byte                                0x0002d5b4   Section        0  nrfx_uart.o(i.tx_byte)
    tx_byte                                  0x0002d5b5   Thumb Code    32  nrfx_uart.o(i.tx_byte)
    i.tx_done_event                          0x0002d5d4   Section        0  nrfx_uart.o(i.tx_done_event)
    tx_done_event                            0x0002d5d5   Thumb Code    26  nrfx_uart.o(i.tx_done_event)
    i.tx_done_event                          0x0002d5ee   Section        0  nrfx_uarte.o(i.tx_done_event)
    tx_done_event                            0x0002d5ef   Thumb Code    26  nrfx_uarte.o(i.tx_done_event)
    i.uart_evt_handler                       0x0002d608   Section        0  nrf_drv_uart.o(i.uart_evt_handler)
    uart_evt_handler                         0x0002d609   Thumb Code    42  nrf_drv_uart.o(i.uart_evt_handler)
    i.uart_evt_handler                       0x0002d638   Section        0  nrf_log_backend_uart.o(i.uart_evt_handler)
    uart_evt_handler                         0x0002d639   Thumb Code     8  nrf_log_backend_uart.o(i.uart_evt_handler)
    i.uart_init                              0x0002d644   Section        0  nrf_log_backend_uart.o(i.uart_init)
    uart_init                                0x0002d645   Thumb Code    66  nrf_log_backend_uart.o(i.uart_init)
    i.uart_irq_handler                       0x0002d694   Section        0  nrfx_uart.o(i.uart_irq_handler)
    uart_irq_handler                         0x0002d695   Thumb Code   298  nrfx_uart.o(i.uart_irq_handler)
    i.uarte_evt_handler                      0x0002d7c0   Section        0  nrf_drv_uart.o(i.uarte_evt_handler)
    uarte_evt_handler                        0x0002d7c1   Thumb Code    42  nrf_drv_uart.o(i.uarte_evt_handler)
    i.uarte_irq_handler                      0x0002d7f0   Section        0  nrfx_uarte.o(i.uarte_irq_handler)
    uarte_irq_handler                        0x0002d7f1   Thumb Code   274  nrfx_uarte.o(i.uarte_irq_handler)
    i.uint16_encode                          0x0002d902   Section        0  ble_advdata.o(i.uint16_encode)
    uint16_encode                            0x0002d903   Thumb Code    10  ble_advdata.o(i.uint16_encode)
    i.unsigned_print                         0x0002d90c   Section        0  nrf_fprintf_format.o(i.unsigned_print)
    unsigned_print                           0x0002d90d   Thumb Code   176  nrf_fprintf_format.o(i.unsigned_print)
    i.update_timeout_handler                 0x0002d9c0   Section        0  ble_conn_params.o(i.update_timeout_handler)
    update_timeout_handler                   0x0002d9c1   Thumb Code    98  ble_conn_params.o(i.update_timeout_handler)
    i.use_whitelist                          0x0002da28   Section        0  ble_advertising.o(i.use_whitelist)
    use_whitelist                            0x0002da29   Thumb Code    24  ble_advertising.o(i.use_whitelist)
    i.user_mem_reply                         0x0002da40   Section        0  nrf_ble_qwr.o(i.user_mem_reply)
    user_mem_reply                           0x0002da41   Thumb Code    36  nrf_ble_qwr.o(i.user_mem_reply)
    i.uuid_list_encode                       0x0002da64   Section        0  ble_advdata.o(i.uuid_list_encode)
    uuid_list_encode                         0x0002da65   Thumb Code    48  ble_advdata.o(i.uuid_list_encode)
    i.uuid_list_sized_encode                 0x0002da94   Section        0  ble_advdata.o(i.uuid_list_sized_encode)
    uuid_list_sized_encode                   0x0002da95   Thumb Code   158  ble_advdata.o(i.uuid_list_sized_encode)
    i.validate                               0x0002db32   Section        0  ff.o(i.validate)
    validate                                 0x0002db33   Thumb Code    50  ff.o(i.validate)
    i.wakeup_button_cfg                      0x0002db64   Section        0  bsp.o(i.wakeup_button_cfg)
    wakeup_button_cfg                        0x0002db65   Thumb Code    58  bsp.o(i.wakeup_button_cfg)
    .constdata                               0x0002dba0   Section       28  main.o(.constdata)
    m_block_dev_sdc                          0x0002dba0   Data          28  main.o(.constdata)
    .constdata                               0x0002dbbc   Section        8  boards.o(.constdata)
    m_board_led_list                         0x0002dbbc   Data           4  boards.o(.constdata)
    m_board_btn_list                         0x0002dbc0   Data           4  boards.o(.constdata)
    .constdata                               0x0002dbc4   Section       44  bsp.o(.constdata)
    m_bsp_leds_tmr                           0x0002dbc4   Data           4  bsp.o(.constdata)
    m_bsp_alert_tmr                          0x0002dbc8   Data           4  bsp.o(.constdata)
    m_bsp_button_tmr                         0x0002dbcc   Data           4  bsp.o(.constdata)
    app_buttons                              0x0002dbd0   Data          32  bsp.o(.constdata)
    .constdata                               0x0002dbf0   Section       22  nrf_ble_gatt.o(.constdata)
    .constdata                               0x0002dc08   Section       16  ble_nus.o(.constdata)
    .constdata                               0x0002dc18   Section        4  nrfx_gpiote.o(.constdata)
    .constdata                               0x0002dc1c   Section        4  nrfx_uart.o(.constdata)
    irq_handlers                             0x0002dc1c   Data           4  nrfx_uart.o(.constdata)
    .constdata                               0x0002dc20   Section        4  nrfx_uarte.o(.constdata)
    irq_handlers                             0x0002dc20   Data           4  nrfx_uarte.o(.constdata)
    .constdata                               0x0002dc24   Section       16  nrf_drv_spi.o(.constdata)
    .constdata                               0x0002dc34   Section        4  nrfx_spim.o(.constdata)
    irq_handlers                             0x0002dc34   Data           4  nrfx_spim.o(.constdata)
    .constdata                               0x0002dc38   Section       20  app_timer2.o(.constdata)
    m_req_fifo                               0x0002dc38   Data           4  app_timer2.o(.constdata)
    m_app_timer_sortlist                     0x0002dc40   Data          12  app_timer2.o(.constdata)
    .constdata                               0x0002dc4c   Section       16  nrf_fprintf_format.o(.constdata)
    _aV2C                                    0x0002dc4c   Data          16  nrf_fprintf_format.o(.constdata)
    .constdata                               0x0002dc5c   Section       24  nrf_pwr_mgmt.o(.constdata)
    pwr_mgmt_data_array                      0x0002dc5c   Data          24  nrf_pwr_mgmt.o(.constdata)
    .constdata                               0x0002dc74   Section       12  nrf_pwr_mgmt.o(.constdata)
    pwr_mgmt_data                            0x0002dc74   Data          12  nrf_pwr_mgmt.o(.constdata)
    .constdata                               0x0002dc80   Section      316  nrf_strerror.o(.constdata)
    m_unknown_str                            0x0002dc80   Data          19  nrf_strerror.o(.constdata)
    nrf_strerror_array                       0x0002dc94   Data         296  nrf_strerror.o(.constdata)
    .constdata                               0x0002ddbc   Section       32  app_sdcard.o(.constdata)
    m_spi                                    0x0002ddbc   Data          16  app_sdcard.o(.constdata)
    .constdata                               0x0002dddc   Section       24  nrf_block_dev_sdc.o(.constdata)
    .constdata                               0x0002ddf4   Section       72  nrf_block_dev_sdc.o(.constdata)
    .constdata                               0x0002de3c   Section       12  nrf_log_backend_rtt.o(.constdata)
    .constdata                               0x0002de50   Section        6  nrf_log_backend_rtt.o(.constdata)
    delay_machine_code                       0x0002de50   Data           6  nrf_log_backend_rtt.o(.constdata)
    .constdata                               0x0002de58   Section       12  nrf_log_frontend.o(.constdata)
    m_log_push_ringbuf                       0x0002de58   Data          12  nrf_log_frontend.o(.constdata)
    .constdata                               0x0002de64   Section       12  nrf_log_backend_uart.o(.constdata)
    .constdata                               0x0002de70   Section       32  nrf_log_backend_uart.o(.constdata)
    .constdata                               0x0002de90   Section       16  nrf_sdh.o(.constdata)
    sdh_req_observers_array                  0x0002de90   Data          16  nrf_sdh.o(.constdata)
    .constdata                               0x0002dea0   Section       40  nrf_sdh.o(.constdata)
    sdh_req_observers                        0x0002dea4   Data          12  nrf_sdh.o(.constdata)
    sdh_state_observers                      0x0002deb0   Data          12  nrf_sdh.o(.constdata)
    sdh_stack_observers                      0x0002debc   Data          12  nrf_sdh.o(.constdata)
    .constdata                               0x0002dec8   Section       16  nrf_sdh.o(.constdata)
    sdh_state_observers_array                0x0002dec8   Data          16  nrf_sdh.o(.constdata)
    .constdata                               0x0002ded8   Section       16  nrf_sdh.o(.constdata)
    sdh_stack_observers_array                0x0002ded8   Data          16  nrf_sdh.o(.constdata)
    .constdata                               0x0002dee8   Section       32  nrf_sdh_ble.o(.constdata)
    sdh_ble_observers_array                  0x0002dee8   Data          32  nrf_sdh_ble.o(.constdata)
    .constdata                               0x0002df08   Section       16  nrf_sdh_ble.o(.constdata)
    sdh_ble_observers                        0x0002df0c   Data          12  nrf_sdh_ble.o(.constdata)
    .constdata                               0x0002df18   Section       16  nrf_sdh_soc.o(.constdata)
    sdh_soc_observers_array                  0x0002df18   Data          16  nrf_sdh_soc.o(.constdata)
    .constdata                               0x0002df28   Section       12  nrf_sdh_soc.o(.constdata)
    sdh_soc_observers                        0x0002df28   Data          12  nrf_sdh_soc.o(.constdata)
    .constdata                               0x0002df34   Section      129  ctype_o.o(.constdata)
    .constdata                               0x0002dfb8   Section        4  ctype_o.o(.constdata)
    table                                    0x0002dfb8   Data           4  ctype_o.o(.constdata)
    .conststring                             0x0002dfbc   Section       19  main.o(.conststring)
    .conststring                             0x0002dfd0   Section      162  nrf_ble_gatt.o(.conststring)
    .conststring                             0x0002e074   Section     1003  nrf_strerror.o(.conststring)
    .conststring                             0x0002e460   Section      102  nrf_log_str_formatter.o(.conststring)
    .conststring                             0x0002e4c8   Section      463  nrf_sdh_ble.o(.conststring)
    .conststrlit                             0x0002e698   Section       13  nrf_ble_gatt.o(.conststrlit)
    .conststrlit                             0x0002e6a8   Section        8  ble_nus.o(.conststrlit)
    .conststrlit                             0x0002e6b0   Section        6  nrf_drv_clock.o(.conststrlit)
    .conststrlit                             0x0002e6b8   Section        6  nrfx_clock.o(.conststrlit)
    .conststrlit                             0x0002e6c0   Section        7  nrfx_gpiote.o(.conststrlit)
    .conststrlit                             0x0002e6c8   Section        4  nrfx_prs.o(.conststrlit)
    .conststrlit                             0x0002e6cc   Section        5  nrfx_uart.o(.conststrlit)
    .conststrlit                             0x0002e6d4   Section        6  nrfx_uarte.o(.conststrlit)
    .conststrlit                             0x0002e6dc   Section        5  nrfx_spim.o(.conststrlit)
    .conststrlit                             0x0002e6e4   Section       11  app_button.o(.conststrlit)
    .conststrlit                             0x0002e6f0   Section       10  app_timer2.o(.conststrlit)
    .conststrlit                             0x0002e6fc   Section        9  nrf_pwr_mgmt.o(.conststrlit)
    .conststrlit                             0x0002e708   Section        9  nrf_sortlist.o(.conststrlit)
    .conststrlit                             0x0002e714   Section       33  nrf_log_default_backends.o(.conststrlit)
    .conststrlit                             0x0002e738   Section        4  nrf_log_frontend.o(.conststrlit)
    .conststrlit                             0x0002e73c   Section        8  nrf_sdh.o(.conststrlit)
    .conststrlit                             0x0002e744   Section       12  nrf_sdh_ble.o(.conststrlit)
    .conststrlit                             0x0002e750   Section       12  nrf_sdh_soc.o(.conststrlit)
    log_backends                             0x0002e77c   Section       32  nrf_log_default_backends.o(log_backends)
    __tagsym$$used                           0x0002e77c   Number         0  nrf_log_default_backends.o(log_backends)
    rtt_log_backend                          0x0002e77c   Data          16  nrf_log_default_backends.o(log_backends)
    __tagsym$$used                           0x0002e78c   Number         0  nrf_log_default_backends.o(log_backends)
    uart_log_backend                         0x0002e78c   Data          16  nrf_log_default_backends.o(log_backends)
    log_const_data                           0x0002e79c   Section        8  nrf_ble_gatt.o(log_const_data)
    __tagsym$$used                           0x0002e79c   Number         0  nrf_ble_gatt.o(log_const_data)
    log_const_data                           0x0002e7a4   Section        8  ble_nus.o(log_const_data)
    __tagsym$$used                           0x0002e7a4   Number         0  ble_nus.o(log_const_data)
    log_const_data                           0x0002e7ac   Section        8  nrf_drv_clock.o(log_const_data)
    __tagsym$$used                           0x0002e7ac   Number         0  nrf_drv_clock.o(log_const_data)
    log_const_data                           0x0002e7b4   Section        8  nrfx_clock.o(log_const_data)
    __tagsym$$used                           0x0002e7b4   Number         0  nrfx_clock.o(log_const_data)
    log_const_data                           0x0002e7bc   Section        8  nrfx_gpiote.o(log_const_data)
    __tagsym$$used                           0x0002e7bc   Number         0  nrfx_gpiote.o(log_const_data)
    log_const_data                           0x0002e7c4   Section        8  nrfx_prs.o(log_const_data)
    __tagsym$$used                           0x0002e7c4   Number         0  nrfx_prs.o(log_const_data)
    log_const_data                           0x0002e7cc   Section        8  nrfx_uart.o(log_const_data)
    __tagsym$$used                           0x0002e7cc   Number         0  nrfx_uart.o(log_const_data)
    log_const_data                           0x0002e7d4   Section        8  nrfx_uarte.o(log_const_data)
    __tagsym$$used                           0x0002e7d4   Number         0  nrfx_uarte.o(log_const_data)
    log_const_data                           0x0002e7dc   Section        8  nrfx_spim.o(log_const_data)
    __tagsym$$used                           0x0002e7dc   Number         0  nrfx_spim.o(log_const_data)
    log_const_data                           0x0002e7e4   Section        8  app_button.o(log_const_data)
    __tagsym$$used                           0x0002e7e4   Number         0  app_button.o(log_const_data)
    log_const_data                           0x0002e7ec   Section        8  app_timer2.o(log_const_data)
    __tagsym$$used                           0x0002e7ec   Number         0  app_timer2.o(log_const_data)
    log_const_data                           0x0002e7f4   Section        8  nrf_pwr_mgmt.o(log_const_data)
    __tagsym$$used                           0x0002e7f4   Number         0  nrf_pwr_mgmt.o(log_const_data)
    log_const_data                           0x0002e7fc   Section        8  nrf_sortlist.o(log_const_data)
    __tagsym$$used                           0x0002e7fc   Number         0  nrf_sortlist.o(log_const_data)
    log_const_data                           0x0002e804   Section        8  nrf_log_frontend.o(log_const_data)
    __tagsym$$used                           0x0002e804   Number         0  nrf_log_frontend.o(log_const_data)
    log_const_data                           0x0002e80c   Section        8  nrf_sdh.o(log_const_data)
    __tagsym$$used                           0x0002e80c   Number         0  nrf_sdh.o(log_const_data)
    log_const_data                           0x0002e814   Section        8  nrf_sdh_ble.o(log_const_data)
    __tagsym$$used                           0x0002e814   Number         0  nrf_sdh_ble.o(log_const_data)
    log_const_data                           0x0002e81c   Section        8  nrf_sdh_soc.o(log_const_data)
    __tagsym$$used                           0x0002e81c   Number         0  nrf_sdh_soc.o(log_const_data)
    nrf_balloc                               0x0002e824   Section       20  nrf_log_frontend.o(nrf_balloc)
    __tagsym$$used                           0x0002e824   Number         0  nrf_log_frontend.o(nrf_balloc)
    sdh_ble_observers0                       0x0002e838   Section        8  ble_conn_state.o(sdh_ble_observers0)
    __tagsym$$used                           0x0002e838   Number         0  ble_conn_state.o(sdh_ble_observers0)
    m_ble_evt_observer                       0x0002e838   Data           8  ble_conn_state.o(sdh_ble_observers0)
    sdh_ble_observers1                       0x0002e840   Section       16  main.o(sdh_ble_observers1)
    __tagsym$$used                           0x0002e840   Number         0  main.o(sdh_ble_observers1)
    m_gatt_obs                               0x0002e840   Data           8  main.o(sdh_ble_observers1)
    __tagsym$$used                           0x0002e848   Number         0  main.o(sdh_ble_observers1)
    m_advertising_ble_obs                    0x0002e848   Data           8  main.o(sdh_ble_observers1)
    sdh_ble_observers1                       0x0002e850   Section        8  bsp_btn_ble.o(sdh_ble_observers1)
    __tagsym$$used                           0x0002e850   Number         0  bsp_btn_ble.o(sdh_ble_observers1)
    m_ble_observer                           0x0002e850   Data           8  bsp_btn_ble.o(sdh_ble_observers1)
    sdh_ble_observers1                       0x0002e858   Section        8  ble_conn_params.o(sdh_ble_observers1)
    __tagsym$$used                           0x0002e858   Number         0  ble_conn_params.o(sdh_ble_observers1)
    m_ble_observer                           0x0002e858   Data           8  ble_conn_params.o(sdh_ble_observers1)
    sdh_ble_observers2                       0x0002e860   Section       16  main.o(sdh_ble_observers2)
    __tagsym$$used                           0x0002e860   Number         0  main.o(sdh_ble_observers2)
    m_nus_obs                                0x0002e860   Data           8  main.o(sdh_ble_observers2)
    __tagsym$$used                           0x0002e868   Number         0  main.o(sdh_ble_observers2)
    m_qwr_obs                                0x0002e868   Data           8  main.o(sdh_ble_observers2)
    sdh_ble_observers3                       0x0002e870   Section        8  main.o(sdh_ble_observers3)
    __tagsym$$used                           0x0002e870   Number         0  main.o(sdh_ble_observers3)
    m_ble_observer                           0x0002e870   Data           8  main.o(sdh_ble_observers3)
    sdh_soc_observers0                       0x0002e878   Section        8  nrf_drv_clock.o(sdh_soc_observers0)
    __tagsym$$used                           0x0002e878   Number         0  nrf_drv_clock.o(sdh_soc_observers0)
    m_soc_evt_observer                       0x0002e878   Data           8  nrf_drv_clock.o(sdh_soc_observers0)
    sdh_stack_observers0                     0x0002e880   Section        8  nrf_sdh_ble.o(sdh_stack_observers0)
    __tagsym$$used                           0x0002e880   Number         0  nrf_sdh_ble.o(sdh_stack_observers0)
    m_nrf_sdh_ble_evts_poll                  0x0002e880   Data           8  nrf_sdh_ble.o(sdh_stack_observers0)
    sdh_stack_observers0                     0x0002e888   Section        8  nrf_sdh_soc.o(sdh_stack_observers0)
    __tagsym$$used                           0x0002e888   Number         0  nrf_sdh_soc.o(sdh_stack_observers0)
    m_nrf_sdh_soc_evts_poll                  0x0002e888   Data           8  nrf_sdh_soc.o(sdh_stack_observers0)
    sdh_state_observers0                     0x0002e890   Section        8  nrf_drv_clock.o(sdh_state_observers0)
    __tagsym$$used                           0x0002e890   Number         0  nrf_drv_clock.o(sdh_state_observers0)
    m_sd_state_observer                      0x0002e890   Data           8  nrf_drv_clock.o(sdh_state_observers0)
    .data                                    0x20002ad8   Section       60  main.o(.data)
    m_conn_handle                            0x20002adc   Data           2  main.o(.data)
    m_ble_nus_max_data_len                   0x20002ade   Data           2  main.o(.data)
    m_adv_uuids                              0x20002ae4   Data           4  main.o(.data)
    data_buffer                              0x20002ae8   Data           4  main.o(.data)
    m_nus                                    0x20002aec   Data          28  main.o(.data)
    drives                                   0x20002b08   Data          12  main.o(.data)
    .data                                    0x20002b14   Section        8  main.o(.data)
    m_nus_link_ctx_storage                   0x20002b14   Data           8  main.o(.data)
    .data                                    0x20002b1c   Section        4  main.o(.data)
    m_nus_link_ctx_storage_ctx_data_pool     0x20002b1c   Data           4  main.o(.data)
    .data                                    0x20002b20   Section       16  bsp.o(.data)
    m_stable_state                           0x20002b20   Data           1  bsp.o(.data)
    m_leds_clear                             0x20002b21   Data           1  bsp.o(.data)
    m_alert_on                               0x20002b22   Data           1  bsp.o(.data)
    current_long_push_pin_no                 0x20002b23   Data           1  bsp.o(.data)
    m_indication_type                        0x20002b24   Data           4  bsp.o(.data)
    m_registered_callback                    0x20002b28   Data           4  bsp.o(.data)
    release_event_at_push                    0x20002b2c   Data           4  bsp.o(.data)
    .data                                    0x20002b30   Section        8  bsp_btn_ble.o(.data)
    m_error_handler                          0x20002b30   Data           4  bsp_btn_ble.o(.data)
    m_num_connections                        0x20002b34   Data           4  bsp_btn_ble.o(.data)
    .data                                    0x20002b38   Section        8  ble_conn_params.o(.data)
    m_preferred_conn_params                  0x20002b38   Data           8  ble_conn_params.o(.data)
    .data                                    0x20002b40   Section       12  nrf_drv_uart.o(.data)
    m_handlers                               0x20002b44   Data           4  nrf_drv_uart.o(.data)
    m_contexts                               0x20002b48   Data           4  nrf_drv_uart.o(.data)
    .data                                    0x20002b4c   Section        8  nrfx_clock.o(.data)
    m_clock_cb                               0x20002b4c   Data           8  nrfx_clock.o(.data)
    .data                                    0x20002b54   Section        8  nrfx_prs.o(.data)
    m_prs_box_4                              0x20002b54   Data           8  nrfx_prs.o(.data)
    .data                                    0x20002b60   Section       32  app_timer2.o(.data)
    m_global_active                          0x20002b60   Data           1  app_timer2.o(.data)
    mp_active_timer                          0x20002b64   Data           4  app_timer2.o(.data)
    m_rtc_inst                               0x20002b68   Data           8  app_timer2.o(.data)
    m_base_counter                           0x20002b70   Data           8  app_timer2.o(.data)
    m_stamp64                                0x20002b78   Data           8  app_timer2.o(.data)
    .data                                    0x20002b80   Section        4  app_timer2.o(.data)
    m_app_timer_sortlist_sortlist_cb         0x20002b80   Data           4  app_timer2.o(.data)
    .data                                    0x20002b84   Section       28  app_uart_fifo.o(.data)
    tx_buffer                                0x20002b84   Data           1  app_uart_fifo.o(.data)
    rx_buffer                                0x20002b85   Data           1  app_uart_fifo.o(.data)
    m_rx_ovf                                 0x20002b86   Data           1  app_uart_fifo.o(.data)
    m_event_handler                          0x20002b88   Data           4  app_uart_fifo.o(.data)
    app_uart_inst                            0x20002b8c   Data          20  app_uart_fifo.o(.data)
    .data                                    0x20002ba0   Section       12  drv_rtc.o(.data)
    m_handlers                               0x20002ba0   Data           4  drv_rtc.o(.data)
    m_cb                                     0x20002ba4   Data           8  drv_rtc.o(.data)
    .data                                    0x20002bac   Section        8  nrf_pwr_mgmt.o(.data)
    m_pwr_mgmt_evt                           0x20002bac   Data           1  nrf_pwr_mgmt.o(.data)
    m_shutdown_started                       0x20002bad   Data           1  nrf_pwr_mgmt.o(.data)
    m_sysoff_mtx                             0x20002bb0   Data           4  nrf_pwr_mgmt.o(.data)
    .data                                    0x20002bb4   Section        8  nrf_block_dev_sdc.o(.data)
    m_last_result                            0x20002bb4   Data           1  nrf_block_dev_sdc.o(.data)
    m_active_sdc_dev                         0x20002bb8   Data           4  nrf_block_dev_sdc.o(.data)
    .data                                    0x20002bbc   Section        1  nrf_log_backend_rtt.o(.data)
    m_host_present                           0x20002bbc   Data           1  nrf_log_backend_rtt.o(.data)
    .data                                    0x20002bc0   Section        8  nrf_log_default_backends.o(.data)
    log_backend_cb_rtt_log_backend           0x20002bc0   Data           8  nrf_log_default_backends.o(.data)
    .data                                    0x20002bc8   Section        8  nrf_log_default_backends.o(.data)
    log_backend_cb_uart_log_backend          0x20002bc8   Data           8  nrf_log_default_backends.o(.data)
    .data                                    0x20002bd0   Section        4  nrf_log_frontend.o(.data)
    m_buffer_mask                            0x20002bd0   Data           4  nrf_log_frontend.o(.data)
    .data                                    0x20002bd4   Section        8  nrf_log_frontend.o(.data)
    log_mempool_nrf_balloc_pool_stack        0x20002bd4   Data           8  nrf_log_frontend.o(.data)
    .data                                    0x20002bdc   Section        8  nrf_log_frontend.o(.data)
    log_mempool_nrf_balloc_cb                0x20002bdc   Data           8  nrf_log_frontend.o(.data)
    .data                                    0x20002be4   Section       64  nrf_log_str_formatter.o(.data)
    m_freq                                   0x20002be4   Data           4  nrf_log_str_formatter.o(.data)
    m_timestamp_div                          0x20002be8   Data           4  nrf_log_str_formatter.o(.data)
    severity_names                           0x20002bec   Data          20  nrf_log_str_formatter.o(.data)
    m_colors                                 0x20002c00   Data          36  nrf_log_str_formatter.o(.data)
    .data                                    0x20002c24   Section       24  nrf_log_backend_uart.o(.data)
    m_xfer_done                              0x20002c24   Data           1  nrf_log_backend_uart.o(.data)
    m_async_mode                             0x20002c25   Data           1  nrf_log_backend_uart.o(.data)
    .data                                    0x20002c3c   Section        3  nrf_sdh.o(.data)
    m_nrf_sdh_enabled                        0x20002c3c   Data           1  nrf_sdh.o(.data)
    m_nrf_sdh_suspended                      0x20002c3d   Data           1  nrf_sdh.o(.data)
    m_nrf_sdh_continue                       0x20002c3e   Data           1  nrf_sdh.o(.data)
    .data                                    0x20002c3f   Section        1  nrf_sdh_ble.o(.data)
    m_stack_is_enabled                       0x20002c3f   Data           1  nrf_sdh_ble.o(.data)
    .data                                    0x20002c40   Section        8  diskio_blkdev.o(.data)
    m_drives_count                           0x20002c40   Data           1  diskio_blkdev.o(.data)
    m_drives                                 0x20002c44   Data           4  diskio_blkdev.o(.data)
    .data                                    0x20002c48   Section        8  ff.o(.data)
    Fsid                                     0x20002c48   Data           2  ff.o(.data)
    FatFs                                    0x20002c4c   Data           4  ff.o(.data)
    .data                                    0x20002c50   Section        4  system_nrf52.o(.data)
    __tagsym$$used                           0x20002c50   Number         0  system_nrf52.o(.data)
    .bss                                     0x20002c54   Section    32292  main.o(.bss)
    fs                                       0x20002c54   Data         560  main.o(.bss)
    dir                                      0x20002e84   Data          44  main.o(.bss)
    fno                                      0x20002eb0   Data          24  main.o(.bss)
    file                                     0x20002ec8   Data         552  main.o(.bss)
    m_gatt                                   0x2000a624   Data          20  main.o(.bss)
    m_qwr                                    0x2000a638   Data          12  main.o(.bss)
    m_advertising                            0x2000a644   Data        1076  main.o(.bss)
    .bss                                     0x2000aa78   Section       28  main.o(.bss)
    m_block_dev_sdc_work                     0x2000aa78   Data          28  main.o(.bss)
    .bss                                     0x2000aa98   Section       32  bsp.o(.bss)
    m_bsp_leds_tmr_data                      0x2000aa98   Data          32  bsp.o(.bss)
    .bss                                     0x2000aab8   Section       32  bsp.o(.bss)
    m_bsp_alert_tmr_data                     0x2000aab8   Data          32  bsp.o(.bss)
    .bss                                     0x2000aad8   Section       12  bsp.o(.bss)
    m_events_list                            0x2000aad8   Data          12  bsp.o(.bss)
    .bss                                     0x2000aae8   Section       32  bsp.o(.bss)
    m_bsp_button_tmr_data                    0x2000aae8   Data          32  bsp.o(.bss)
    .bss                                     0x2000ab08   Section       80  ble_conn_params.o(.bss)
    m_timer_data                             0x2000ab08   Data          32  ble_conn_params.o(.bss)
    m_conn_params_instances                  0x2000ab28   Data          20  ble_conn_params.o(.bss)
    m_conn_params_config                     0x2000ab3c   Data          28  ble_conn_params.o(.bss)
    .bss                                     0x2000ab58   Section      124  ble_conn_state.o(.bss)
    m_bcs                                    0x2000ab58   Data         124  ble_conn_state.o(.bss)
    .bss                                     0x2000abd4   Section       20  nrf_drv_clock.o(.bss)
    m_clock_cb                               0x2000abd4   Data          20  nrf_drv_clock.o(.bss)
    .bss                                     0x2000abe8   Section       92  nrfx_gpiote.o(.bss)
    m_cb                                     0x2000abe8   Data          92  nrfx_gpiote.o(.bss)
    .bss                                     0x2000ac44   Section       44  nrfx_uart.o(.bss)
    m_cb                                     0x2000ac44   Data          44  nrfx_uart.o(.bss)
    .bss                                     0x2000ac70   Section       36  nrfx_uarte.o(.bss)
    m_cb                                     0x2000ac70   Data          36  nrfx_uarte.o(.bss)
    .bss                                     0x2000ac94   Section       24  nrf_drv_spi.o(.bss)
    m_handlers                               0x2000ac94   Data          12  nrf_drv_spi.o(.bss)
    m_contexts                               0x2000aca0   Data          12  nrf_drv_spi.o(.bss)
    .bss                                     0x2000acac   Section       36  nrfx_spim.o(.bss)
    m_cb                                     0x2000acac   Data          36  nrfx_spim.o(.bss)
    .bss                                     0x2000acd0   Section       16  app_timer2.o(.bss)
    m_req_fifo_inst                          0x2000acd0   Data          16  app_timer2.o(.bss)
    .bss                                     0x2000ace0   Section       32  app_uart_fifo.o(.bss)
    m_rx_fifo                                0x2000ace0   Data          16  app_uart_fifo.o(.bss)
    m_tx_fifo                                0x2000acf0   Data          16  app_uart_fifo.o(.bss)
    .bss                                     0x2000ad00   Section       12  app_util_platform.o(.bss)
    .bss                                     0x2000ad0c   Section       12  nrf_pwr_mgmt.o(.bss)
    m_handlers_iter                          0x2000ad0c   Data          12  nrf_pwr_mgmt.o(.bss)
    .bss                                     0x2000ad18   Section       92  app_sdcard.o(.bss)
    m_cb                                     0x2000ad18   Data          92  app_sdcard.o(.bss)
    .bss                                     0x2000ad74   Section       64  nrf_log_backend_rtt.o(.bss)
    m_string_buff                            0x2000ad74   Data          64  nrf_log_backend_rtt.o(.bss)
    .bss                                     0x2000adb4   Section      192  nrf_log_frontend.o(.bss)
    log_mempool_nrf_balloc_pool_mem          0x2000adb4   Data         192  nrf_log_frontend.o(.bss)
    .bss                                     0x2000ae74   Section      128  nrf_log_frontend.o(.bss)
    m_log_push_ringbuf_buf                   0x2000ae74   Data         128  nrf_log_frontend.o(.bss)
    .bss                                     0x2000aef4   Section       24  nrf_log_frontend.o(.bss)
    m_log_push_ringbuf_cb                    0x2000aef4   Data          24  nrf_log_frontend.o(.bss)
    .bss                                     0x2000af0c   Section     1056  nrf_log_frontend.o(.bss)
    m_log_data                               0x2000af0c   Data        1056  nrf_log_frontend.o(.bss)
    .bss                                     0x2000b32c   Section       64  nrf_log_backend_uart.o(.bss)
    m_string_buff                            0x2000b32c   Data          64  nrf_log_backend_uart.o(.bss)
    .bss                                     0x2000b36c   Section      648  segger_rtt.o(.bss)
    _acUpBuffer                              0x2000b3e4   Data         512  segger_rtt.o(.bss)
    _acDownBuffer                            0x2000b5e4   Data          16  segger_rtt.o(.bss)
    STACK                                    0x2000b5f8   Section     8192  arm_startup_nrf52.o(STACK)

    Global Symbols

    Symbol Name                              Value     Ov Type        Size  Object(Section)

    BuildAttributes$$THM_ISAv4$E$P$D$K$B$S$7EM$VFPi3$EXTD16$VFPS$VFMA$PE$A:L22UL41UL21$X:L11$S22US41US21$IEEE1$IW$USESV6$~STKCKD$USESV7$~SHL$OSPACE$ROPI$EBA8$MICROLIB$REQ8$EABIv2 0x00000000   Number         0  anon$$obj.o ABSOLUTE
    __ARM_use_no_argv                        0x00000000   Number         0  main.o ABSOLUTE
    _printf_a                                0x00000000   Number         0  stubs.o ABSOLUTE
    _printf_c                                0x00000000   Number         0  stubs.o ABSOLUTE
    _printf_charcount                        0x00000000   Number         0  stubs.o ABSOLUTE
    _printf_d                                0x00000000   Number         0  stubs.o ABSOLUTE
    _printf_e                                0x00000000   Number         0  stubs.o ABSOLUTE
    _printf_f                                0x00000000   Number         0  stubs.o ABSOLUTE
    _printf_flags                            0x00000000   Number         0  stubs.o ABSOLUTE
    _printf_fp_dec                           0x00000000   Number         0  stubs.o ABSOLUTE
    _printf_fp_hex                           0x00000000   Number         0  stubs.o ABSOLUTE
    _printf_g                                0x00000000   Number         0  stubs.o ABSOLUTE
    _printf_i                                0x00000000   Number         0  stubs.o ABSOLUTE
    _printf_int_dec                          0x00000000   Number         0  stubs.o ABSOLUTE
    _printf_l                                0x00000000   Number         0  stubs.o ABSOLUTE
    _printf_lc                               0x00000000   Number         0  stubs.o ABSOLUTE
    _printf_ll                               0x00000000   Number         0  stubs.o ABSOLUTE
    _printf_lld                              0x00000000   Number         0  stubs.o ABSOLUTE
    _printf_lli                              0x00000000   Number         0  stubs.o ABSOLUTE
    _printf_llo                              0x00000000   Number         0  stubs.o ABSOLUTE
    _printf_llu                              0x00000000   Number         0  stubs.o ABSOLUTE
    _printf_llx                              0x00000000   Number         0  stubs.o ABSOLUTE
    _printf_longlong_dec                     0x00000000   Number         0  stubs.o ABSOLUTE
    _printf_longlong_hex                     0x00000000   Number         0  stubs.o ABSOLUTE
    _printf_longlong_oct                     0x00000000   Number         0  stubs.o ABSOLUTE
    _printf_ls                               0x00000000   Number         0  stubs.o ABSOLUTE
    _printf_mbtowc                           0x00000000   Number         0  stubs.o ABSOLUTE
    _printf_n                                0x00000000   Number         0  stubs.o ABSOLUTE
    _printf_o                                0x00000000   Number         0  stubs.o ABSOLUTE
    _printf_p                                0x00000000   Number         0  stubs.o ABSOLUTE
    _printf_percent                          0x00000000   Number         0  stubs.o ABSOLUTE
    _printf_pre_padding                      0x00000000   Number         0  stubs.o ABSOLUTE
    _printf_return_value                     0x00000000   Number         0  stubs.o ABSOLUTE
    _printf_s                                0x00000000   Number         0  stubs.o ABSOLUTE
    _printf_sizespec                         0x00000000   Number         0  stubs.o ABSOLUTE
    _printf_str                              0x00000000   Number         0  stubs.o ABSOLUTE
    _printf_truncate_signed                  0x00000000   Number         0  stubs.o ABSOLUTE
    _printf_truncate_unsigned                0x00000000   Number         0  stubs.o ABSOLUTE
    _printf_u                                0x00000000   Number         0  stubs.o ABSOLUTE
    _printf_wc                               0x00000000   Number         0  stubs.o ABSOLUTE
    _printf_wctomb                           0x00000000   Number         0  stubs.o ABSOLUTE
    _printf_widthprec                        0x00000000   Number         0  stubs.o ABSOLUTE
    _printf_x                                0x00000000   Number         0  stubs.o ABSOLUTE
    __cpp_initialize__aeabi_                  - Undefined Weak Reference
    __cxa_finalize                            - Undefined Weak Reference
    _clock_init                               - Undefined Weak Reference
    _microlib_exit                            - Undefined Weak Reference
    log_dynamic_data$$Base                    - Undefined Reference
    pwr_mgmt_data0$$Base                      - Undefined Reference
    pwr_mgmt_data0$$Limit                     - Undefined Reference
    pwr_mgmt_data1$$Base                      - Undefined Reference
    pwr_mgmt_data1$$Limit                     - Undefined Reference
    pwr_mgmt_data2$$Base                      - Undefined Reference
    pwr_mgmt_data2$$Limit                     - Undefined Reference
    sdh_req_observers0$$Base                  - Undefined Reference
    sdh_req_observers0$$Limit                 - Undefined Reference
    sdh_req_observers1$$Base                  - Undefined Reference
    sdh_req_observers1$$Limit                 - Undefined Reference
    sdh_soc_observers1$$Base                  - Undefined Reference
    sdh_soc_observers1$$Limit                 - Undefined Reference
    sdh_stack_observers1$$Base                - Undefined Reference
    sdh_stack_observers1$$Limit               - Undefined Reference
    sdh_state_observers1$$Base                - Undefined Reference
    sdh_state_observers1$$Limit               - Undefined Reference
    __Vectors_Size                           0x00000200   Number         0  arm_startup_nrf52.o ABSOLUTE
    __Vectors                                0x00026000   Data           4  arm_startup_nrf52.o(RESET)
    __Vectors_End                            0x00026200   Data           0  arm_startup_nrf52.o(RESET)
    __main                                   0x00026201   Thumb Code     0  entry.o(.ARM.Collect$$$$00000000)
    _main_stk                                0x00026201   Thumb Code     0  entry2.o(.ARM.Collect$$$$00000001)
    _main_scatterload                        0x00026205   Thumb Code     0  entry5.o(.ARM.Collect$$$$00000004)
    __main_after_scatterload                 0x00026209   Thumb Code     0  entry5.o(.ARM.Collect$$$$00000004)
    _main_clock                              0x00026209   Thumb Code     0  entry7b.o(.ARM.Collect$$$$00000008)
    _main_cpp_init                           0x00026209   Thumb Code     0  entry8b.o(.ARM.Collect$$$$0000000A)
    _main_init                               0x00026209   Thumb Code     0  entry9a.o(.ARM.Collect$$$$0000000B)
    __rt_final_cpp                           0x00026211   Thumb Code     0  entry10a.o(.ARM.Collect$$$$0000000D)
    __rt_final_exit                          0x00026211   Thumb Code     0  entry11a.o(.ARM.Collect$$$$0000000F)
    __asm___12_nrf_atfifo_c_51f461e1__nrf_atfifo_wspace_req 0x00026215   Thumb Code    56  nrf_atfifo.o(.emb_text)
    __asm___12_nrf_atfifo_c_51f461e1__nrf_atfifo_wspace_close 0x0002624d   Thumb Code    18  nrf_atfifo.o(.emb_text)
    __asm___12_nrf_atfifo_c_51f461e1__nrf_atfifo_rspace_req 0x0002625f   Thumb Code    58  nrf_atfifo.o(.emb_text)
    __asm___12_nrf_atfifo_c_51f461e1__nrf_atfifo_rspace_close 0x00026299   Thumb Code    18  nrf_atfifo.o(.emb_text)
    __asm___12_nrf_atfifo_c_51f461e1__nrf_atfifo_space_clear 0x000262ab   Thumb Code    50  nrf_atfifo.o(.emb_text)
    __asm___12_nrf_atomic_c_85ca2469__nrf_atomic_internal_mov 0x000262dd   Thumb Code    24  nrf_atomic.o(.emb_text)
    __asm___12_nrf_atomic_c_85ca2469__nrf_atomic_internal_orr 0x000262f5   Thumb Code    26  nrf_atomic.o(.emb_text)
    __asm___12_nrf_atomic_c_85ca2469__nrf_atomic_internal_and 0x0002630f   Thumb Code    26  nrf_atomic.o(.emb_text)
    __asm___12_nrf_atomic_c_85ca2469__nrf_atomic_internal_eor 0x00026329   Thumb Code    26  nrf_atomic.o(.emb_text)
    __asm___12_nrf_atomic_c_85ca2469__nrf_atomic_internal_add 0x00026343   Thumb Code    26  nrf_atomic.o(.emb_text)
    __asm___12_nrf_atomic_c_85ca2469__nrf_atomic_internal_sub 0x0002635d   Thumb Code    26  nrf_atomic.o(.emb_text)
    __asm___12_nrf_atomic_c_85ca2469__nrf_atomic_internal_cmp_exch 0x00026377   Thumb Code    42  nrf_atomic.o(.emb_text)
    __asm___12_nrf_atomic_c_85ca2469__nrf_atomic_internal_sub_hs 0x000263a1   Thumb Code    30  nrf_atomic.o(.emb_text)
    Reset_Handler                            0x000263c1   Thumb Code     8  arm_startup_nrf52.o(.text)
    NMI_Handler                              0x000263c9   Thumb Code     2  arm_startup_nrf52.o(.text)
    HardFault_Handler                        0x000263cb   Thumb Code     2  arm_startup_nrf52.o(.text)
    MemoryManagement_Handler                 0x000263cd   Thumb Code     2  arm_startup_nrf52.o(.text)
    BusFault_Handler                         0x000263cf   Thumb Code     2  arm_startup_nrf52.o(.text)
    UsageFault_Handler                       0x000263d1   Thumb Code     2  arm_startup_nrf52.o(.text)
    SVC_Handler                              0x000263d3   Thumb Code     2  arm_startup_nrf52.o(.text)
    DebugMon_Handler                         0x000263d5   Thumb Code     2  arm_startup_nrf52.o(.text)
    PendSV_Handler                           0x000263d7   Thumb Code     2  arm_startup_nrf52.o(.text)
    SysTick_Handler                          0x000263d9   Thumb Code     2  arm_startup_nrf52.o(.text)
    CCM_AAR_IRQHandler                       0x000263db   Thumb Code     0  arm_startup_nrf52.o(.text)
    COMP_LPCOMP_IRQHandler                   0x000263db   Thumb Code     0  arm_startup_nrf52.o(.text)
    ECB_IRQHandler                           0x000263db   Thumb Code     0  arm_startup_nrf52.o(.text)
    FPU_IRQHandler                           0x000263db   Thumb Code     0  arm_startup_nrf52.o(.text)
    I2S_IRQHandler                           0x000263db   Thumb Code     0  arm_startup_nrf52.o(.text)
    MWU_IRQHandler                           0x000263db   Thumb Code     0  arm_startup_nrf52.o(.text)
    NFCT_IRQHandler                          0x000263db   Thumb Code     0  arm_startup_nrf52.o(.text)
    PDM_IRQHandler                           0x000263db   Thumb Code     0  arm_startup_nrf52.o(.text)
    PWM0_IRQHandler                          0x000263db   Thumb Code     0  arm_startup_nrf52.o(.text)
    PWM1_IRQHandler                          0x000263db   Thumb Code     0  arm_startup_nrf52.o(.text)
    PWM2_IRQHandler                          0x000263db   Thumb Code     0  arm_startup_nrf52.o(.text)
    QDEC_IRQHandler                          0x000263db   Thumb Code     0  arm_startup_nrf52.o(.text)
    RADIO_IRQHandler                         0x000263db   Thumb Code     0  arm_startup_nrf52.o(.text)
    RNG_IRQHandler                           0x000263db   Thumb Code     0  arm_startup_nrf52.o(.text)
    RTC0_IRQHandler                          0x000263db   Thumb Code     0  arm_startup_nrf52.o(.text)
    RTC2_IRQHandler                          0x000263db   Thumb Code     0  arm_startup_nrf52.o(.text)
    SAADC_IRQHandler                         0x000263db   Thumb Code     0  arm_startup_nrf52.o(.text)
    SPIM1_SPIS1_TWIM1_TWIS1_SPI1_TWI1_IRQHandler 0x000263db   Thumb Code     0  arm_startup_nrf52.o(.text)
    SPIM2_SPIS2_SPI2_IRQHandler              0x000263db   Thumb Code     0  arm_startup_nrf52.o(.text)
    SWI0_EGU0_IRQHandler                     0x000263db   Thumb Code     0  arm_startup_nrf52.o(.text)
    SWI1_EGU1_IRQHandler                     0x000263db   Thumb Code     0  arm_startup_nrf52.o(.text)
    SWI3_EGU3_IRQHandler                     0x000263db   Thumb Code     0  arm_startup_nrf52.o(.text)
    SWI4_EGU4_IRQHandler                     0x000263db   Thumb Code     0  arm_startup_nrf52.o(.text)
    SWI5_EGU5_IRQHandler                     0x000263db   Thumb Code     0  arm_startup_nrf52.o(.text)
    TEMP_IRQHandler                          0x000263db   Thumb Code     0  arm_startup_nrf52.o(.text)
    TIMER0_IRQHandler                        0x000263db   Thumb Code     0  arm_startup_nrf52.o(.text)
    TIMER1_IRQHandler                        0x000263db   Thumb Code     0  arm_startup_nrf52.o(.text)
    TIMER3_IRQHandler                        0x000263db   Thumb Code     0  arm_startup_nrf52.o(.text)
    TIMER4_IRQHandler                        0x000263db   Thumb Code     0  arm_startup_nrf52.o(.text)
    WDT_IRQHandler                           0x000263db   Thumb Code     0  arm_startup_nrf52.o(.text)
    __aeabi_uldivmod                         0x000263e5   Thumb Code    98  uldiv.o(.text)
    __aeabi_llsl                             0x00026447   Thumb Code    30  llshl.o(.text)
    _ll_shift_l                              0x00026447   Thumb Code     0  llshl.o(.text)
    __rt_ctype_table                         0x00026465   Thumb Code     4  ctype_o.o(.text)
    __aeabi_memcpy                           0x0002646d   Thumb Code    36  memcpya.o(.text)
    __aeabi_memcpy4                          0x0002646d   Thumb Code     0  memcpya.o(.text)
    __aeabi_memcpy8                          0x0002646d   Thumb Code     0  memcpya.o(.text)
    __aeabi_memset                           0x00026491   Thumb Code    14  memseta.o(.text)
    __aeabi_memset4                          0x00026491   Thumb Code     0  memseta.o(.text)
    __aeabi_memset8                          0x00026491   Thumb Code     0  memseta.o(.text)
    __aeabi_memclr                           0x0002649f   Thumb Code     4  memseta.o(.text)
    __aeabi_memclr4                          0x0002649f   Thumb Code     0  memseta.o(.text)
    __aeabi_memclr8                          0x0002649f   Thumb Code     0  memseta.o(.text)
    _memset$wrapper                          0x000264a3   Thumb Code    18  memseta.o(.text)
    strlen                                   0x000264b5   Thumb Code    14  strlen.o(.text)
    strcpy                                   0x000264c3   Thumb Code    18  strcpy.o(.text)
    __aeabi_uidiv                            0x000264d5   Thumb Code     0  uidiv.o(.text)
    __aeabi_uidivmod                         0x000264d5   Thumb Code    44  uidiv.o(.text)
    __aeabi_llsr                             0x00026501   Thumb Code    32  llushr.o(.text)
    _ll_ushift_r                             0x00026501   Thumb Code     0  llushr.o(.text)
    __scatterload                            0x00026521   Thumb Code    28  init.o(.text)
    __scatterload_rt2                        0x00026521   Thumb Code     0  init.o(.text)
    __decompress                             0x00026545   Thumb Code     0  __dczerorl2.o(.text)
    __decompress1                            0x00026545   Thumb Code    86  __dczerorl2.o(.text)
    GPIOTE_IRQHandler                        0x0002659d   Thumb Code   154  nrfx_gpiote.o(i.GPIOTE_IRQHandler)
    POWER_CLOCK_IRQHandler                   0x00026641   Thumb Code    82  nrfx_clock.o(i.POWER_CLOCK_IRQHandler)
    RTC1_IRQHandler                          0x00026699   Thumb Code    12  drv_rtc.o(i.RTC1_IRQHandler)
    SEGGER_RTT_Init                          0x000266a9   Thumb Code     4  segger_rtt.o(i.SEGGER_RTT_Init)
    SEGGER_RTT_WriteNoLock                   0x000266ad   Thumb Code    86  segger_rtt.o(i.SEGGER_RTT_WriteNoLock)
    SPIM0_SPIS0_TWIM0_TWIS0_SPI0_TWI0_IRQHandler 0x00026709   Thumb Code    76  nrfx_spim.o(i.SPIM0_SPIS0_TWIM0_TWIS0_SPI0_TWI0_IRQHandler)
    SWI2_EGU2_IRQHandler                     0x0002675d   Thumb Code     4  nrf_sdh.o(i.SWI2_EGU2_IRQHandler)
    SystemInit                               0x00026761   Thumb Code   112  system_nrf52.o(i.SystemInit)
    TIMER2_IRQHandler                        0x000267e5   Thumb Code   124  main.o(i.TIMER2_IRQHandler)
    UARTE0_UART0_IRQHandler                  0x00026875   Thumb Code     6  nrfx_prs.o(i.UARTE0_UART0_IRQHandler)
    __0sprintf$1                             0x0002699d   Thumb Code    34  printf1.o(i.__0sprintf$1)
    __1sprintf$1                             0x0002699d   Thumb Code     0  printf1.o(i.__0sprintf$1)
    __2sprintf                               0x0002699d   Thumb Code     0  printf1.o(i.__0sprintf$1)
    __scatterload_copy                       0x000269c5   Thumb Code    14  handlers.o(i.__scatterload_copy)
    __scatterload_null                       0x000269d3   Thumb Code     2  handlers.o(i.__scatterload_null)
    __scatterload_zeroinit                   0x000269d5   Thumb Code    14  handlers.o(i.__scatterload_zeroinit)
    app_error_fault_handler                  0x00026bad   Thumb Code    86  app_error_weak.o(i.app_error_fault_handler)
    app_error_handler_bare                   0x00026c31   Thumb Code    22  app_error.o(i.app_error_handler_bare)
    app_fifo_get                             0x00026c47   Thumb Code    22  app_fifo.o(i.app_fifo_get)
    app_fifo_put                             0x00026c5d   Thumb Code    26  app_fifo.o(i.app_fifo_put)
    app_sdc_block_read                       0x00026c79   Thumb Code    84  app_sdcard.o(i.app_sdc_block_read)
    app_sdc_block_write                      0x00026cd1   Thumb Code   104  app_sdcard.o(i.app_sdc_block_write)
    app_sdc_busy_check                       0x00026d3d   Thumb Code    24  app_sdcard.o(i.app_sdc_busy_check)
    app_sdc_info_get                         0x00026d59   Thumb Code    18  app_sdcard.o(i.app_sdc_info_get)
    app_sdc_init                             0x00026d71   Thumb Code   190  app_sdcard.o(i.app_sdc_init)
    app_sdc_uninit                           0x00026e3d   Thumb Code    62  app_sdcard.o(i.app_sdc_uninit)
    app_timer_create                         0x00026e85   Thumb Code    22  app_timer2.o(i.app_timer_create)
    app_timer_start                          0x00026e9b   Thumb Code    48  app_timer2.o(i.app_timer_start)
    app_timer_stop                           0x00026ecb   Thumb Code    12  app_timer2.o(i.app_timer_stop)
    app_uart_put                             0x00026ed9   Thumb Code    70  app_uart_fifo.o(i.app_uart_put)
    app_util_critical_region_enter           0x00026f2d   Thumb Code    64  app_util_platform.o(i.app_util_critical_region_enter)
    app_util_critical_region_exit            0x00026f75   Thumb Code    46  app_util_platform.o(i.app_util_critical_region_exit)
    blcm_link_ctx_get                        0x000270b9   Thumb Code    72  ble_link_ctx_manager.o(i.blcm_link_ctx_get)
    ble_advdata_encode                       0x00027101   Thumb Code   386  ble_advdata.o(i.ble_advdata_encode)
    ble_advdata_parse                        0x00027283   Thumb Code    32  ble_advdata.o(i.ble_advdata_parse)
    ble_advdata_search                       0x000272a3   Thumb Code    70  ble_advdata.o(i.ble_advdata_search)
    ble_advertising_conn_cfg_tag_set         0x000272e9   Thumb Code     6  ble_advertising.o(i.ble_advertising_conn_cfg_tag_set)
    ble_advertising_init                     0x000272ef   Thumb Code   248  ble_advertising.o(i.ble_advertising_init)
    ble_advertising_on_ble_evt               0x000273e7   Thumb Code   106  ble_advertising.o(i.ble_advertising_on_ble_evt)
    ble_advertising_start                    0x00027451   Thumb Code   560  ble_advertising.o(i.ble_advertising_start)
    ble_conn_params_init                     0x00027681   Thumb Code    90  ble_conn_params.o(i.ble_conn_params_init)
    ble_conn_state_conn_idx                  0x000276e9   Thumb Code    18  ble_conn_state.o(i.ble_conn_state_conn_idx)
    ble_conn_state_valid                     0x000276fd   Thumb Code    16  ble_conn_state.o(i.ble_conn_state_valid)
    ble_nus_init                             0x00027ad1   Thumb Code   206  ble_nus.o(i.ble_nus_init)
    ble_nus_on_ble_evt                       0x00027ba5   Thumb Code   118  ble_nus.o(i.ble_nus_on_ble_evt)
    ble_srv_is_notification_enabled          0x00027c1b   Thumb Code     8  ble_srv_common.o(i.ble_srv_is_notification_enabled)
    bsp_board_button_idx_to_pin              0x00027e35   Thumb Code     6  boards.o(i.bsp_board_button_idx_to_pin)
    bsp_board_led_invert                     0x00027e41   Thumb Code    32  boards.o(i.bsp_board_led_invert)
    bsp_board_led_off                        0x00027e65   Thumb Code    10  boards.o(i.bsp_board_led_off)
    bsp_board_led_on                         0x00027e75   Thumb Code    10  boards.o(i.bsp_board_led_on)
    bsp_board_led_state_get                  0x00027e85   Thumb Code    28  boards.o(i.bsp_board_led_state_get)
    bsp_board_leds_off                       0x00027ea5   Thumb Code    18  boards.o(i.bsp_board_leds_off)
    bsp_board_leds_on                        0x00027eb7   Thumb Code    18  boards.o(i.bsp_board_leds_on)
    bsp_board_pin_to_button_idx              0x00027ec9   Thumb Code    30  boards.o(i.bsp_board_pin_to_button_idx)
    bsp_btn_ble_sleep_mode_prepare           0x00027eed   Thumb Code    30  bsp_btn_ble.o(i.bsp_btn_ble_sleep_mode_prepare)
    bsp_event_to_button_action_assign        0x00027f9d   Thumb Code    64  bsp.o(i.bsp_event_to_button_action_assign)
    bsp_indication_set                       0x00027fe1   Thumb Code    20  bsp.o(i.bsp_indication_set)
    bsp_wakeup_button_enable                 0x000281c1   Thumb Code     6  bsp.o(i.bsp_wakeup_button_enable)
    buffer_is_empty                          0x0002828d   Thumb Code    18  nrf_log_frontend.o(i.buffer_is_empty)
    characteristic_add                       0x000282b5   Thumb Code   400  ble_srv_common.o(i.characteristic_add)
    conn_handle_list_get                     0x00028529   Thumb Code    62  ble_conn_state.o(i.conn_handle_list_get)
    disk_initialize                          0x00028b29   Thumb Code   114  diskio_blkdev.o(i.disk_initialize)
    disk_ioctl                               0x00028ba9   Thumb Code   118  diskio_blkdev.o(i.disk_ioctl)
    disk_read                                0x00028c25   Thumb Code   120  diskio_blkdev.o(i.disk_read)
    disk_status                              0x00028ca1   Thumb Code    26  diskio_blkdev.o(i.disk_status)
    disk_write                               0x00028cc1   Thumb Code   130  diskio_blkdev.o(i.disk_write)
    diskio_blockdev_register                 0x00028d49   Thumb Code     8  diskio_blkdev.o(i.diskio_blockdev_register)
    drv_rtc_counter_get                      0x00028d69   Thumb Code     8  drv_rtc.o(i.drv_rtc_counter_get)
    drv_rtc_irq_trigger                      0x00028d71   Thumb Code    30  drv_rtc.o(i.drv_rtc_irq_trigger)
    f_close                                  0x00028d8f   Thumb Code    30  ff.o(i.f_close)
    f_mount                                  0x00028dad   Thumb Code    72  ff.o(i.f_mount)
    f_open                                   0x00028df9   Thumb Code   432  ff.o(i.f_open)
    f_opendir                                0x00028fad   Thumb Code    98  ff.o(i.f_opendir)
    f_readdir                                0x0002900f   Thumb Code    64  ff.o(i.f_readdir)
    f_sync                                   0x00029051   Thumb Code   138  ff.o(i.f_sync)
    f_write                                  0x000290e1   Thumb Code   382  ff.o(i.f_write)
    gatt_evt_handler                         0x000298a9   Thumb Code    52  main.o(i.gatt_evt_handler)
    gatt_init                                0x00029905   Thumb Code    38  main.o(i.gatt_init)
    main                                     0x00029db5   Thumb Code   428  main.o(i.main)
    nrf_atfifo_item_alloc                    0x0002a1a1   Thumb Code    22  nrf_atfifo.o(i.nrf_atfifo_item_alloc)
    nrf_atfifo_item_put                      0x0002a1b7   Thumb Code    22  nrf_atfifo.o(i.nrf_atfifo_item_put)
    nrf_atflags_clear                        0x0002a1cd   Thumb Code    22  nrf_atflags.o(i.nrf_atflags_clear)
    nrf_atflags_get                          0x0002a1e3   Thumb Code    22  nrf_atflags.o(i.nrf_atflags_get)
    nrf_atflags_set                          0x0002a1f9   Thumb Code    20  nrf_atflags.o(i.nrf_atflags_set)
    nrf_atomic_flag_clear_fetch              0x0002a20d   Thumb Code     6  nrf_atomic.o(i.nrf_atomic_flag_clear_fetch)
    nrf_atomic_flag_set                      0x0002a213   Thumb Code     6  nrf_atomic.o(i.nrf_atomic_flag_set)
    nrf_atomic_u32_add                       0x0002a219   Thumb Code    12  nrf_atomic.o(i.nrf_atomic_u32_add)
    nrf_atomic_u32_and                       0x0002a225   Thumb Code    12  nrf_atomic.o(i.nrf_atomic_u32_and)
    nrf_atomic_u32_fetch_and                 0x0002a231   Thumb Code    10  nrf_atomic.o(i.nrf_atomic_u32_fetch_and)
    nrf_atomic_u32_fetch_store               0x0002a23b   Thumb Code    10  nrf_atomic.o(i.nrf_atomic_u32_fetch_store)
    nrf_atomic_u32_or                        0x0002a245   Thumb Code    12  nrf_atomic.o(i.nrf_atomic_u32_or)
    nrf_atomic_u32_sub                       0x0002a251   Thumb Code    12  nrf_atomic.o(i.nrf_atomic_u32_sub)
    nrf_balloc_alloc                         0x0002a25d   Thumb Code    68  nrf_balloc.o(i.nrf_balloc_alloc)
    nrf_balloc_free                          0x0002a2a1   Thumb Code    48  nrf_balloc.o(i.nrf_balloc_free)
    nrf_balloc_init                          0x0002a2d1   Thumb Code    48  nrf_balloc.o(i.nrf_balloc_init)
    nrf_ble_gatt_att_mtu_periph_set          0x0002a311   Thumb Code    24  nrf_ble_gatt.o(i.nrf_ble_gatt_att_mtu_periph_set)
    nrf_ble_gatt_init                        0x0002a329   Thumb Code    34  nrf_ble_gatt.o(i.nrf_ble_gatt_init)
    nrf_ble_gatt_on_ble_evt                  0x0002a34d   Thumb Code   270  nrf_ble_gatt.o(i.nrf_ble_gatt_on_ble_evt)
    nrf_ble_qwr_conn_handle_assign           0x0002a49d   Thumb Code    22  nrf_ble_qwr.o(i.nrf_ble_qwr_conn_handle_assign)
    nrf_ble_qwr_init                         0x0002a4b3   Thumb Code    36  nrf_ble_qwr.o(i.nrf_ble_qwr_init)
    nrf_ble_qwr_on_ble_evt                   0x0002a4d7   Thumb Code   182  nrf_ble_qwr.o(i.nrf_ble_qwr_on_ble_evt)
    nrf_drv_clock_init                       0x0002a5b1   Thumb Code    56  nrf_drv_clock.o(i.nrf_drv_clock_init)
    nrf_drv_clock_lfclk_release              0x0002a5f1   Thumb Code    48  nrf_drv_clock.o(i.nrf_drv_clock_lfclk_release)
    nrf_drv_spi_init                         0x0002a625   Thumb Code    98  nrf_drv_spi.o(i.nrf_drv_spi_init)
    nrf_drv_uart_init                        0x0002a6ad   Thumb Code    90  nrf_drv_uart.o(i.nrf_drv_uart_init)
    nrf_fprintf                              0x0002a735   Thumb Code    26  nrf_fprintf.o(i.nrf_fprintf)
    nrf_fprintf_buffer_flush                 0x0002a74f   Thumb Code    24  nrf_fprintf.o(i.nrf_fprintf_buffer_flush)
    nrf_fprintf_fmt                          0x0002a767   Thumb Code   474  nrf_fprintf_format.o(i.nrf_fprintf_fmt)
    nrf_log_backend_add                      0x0002ab09   Thumb Code    86  nrf_log_frontend.o(i.nrf_log_backend_add)
    nrf_log_backend_rtt_init                 0x0002ab67   Thumb Code     4  nrf_log_backend_rtt.o(i.nrf_log_backend_rtt_init)
    nrf_log_backend_serial_put               0x0002ab85   Thumb Code   200  nrf_log_backend_serial.o(i.nrf_log_backend_serial_put)
    nrf_log_backend_uart_init                0x0002ac4f   Thumb Code     6  nrf_log_backend_uart.o(i.nrf_log_backend_uart_init)
    nrf_log_color_id_get                     0x0002ac99   Thumb Code    42  nrf_log_frontend.o(i.nrf_log_color_id_get)
    nrf_log_default_backends_init            0x0002acc9   Thumb Code    46  nrf_log_default_backends.o(i.nrf_log_default_backends_init)
    nrf_log_frontend_dequeue                 0x0002acfd   Thumb Code   528  nrf_log_frontend.o(i.nrf_log_frontend_dequeue)
    nrf_log_frontend_std_0                   0x0002af35   Thumb Code     8  nrf_log_frontend.o(i.nrf_log_frontend_std_0)
    nrf_log_frontend_std_1                   0x0002af3d   Thumb Code    14  nrf_log_frontend.o(i.nrf_log_frontend_std_1)
    nrf_log_frontend_std_2                   0x0002af4b   Thumb Code    16  nrf_log_frontend.o(i.nrf_log_frontend_std_2)
    nrf_log_hexdump_entry_process            0x0002af5d   Thumb Code   150  nrf_log_str_formatter.o(i.nrf_log_hexdump_entry_process)
    nrf_log_init                             0x0002b00d   Thumb Code    28  nrf_log_frontend.o(i.nrf_log_init)
    nrf_log_module_cnt_get                   0x0002b035   Thumb Code    10  nrf_log_frontend.o(i.nrf_log_module_cnt_get)
    nrf_log_module_name_get                  0x0002b049   Thumb Code    24  nrf_log_frontend.o(i.nrf_log_module_name_get)
    nrf_log_panic                            0x0002b065   Thumb Code    36  nrf_log_frontend.o(i.nrf_log_panic)
    nrf_log_std_entry_process                0x0002b08d   Thumb Code   182  nrf_log_str_formatter.o(i.nrf_log_std_entry_process)
    nrf_memobj_alloc                         0x0002b143   Thumb Code    96  nrf_memobj.o(i.nrf_memobj_alloc)
    nrf_memobj_free                          0x0002b1a3   Thumb Code    50  nrf_memobj.o(i.nrf_memobj_free)
    nrf_memobj_get                           0x0002b1d5   Thumb Code     8  nrf_memobj.o(i.nrf_memobj_get)
    nrf_memobj_pool_init                     0x0002b1dd   Thumb Code     4  nrf_memobj.o(i.nrf_memobj_pool_init)
    nrf_memobj_put                           0x0002b1e1   Thumb Code    30  nrf_memobj.o(i.nrf_memobj_put)
    nrf_memobj_read                          0x0002b1ff   Thumb Code    16  nrf_memobj.o(i.nrf_memobj_read)
    nrf_memobj_write                         0x0002b20f   Thumb Code    16  nrf_memobj.o(i.nrf_memobj_write)
    nrf_pwr_mgmt_init                        0x0002b221   Thumb Code    28  nrf_pwr_mgmt.o(i.nrf_pwr_mgmt_init)
    nrf_ringbuf_init                         0x0002b24d   Thumb Code    28  nrf_ringbuf.o(i.nrf_ringbuf_init)
    nrf_sdh_ble_app_ram_start_get            0x0002b269   Thumb Code    16  nrf_sdh_ble.o(i.nrf_sdh_ble_app_ram_start_get)
    nrf_sdh_ble_default_cfg_set              0x0002b27d   Thumb Code   272  nrf_sdh_ble.o(i.nrf_sdh_ble_default_cfg_set)
    nrf_sdh_ble_enable                       0x0002b3ad   Thumb Code   116  nrf_sdh_ble.o(i.nrf_sdh_ble_enable)
    nrf_sdh_enable_request                   0x0002b53d   Thumb Code   102  nrf_sdh.o(i.nrf_sdh_enable_request)
    nrf_sdh_evts_poll                        0x0002b5b1   Thumb Code    32  nrf_sdh.o(i.nrf_sdh_evts_poll)
    nrf_sdh_is_enabled                       0x0002b5d5   Thumb Code     6  nrf_sdh.o(i.nrf_sdh_is_enabled)
    nrf_section_iter_init                    0x0002b61d   Thumb Code    10  nrf_section_iter.o(i.nrf_section_iter_init)
    nrf_section_iter_next                    0x0002b64b   Thumb Code    32  nrf_section_iter.o(i.nrf_section_iter_next)
    nrf_strerror_find                        0x0002b675   Thumb Code    52  nrf_strerror.o(i.nrf_strerror_find)
    nrf_strerror_get                         0x0002b6ad   Thumb Code    14  nrf_strerror.o(i.nrf_strerror_get)
    nrfx_clock_enable                        0x0002b709   Thumb Code    34  nrfx_clock.o(i.nrfx_clock_enable)
    nrfx_clock_init                          0x0002b735   Thumb Code    26  nrfx_clock.o(i.nrfx_clock_init)
    nrfx_clock_lfclk_stop                    0x0002b755   Thumb Code    38  nrfx_clock.o(i.nrfx_clock_lfclk_stop)
    nrfx_prs_acquire                         0x0002b7a5   Thumb Code    58  nrfx_prs.o(i.nrfx_prs_acquire)
    nrfx_prs_release                         0x0002b7df   Thumb Code    18  nrfx_prs.o(i.nrfx_prs_release)
    nrfx_spim_init                           0x0002b7f1   Thumb Code   356  nrfx_spim.o(i.nrfx_spim_init)
    nrfx_spim_uninit                         0x0002b95d   Thumb Code   138  nrfx_spim.o(i.nrfx_spim_uninit)
    nrfx_spim_xfer                           0x0002b9f1   Thumb Code    94  nrfx_spim.o(i.nrfx_spim_xfer)
    nrfx_uart_0_irq_handler                  0x0002ba55   Thumb Code     8  nrfx_uart.o(i.nrfx_uart_0_irq_handler)
    nrfx_uart_init                           0x0002ba65   Thumb Code   200  nrfx_uart.o(i.nrfx_uart_init)
    nrfx_uart_tx                             0x0002bb39   Thumb Code   162  nrfx_uart.o(i.nrfx_uart_tx)
    nrfx_uart_tx_in_progress                 0x0002bbe1   Thumb Code    26  nrfx_uart.o(i.nrfx_uart_tx_in_progress)
    nrfx_uart_uninit                         0x0002bc01   Thumb Code   182  nrfx_uart.o(i.nrfx_uart_uninit)
    nrfx_uarte_0_irq_handler                 0x0002bcc1   Thumb Code     8  nrfx_uarte.o(i.nrfx_uarte_0_irq_handler)
    nrfx_uarte_init                          0x0002bcd1   Thumb Code   100  nrfx_uarte.o(i.nrfx_uarte_init)
    nrfx_uarte_tx                            0x0002bd3d   Thumb Code   166  nrfx_uarte.o(i.nrfx_uarte_tx)
    nrfx_uarte_tx_in_progress                0x0002bde9   Thumb Code    22  nrfx_uarte.o(i.nrfx_uarte_tx_in_progress)
    nrfx_uarte_uninit                        0x0002be05   Thumb Code   254  nrfx_uarte.o(i.nrfx_uarte_uninit)
    nvmc_config                              0x0002bfa5   Thumb Code    14  system_nrf52.o(i.nvmc_config)
    saadc_init                               0x0002c5d5   Thumb Code    54  main.o(i.saadc_init)
    saadc_start                              0x0002c619   Thumb Code    30  main.o(i.saadc_start)
    timer_init                               0x0002d531   Thumb Code    62  main.o(i.timer_init)
    nrf_block_device_sdc_ops                 0x0002dddc   Data          24  nrf_block_dev_sdc.o(.constdata)
    nrf_log_backend_rtt_api                  0x0002de3c   Data          12  nrf_log_backend_rtt.o(.constdata)
    nrf_log_backend_uart_api                 0x0002de64   Data          12  nrf_log_backend_uart.o(.constdata)
    m_ram_start                              0x0002df08   Data           4  nrf_sdh_ble.o(.constdata)
    __ctype_table                            0x0002df34   Data         129  ctype_o.o(.constdata)
    Region$$Table$$Base                      0x0002e75c   Number         0  anon$$obj.o(Region$$Table)
    Region$$Table$$Limit                     0x0002e77c   Number         0  anon$$obj.o(Region$$Table)
    log_const_data$$Base                     0x0002e79c   Number         0  nrf_ble_gatt.o(log_const_data)
    m_nrf_log_nrf_ble_gatt_logs_data_const   0x0002e79c   Data           8  nrf_ble_gatt.o(log_const_data)
    m_nrf_log_ble_nus_logs_data_const        0x0002e7a4   Data           8  ble_nus.o(log_const_data)
    m_nrf_log_clock_logs_data_const          0x0002e7ac   Data           8  nrf_drv_clock.o(log_const_data)
    m_nrf_log_CLOCK_logs_data_const          0x0002e7b4   Data           8  nrfx_clock.o(log_const_data)
    m_nrf_log_GPIOTE_logs_data_const         0x0002e7bc   Data           8  nrfx_gpiote.o(log_const_data)
    m_nrf_log_PRS_logs_data_const            0x0002e7c4   Data           8  nrfx_prs.o(log_const_data)
    m_nrf_log_UART_logs_data_const           0x0002e7cc   Data           8  nrfx_uart.o(log_const_data)
    m_nrf_log_UARTE_logs_data_const          0x0002e7d4   Data           8  nrfx_uarte.o(log_const_data)
    m_nrf_log_SPIM_logs_data_const           0x0002e7dc   Data           8  nrfx_spim.o(log_const_data)
    m_nrf_log_app_button_logs_data_const     0x0002e7e4   Data           8  app_button.o(log_const_data)
    m_nrf_log_app_timer_logs_data_const      0x0002e7ec   Data           8  app_timer2.o(log_const_data)
    m_nrf_log_pwr_mgmt_logs_data_const       0x0002e7f4   Data           8  nrf_pwr_mgmt.o(log_const_data)
    m_nrf_log_sortlist_logs_data_const       0x0002e7fc   Data           8  nrf_sortlist.o(log_const_data)
    m_nrf_log_app_logs_data_const            0x0002e804   Data           8  nrf_log_frontend.o(log_const_data)
    m_nrf_log_nrf_sdh_logs_data_const        0x0002e80c   Data           8  nrf_sdh.o(log_const_data)
    m_nrf_log_nrf_sdh_ble_logs_data_const    0x0002e814   Data           8  nrf_sdh_ble.o(log_const_data)
    m_nrf_log_nrf_sdh_soc_logs_data_const    0x0002e81c   Data           8  nrf_sdh_soc.o(log_const_data)
    log_const_data$$Limit                    0x0002e824   Number         0  nrf_sdh_soc.o(log_const_data)
    log_mempool                              0x0002e824   Data          20  nrf_log_frontend.o(nrf_balloc)
    sdh_ble_observers0$$Base                 0x0002e838   Number         0  ble_conn_state.o(sdh_ble_observers0)
    sdh_ble_observers0$$Limit                0x0002e840   Number         0  ble_conn_state.o(sdh_ble_observers0)
    sdh_ble_observers1$$Base                 0x0002e840   Number         0  main.o(sdh_ble_observers1)
    sdh_ble_observers1$$Limit                0x0002e860   Number         0  ble_conn_params.o(sdh_ble_observers1)
    sdh_ble_observers2$$Base                 0x0002e860   Number         0  main.o(sdh_ble_observers2)
    sdh_ble_observers2$$Limit                0x0002e870   Number         0  main.o(sdh_ble_observers2)
    sdh_ble_observers3$$Base                 0x0002e870   Number         0  main.o(sdh_ble_observers3)
    sdh_ble_observers3$$Limit                0x0002e878   Number         0  main.o(sdh_ble_observers3)
    sdh_soc_observers0$$Base                 0x0002e878   Number         0  nrf_drv_clock.o(sdh_soc_observers0)
    sdh_soc_observers0$$Limit                0x0002e880   Number         0  nrf_drv_clock.o(sdh_soc_observers0)
    sdh_stack_observers0$$Base               0x0002e880   Number         0  nrf_sdh_ble.o(sdh_stack_observers0)
    sdh_stack_observers0$$Limit              0x0002e890   Number         0  nrf_sdh_soc.o(sdh_stack_observers0)
    sdh_state_observers0$$Base               0x0002e890   Number         0  nrf_drv_clock.o(sdh_state_observers0)
    sdh_state_observers0$$Limit              0x0002e898   Number         0  nrf_drv_clock.o(sdh_state_observers0)
    Image$$RW_IRAM1$$Base                    0x20002ad8   Number         0  anon$$obj.o ABSOLUTE
    user_info_written                        0x20002ad8   Data           1  main.o(.data)
    count_EMG_data                           0x20002ada   Data           2  main.o(.data)
    count_sample                             0x20002ae0   Data           4  main.o(.data)
    nrf_drv_uart_use_easy_dma                0x20002b40   Data           1  nrf_drv_uart.o(.data)
    m_uart                                   0x20002c28   Data          20  nrf_log_backend_uart.o(.data)
    SystemCoreClock                          0x20002c50   Data           4  system_nrf52.o(.data)
    EMG_data                                 0x200030f0   Data       30001  main.o(.bss)
    nrf_nvic_state                           0x2000ad00   Data          12  app_util_platform.o(.bss)
    _SEGGER_RTT                              0x2000b36c   Data         120  segger_rtt.o(.bss)
    __initial_sp                             0x2000d5f8   Data           0  arm_startup_nrf52.o(STACK)



==============================================================================

Memory Map of the image

  Image Entry point : 0x00026201

  Load Region LR_IROM1 (Base: 0x00026000, Size: 0x00008a14, Max: 0x0005a000, ABSOLUTE, COMPRESSED[0x000088fc])

    Execution Region ER_IROM1 (Exec base: 0x00026000, Load base: 0x00026000, Size: 0x00008898, Max: 0x0005a000, ABSOLUTE)

    Exec Addr    Load Addr    Size         Type   Attr      Idx    E Section Name        Object

    0x00026000   0x00026000   0x00000200   Data   RO         5971    RESET               arm_startup_nrf52.o
    0x00026200   0x00026200   0x00000000   Code   RO         6037  * .ARM.Collect$$$$00000000  mc_w.l(entry.o)
    0x00026200   0x00026200   0x00000004   Code   RO         6345    .ARM.Collect$$$$00000001  mc_w.l(entry2.o)
    0x00026204   0x00026204   0x00000004   Code   RO         6348    .ARM.Collect$$$$00000004  mc_w.l(entry5.o)
    0x00026208   0x00026208   0x00000000   Code   RO         6350    .ARM.Collect$$$$00000008  mc_w.l(entry7b.o)
    0x00026208   0x00026208   0x00000000   Code   RO         6352    .ARM.Collect$$$$0000000A  mc_w.l(entry8b.o)
    0x00026208   0x00026208   0x00000008   Code   RO         6353    .ARM.Collect$$$$0000000B  mc_w.l(entry9a.o)
    0x00026210   0x00026210   0x00000000   Code   RO         6355    .ARM.Collect$$$$0000000D  mc_w.l(entry10a.o)
    0x00026210   0x00026210   0x00000000   Code   RO         6357    .ARM.Collect$$$$0000000F  mc_w.l(entry11a.o)
    0x00026210   0x00026210   0x00000004   Code   RO         6346    .ARM.Collect$$$$00002712  mc_w.l(entry2.o)
    0x00026214   0x00026214   0x000000c8   Code   RO         3720    .emb_text           nrf_atfifo.o
    0x000262dc   0x000262dc   0x000000e2   Code   RO         3856    .emb_text           nrf_atomic.o
    0x000263be   0x000263be   0x00000002   PAD
    0x000263c0   0x000263c0   0x00000024   Code   RO         5972    .text               arm_startup_nrf52.o
    0x000263e4   0x000263e4   0x00000062   Code   RO         6040    .text               mc_w.l(uldiv.o)
    0x00026446   0x00026446   0x0000001e   Code   RO         6042    .text               mc_w.l(llshl.o)
    0x00026464   0x00026464   0x00000008   Code   RO         6044    .text               mc_w.l(ctype_o.o)
    0x0002646c   0x0002646c   0x00000024   Code   RO         6072    .text               mc_w.l(memcpya.o)
    0x00026490   0x00026490   0x00000024   Code   RO         6074    .text               mc_w.l(memseta.o)
    0x000264b4   0x000264b4   0x0000000e   Code   RO         6076    .text               mc_w.l(strlen.o)
    0x000264c2   0x000264c2   0x00000012   Code   RO         6080    .text               mc_w.l(strcpy.o)
    0x000264d4   0x000264d4   0x0000002c   Code   RO         6359    .text               mc_w.l(uidiv.o)
    0x00026500   0x00026500   0x00000020   Code   RO         6361    .text               mc_w.l(llushr.o)
    0x00026520   0x00026520   0x00000024   Code   RO         6374    .text               mc_w.l(init.o)
    0x00026544   0x00026544   0x00000056   Code   RO         6388    .text               mc_w.l(__dczerorl2.o)
    0x0002659a   0x0002659a   0x00000002   PAD
    0x0002659c   0x0002659c   0x000000a4   Code   RO         2024    i.GPIOTE_IRQHandler  nrfx_gpiote.o
    0x00026640   0x00026640   0x00000058   Code   RO         1885    i.POWER_CLOCK_IRQHandler  nrfx_clock.o
    0x00026698   0x00026698   0x00000010   Code   RO         3506    i.RTC1_IRQHandler   drv_rtc.o
    0x000266a8   0x000266a8   0x00000004   Code   RO         5135    i.SEGGER_RTT_Init   segger_rtt.o
    0x000266ac   0x000266ac   0x0000005c   Code   RO         5149    i.SEGGER_RTT_WriteNoLock  segger_rtt.o
    0x00026708   0x00026708   0x00000054   Code   RO         2792    i.SPIM0_SPIS0_TWIM0_TWIS0_SPI0_TWI0_IRQHandler  nrfx_spim.o
    0x0002675c   0x0002675c   0x00000004   Code   RO         5386    i.SWI2_EGU2_IRQHandler  nrf_sdh.o
    0x00026760   0x00026760   0x00000084   Code   RO         5980    i.SystemInit        system_nrf52.o
    0x000267e4   0x000267e4   0x00000090   Code   RO            4    i.TIMER2_IRQHandler  main.o
    0x00026874   0x00026874   0x0000000c   Code   RO         2325    i.UARTE0_UART0_IRQHandler  nrfx_prs.o
    0x00026880   0x00026880   0x00000068   Code   RO         5153    i._DoInit           segger_rtt.o
    0x000268e8   0x000268e8   0x00000016   Code   RO         5154    i._GetAvailWriteSpace  segger_rtt.o
    0x000268fe   0x000268fe   0x0000005a   Code   RO         5156    i._WriteBlocking    segger_rtt.o
    0x00026958   0x00026958   0x00000042   Code   RO         5157    i._WriteNoCheck     segger_rtt.o
    0x0002699a   0x0002699a   0x00000002   PAD
    0x0002699c   0x0002699c   0x00000028   Code   RO         6131    i.__0sprintf$1      mc_w.l(printf1.o)
    0x000269c4   0x000269c4   0x0000000e   Code   RO         6382    i.__scatterload_copy  mc_w.l(handlers.o)
    0x000269d2   0x000269d2   0x00000002   Code   RO         6383    i.__scatterload_null  mc_w.l(handlers.o)
    0x000269d4   0x000269d4   0x0000000e   Code   RO         6384    i.__scatterload_zeroinit  mc_w.l(handlers.o)
    0x000269e2   0x000269e2   0x00000002   PAD
    0x000269e4   0x000269e4   0x00000024   Code   RO         5387    i.__sd_nvic_app_accessible_irq  nrf_sdh.o
    0x00026a08   0x00026a08   0x00000154   Code   RO         6136    i._printf_core      mc_w.l(printf1.o)
    0x00026b5c   0x00026b5c   0x0000000a   Code   RO         6138    i._sputc            mc_w.l(printf1.o)
    0x00026b66   0x00026b66   0x00000010   Code   RO          901    i.adv_set_data_size_max_get  ble_advertising.o
    0x00026b76   0x00026b76   0x00000036   Code   RO          679    i.advertising_buttons_configure  bsp_btn_ble.o
    0x00026bac   0x00026bac   0x00000084   Code   RO         3064    i.app_error_fault_handler  app_error_weak.o
    0x00026c30   0x00026c30   0x00000016   Code   RO         3008    i.app_error_handler_bare  app_error.o
    0x00026c46   0x00026c46   0x00000016   Code   RO         3099    i.app_fifo_get      app_fifo.o
    0x00026c5c   0x00026c5c   0x0000001a   Code   RO         3102    i.app_fifo_put      app_fifo.o
    0x00026c76   0x00026c76   0x00000002   PAD
    0x00026c78   0x00026c78   0x00000058   Code   RO         4484    i.app_sdc_block_read  app_sdcard.o
    0x00026cd0   0x00026cd0   0x0000006c   Code   RO         4485    i.app_sdc_block_write  app_sdcard.o
    0x00026d3c   0x00026d3c   0x0000001c   Code   RO         4486    i.app_sdc_busy_check  app_sdcard.o
    0x00026d58   0x00026d58   0x00000018   Code   RO         4487    i.app_sdc_info_get  app_sdcard.o
    0x00026d70   0x00026d70   0x000000cc   Code   RO         4488    i.app_sdc_init      app_sdcard.o
    0x00026e3c   0x00026e3c   0x00000048   Code   RO         4489    i.app_sdc_uninit    app_sdcard.o
    0x00026e84   0x00026e84   0x00000016   Code   RO         3224    i.app_timer_create  app_timer2.o
    0x00026e9a   0x00026e9a   0x00000030   Code   RO         3228    i.app_timer_start   app_timer2.o
    0x00026eca   0x00026eca   0x0000000c   Code   RO         3229    i.app_timer_stop    app_timer2.o
    0x00026ed6   0x00026ed6   0x00000002   PAD
    0x00026ed8   0x00026ed8   0x00000054   Code   RO         3365    i.app_uart_put      app_uart_fifo.o
    0x00026f2c   0x00026f2c   0x00000048   Code   RO         3438    i.app_util_critical_region_enter  app_util_platform.o
    0x00026f74   0x00026f74   0x00000034   Code   RO         3439    i.app_util_critical_region_exit  app_util_platform.o
    0x00026fa8   0x00026fa8   0x00000088   Code   RO         2379    i.apply_config      nrfx_uart.o
    0x00027030   0x00027030   0x00000088   Code   RO         2567    i.apply_config      nrfx_uarte.o
    0x000270b8   0x000270b8   0x00000048   Code   RO         1253    i.blcm_link_ctx_get  ble_link_ctx_manager.o
    0x00027100   0x00027100   0x00000182   Code   RO          789    i.ble_advdata_encode  ble_advdata.o
    0x00027282   0x00027282   0x00000020   Code   RO          791    i.ble_advdata_parse  ble_advdata.o
    0x000272a2   0x000272a2   0x00000046   Code   RO          792    i.ble_advdata_search  ble_advdata.o
    0x000272e8   0x000272e8   0x00000006   Code   RO          903    i.ble_advertising_conn_cfg_tag_set  ble_advertising.o
    0x000272ee   0x000272ee   0x000000f8   Code   RO          904    i.ble_advertising_init  ble_advertising.o
    0x000273e6   0x000273e6   0x0000006a   Code   RO          906    i.ble_advertising_on_ble_evt  ble_advertising.o
    0x00027450   0x00027450   0x00000230   Code   RO          909    i.ble_advertising_start  ble_advertising.o
    0x00027680   0x00027680   0x00000068   Code   RO         1003    i.ble_conn_params_init  ble_conn_params.o
    0x000276e8   0x000276e8   0x00000012   Code   RO         1085    i.ble_conn_state_conn_idx  ble_conn_state.o
    0x000276fa   0x000276fa   0x00000002   PAD
    0x000276fc   0x000276fc   0x00000014   Code   RO         1099    i.ble_conn_state_valid  ble_conn_state.o
    0x00027710   0x00027710   0x00000060   Code   RO          795    i.ble_device_addr_encode  ble_advdata.o
    0x00027770   0x00027770   0x000000dc   Code   RO            5    i.ble_evt_handler   main.o
    0x0002784c   0x0002784c   0x00000070   Code   RO          680    i.ble_evt_handler   bsp_btn_ble.o
    0x000278bc   0x000278bc   0x000000fc   Code   RO         1005    i.ble_evt_handler   ble_conn_params.o
    0x000279b8   0x000279b8   0x00000118   Code   RO         1100    i.ble_evt_handler   ble_conn_state.o
    0x00027ad0   0x00027ad0   0x000000d4   Code   RO         1483    i.ble_nus_init      ble_nus.o
    0x00027ba4   0x00027ba4   0x00000076   Code   RO         1484    i.ble_nus_on_ble_evt  ble_nus.o
    0x00027c1a   0x00027c1a   0x00000008   Code   RO         1279    i.ble_srv_is_notification_enabled  ble_srv_common.o
    0x00027c22   0x00027c22   0x00000002   PAD
    0x00027c24   0x00027c24   0x0000002c   Code   RO         5596    i.block_dev_handler  diskio_blkdev.o
    0x00027c50   0x00027c50   0x00000004   Code   RO         4621    i.block_dev_sdc_geometry  nrf_block_dev_sdc.o
    0x00027c54   0x00027c54   0x00000074   Code   RO         4622    i.block_dev_sdc_init  nrf_block_dev_sdc.o
    0x00027cc8   0x00027cc8   0x00000020   Code   RO         4623    i.block_dev_sdc_ioctl  nrf_block_dev_sdc.o
    0x00027ce8   0x00027ce8   0x0000007c   Code   RO         4624    i.block_dev_sdc_read_req  nrf_block_dev_sdc.o
    0x00027d64   0x00027d64   0x00000054   Code   RO         4625    i.block_dev_sdc_uninit  nrf_block_dev_sdc.o
    0x00027db8   0x00027db8   0x0000007c   Code   RO         4626    i.block_dev_sdc_write_req  nrf_block_dev_sdc.o
    0x00027e34   0x00027e34   0x0000000c   Code   RO          445    i.bsp_board_button_idx_to_pin  boards.o
    0x00027e40   0x00027e40   0x00000024   Code   RO          449    i.bsp_board_led_invert  boards.o
    0x00027e64   0x00027e64   0x00000010   Code   RO          450    i.bsp_board_led_off  boards.o
    0x00027e74   0x00027e74   0x00000010   Code   RO          451    i.bsp_board_led_on  boards.o
    0x00027e84   0x00027e84   0x00000020   Code   RO          452    i.bsp_board_led_state_get  boards.o
    0x00027ea4   0x00027ea4   0x00000012   Code   RO          453    i.bsp_board_leds_off  boards.o
    0x00027eb6   0x00027eb6   0x00000012   Code   RO          454    i.bsp_board_leds_on  boards.o
    0x00027ec8   0x00027ec8   0x00000024   Code   RO          455    i.bsp_board_pin_to_button_idx  boards.o
    0x00027eec   0x00027eec   0x0000001e   Code   RO          682    i.bsp_btn_ble_sleep_mode_prepare  bsp_btn_ble.o
    0x00027f0a   0x00027f0a   0x00000002   PAD
    0x00027f0c   0x00027f0c   0x00000090   Code   RO          563    i.bsp_button_event_handler  bsp.o
    0x00027f9c   0x00027f9c   0x00000044   Code   RO          567    i.bsp_event_to_button_action_assign  bsp.o
    0x00027fe0   0x00027fe0   0x00000018   Code   RO          568    i.bsp_indication_set  bsp.o
    0x00027ff8   0x00027ff8   0x000001c8   Code   RO          570    i.bsp_led_indication  bsp.o
    0x000281c0   0x000281c0   0x00000006   Code   RO          572    i.bsp_wakeup_button_enable  bsp.o
    0x000281c6   0x000281c6   0x00000002   PAD
    0x000281c8   0x000281c8   0x00000094   Code   RO         4822    i.buf_prealloc      nrf_log_frontend.o
    0x0002825c   0x0002825c   0x0000002e   Code   RO         4068    i.buffer_add        nrf_fprintf_format.o
    0x0002828a   0x0002828a   0x00000002   PAD
    0x0002828c   0x0002828c   0x00000018   Code   RO         4823    i.buffer_is_empty   nrf_log_frontend.o
    0x000282a4   0x000282a4   0x00000010   Code   RO         2027    i.channel_port_get  nrfx_gpiote.o
    0x000282b4   0x000282b4   0x00000190   Code   RO         1281    i.characteristic_add  ble_srv_common.o
    0x00028444   0x00028444   0x00000070   Code   RO         5676    i.check_fs          ff.o
    0x000284b4   0x000284b4   0x00000028   Code   RO         1540    i.clock_clk_started_notify  nrf_drv_clock.o
    0x000284dc   0x000284dc   0x0000001c   Code   RO         1541    i.clock_irq_handler  nrf_drv_clock.o
    0x000284f8   0x000284f8   0x00000018   Code   RO         5677    i.clust2sect        ff.o
    0x00028510   0x00028510   0x00000018   Code   RO         3231    i.compare_func      app_timer2.o
    0x00028528   0x00028528   0x0000003e   Code   RO         1101    i.conn_handle_list_get  ble_conn_state.o
    0x00028566   0x00028566   0x00000088   Code   RO          796    i.conn_int_encode   ble_advdata.o
    0x000285ee   0x000285ee   0x00000004   Code   RO            6    i.conn_params_error_handler  main.o
    0x000285f2   0x000285f2   0x00000002   PAD
    0x000285f4   0x000285f4   0x00000048   Code   RO         1006    i.conn_params_negotiation  ble_conn_params.o
    0x0002863c   0x0002863c   0x000000a4   Code   RO         5678    i.create_chain      ff.o
    0x000286e0   0x000286e0   0x000000e4   Code   RO         5679    i.create_name       ff.o
    0x000287c4   0x000287c4   0x000000c0   Code   RO         1339    i.data_length_update  nrf_ble_gatt.o
    0x00028884   0x00028884   0x00000004   Code   RO         5597    i.default_wait_func  diskio_blkdev.o
    0x00028888   0x00028888   0x00000064   Code   RO         5680    i.dir_find          ff.o
    0x000288ec   0x000288ec   0x000000f4   Code   RO         5681    i.dir_next          ff.o
    0x000289e0   0x000289e0   0x00000060   Code   RO         5682    i.dir_read          ff.o
    0x00028a40   0x00028a40   0x00000066   Code   RO         5683    i.dir_register      ff.o
    0x00028aa6   0x00028aa6   0x00000082   Code   RO         5685    i.dir_sdi           ff.o
    0x00028b28   0x00028b28   0x00000080   Code   RO         5598    i.disk_initialize   diskio_blkdev.o
    0x00028ba8   0x00028ba8   0x0000007c   Code   RO         5599    i.disk_ioctl        diskio_blkdev.o
    0x00028c24   0x00028c24   0x0000007c   Code   RO         5600    i.disk_read         diskio_blkdev.o
    0x00028ca0   0x00028ca0   0x00000020   Code   RO         5601    i.disk_status       diskio_blkdev.o
    0x00028cc0   0x00028cc0   0x00000088   Code   RO         5603    i.disk_write        diskio_blkdev.o
    0x00028d48   0x00028d48   0x0000000c   Code   RO         5604    i.diskio_blockdev_register  diskio_blkdev.o
    0x00028d54   0x00028d54   0x00000014   Code   RO         4824    i.dropped_sat16_get  nrf_log_frontend.o
    0x00028d68   0x00028d68   0x00000008   Code   RO         3512    i.drv_rtc_counter_get  drv_rtc.o
    0x00028d70   0x00028d70   0x0000001e   Code   RO         3514    i.drv_rtc_irq_trigger  drv_rtc.o
    0x00028d8e   0x00028d8e   0x0000001e   Code   RO         5686    i.f_close           ff.o
    0x00028dac   0x00028dac   0x0000004c   Code   RO         5693    i.f_mount           ff.o
    0x00028df8   0x00028df8   0x000001b4   Code   RO         5694    i.f_open            ff.o
    0x00028fac   0x00028fac   0x00000062   Code   RO         5695    i.f_opendir         ff.o
    0x0002900e   0x0002900e   0x00000040   Code   RO         5700    i.f_readdir         ff.o
    0x0002904e   0x0002904e   0x00000002   PAD
    0x00029050   0x00029050   0x00000090   Code   RO         5703    i.f_sync            ff.o
    0x000290e0   0x000290e0   0x0000017e   Code   RO         5706    i.f_write           ff.o
    0x0002925e   0x0002925e   0x00000002   PAD
    0x00029260   0x00029260   0x0000032c   Code   RO            7    i.fatfs_example     main.o
    0x0002958c   0x0002958c   0x00000014   Code   RO         3105    i.fifo_get          app_fifo.o
    0x000295a0   0x000295a0   0x00000012   Code   RO         3106    i.fifo_put          app_fifo.o
    0x000295b2   0x000295b2   0x00000002   PAD
    0x000295b4   0x000295b4   0x0000024c   Code   RO         5707    i.find_volume       ff.o
    0x00029800   0x00029800   0x0000000a   Code   RO         1102    i.flag_toggle       ble_conn_state.o
    0x0002980a   0x0002980a   0x00000028   Code   RO          911    i.flags_set         ble_advertising.o
    0x00029832   0x00029832   0x00000074   Code   RO         5708    i.follow_path       ff.o
    0x000298a6   0x000298a6   0x00000002   PAD
    0x000298a8   0x000298a8   0x0000005c   Code   RO            8    i.gatt_evt_handler  main.o
    0x00029904   0x00029904   0x00000030   Code   RO            9    i.gatt_init         main.o
    0x00029934   0x00029934   0x000000be   Code   RO         5709    i.get_fat           ff.o
    0x000299f2   0x000299f2   0x00000062   Code   RO         5710    i.get_fileinfo      ff.o
    0x00029a54   0x00029a54   0x0000003c   Code   RO         5711    i.get_ldnumber      ff.o
    0x00029a90   0x00029a90   0x00000034   Code   RO         3232    i.get_now           app_timer2.o
    0x00029ac4   0x00029ac4   0x00000014   Code   RO         1007    i.instance_get      ble_conn_params.o
    0x00029ad8   0x00029ad8   0x000000a6   Code   RO         4069    i.int_print         nrf_fprintf_format.o
    0x00029b7e   0x00029b7e   0x00000002   PAD
    0x00029b80   0x00029b80   0x00000088   Code   RO         2568    i.interrupts_enable  nrfx_uarte.o
    0x00029c08   0x00029c08   0x00000034   Code   RO         4825    i.invalid_packets_omit  nrf_log_frontend.o
    0x00029c3c   0x00029c3c   0x00000044   Code   RO         1008    i.is_conn_params_ok  ble_conn_params.o
    0x00029c80   0x00029c80   0x00000026   Code   RO         5712    i.ld_clust          ff.o
    0x00029ca6   0x00029ca6   0x00000016   Code   RO         5713    i.ld_dword          ff.o
    0x00029cbc   0x00029cbc   0x0000000a   Code   RO         5714    i.ld_word           ff.o
    0x00029cc6   0x00029cc6   0x00000002   PAD
    0x00029cc8   0x00029cc8   0x00000030   Code   RO          574    i.leds_off          bsp.o
    0x00029cf8   0x00029cf8   0x00000018   Code   RO         1340    i.link_init         nrf_ble_gatt.o
    0x00029d10   0x00029d10   0x000000a4   Code   RO         4826    i.log_skip          nrf_log_frontend.o
    0x00029db4   0x00029db4   0x000001e0   Code   RO           10    i.main              main.o
    0x00029f94   0x00029f94   0x00000064   Code   RO          797    i.manuf_specific_data_encode  ble_advdata.o
    0x00029ff8   0x00029ff8   0x00000012   Code   RO         5715    i.mem_cpy           ff.o
    0x0002a00a   0x0002a00a   0x00000002   PAD
    0x0002a00c   0x0002a00c   0x0000000e   Code   RO         5716    i.mem_set           ff.o
    0x0002a01a   0x0002a01a   0x0000007e   Code   RO         4108    i.memobj_op         nrf_memobj.o
    0x0002a098   0x0002a098   0x00000030   Code   RO         4827    i.module_idx_get    nrf_log_frontend.o
    0x0002a0c8   0x0002a0c8   0x00000032   Code   RO         5717    i.move_window       ff.o
    0x0002a0fa   0x0002a0fa   0x000000a6   Code   RO          798    i.name_encode       ble_advdata.o
    0x0002a1a0   0x0002a1a0   0x00000016   Code   RO         3725    i.nrf_atfifo_item_alloc  nrf_atfifo.o
    0x0002a1b6   0x0002a1b6   0x00000016   Code   RO         3728    i.nrf_atfifo_item_put  nrf_atfifo.o
    0x0002a1cc   0x0002a1cc   0x00000016   Code   RO         3790    i.nrf_atflags_clear  nrf_atflags.o
    0x0002a1e2   0x0002a1e2   0x00000016   Code   RO         3795    i.nrf_atflags_get   nrf_atflags.o
    0x0002a1f8   0x0002a1f8   0x00000014   Code   RO         3797    i.nrf_atflags_set   nrf_atflags.o
    0x0002a20c   0x0002a20c   0x00000006   Code   RO         3858    i.nrf_atomic_flag_clear_fetch  nrf_atomic.o
    0x0002a212   0x0002a212   0x00000006   Code   RO         3859    i.nrf_atomic_flag_set  nrf_atomic.o
    0x0002a218   0x0002a218   0x0000000c   Code   RO         3861    i.nrf_atomic_u32_add  nrf_atomic.o
    0x0002a224   0x0002a224   0x0000000c   Code   RO         3862    i.nrf_atomic_u32_and  nrf_atomic.o
    0x0002a230   0x0002a230   0x0000000a   Code   RO         3865    i.nrf_atomic_u32_fetch_and  nrf_atomic.o
    0x0002a23a   0x0002a23a   0x0000000a   Code   RO         3867    i.nrf_atomic_u32_fetch_store  nrf_atomic.o
    0x0002a244   0x0002a244   0x0000000c   Code   RO         3871    i.nrf_atomic_u32_or  nrf_atomic.o
    0x0002a250   0x0002a250   0x0000000c   Code   RO         3873    i.nrf_atomic_u32_sub  nrf_atomic.o
    0x0002a25c   0x0002a25c   0x00000044   Code   RO         3992    i.nrf_balloc_alloc  nrf_balloc.o
    0x0002a2a0   0x0002a2a0   0x00000030   Code   RO         3993    i.nrf_balloc_free   nrf_balloc.o
    0x0002a2d0   0x0002a2d0   0x00000030   Code   RO         3994    i.nrf_balloc_init   nrf_balloc.o
    0x0002a300   0x0002a300   0x00000010   Code   RO         2028    i.nrf_bitmask_bit_is_set  nrfx_gpiote.o
    0x0002a310   0x0002a310   0x00000018   Code   RO         1342    i.nrf_ble_gatt_att_mtu_periph_set  nrf_ble_gatt.o
    0x0002a328   0x0002a328   0x00000022   Code   RO         1346    i.nrf_ble_gatt_init  nrf_ble_gatt.o
    0x0002a34a   0x0002a34a   0x00000002   PAD
    0x0002a34c   0x0002a34c   0x00000150   Code   RO         1347    i.nrf_ble_gatt_on_ble_evt  nrf_ble_gatt.o
    0x0002a49c   0x0002a49c   0x00000016   Code   RO         1441    i.nrf_ble_qwr_conn_handle_assign  nrf_ble_qwr.o
    0x0002a4b2   0x0002a4b2   0x00000024   Code   RO         1442    i.nrf_ble_qwr_init  nrf_ble_qwr.o
    0x0002a4d6   0x0002a4d6   0x000000b6   Code   RO         1443    i.nrf_ble_qwr_on_ble_evt  nrf_ble_qwr.o
    0x0002a58c   0x0002a58c   0x00000006   Code   RO         5605    i.nrf_blk_dev_ioctl  diskio_blkdev.o
    0x0002a592   0x0002a592   0x0000000e   Code   RO         1886    i.nrf_clock_event_check  nrfx_clock.o
    0x0002a5a0   0x0002a5a0   0x00000010   Code   RO         1887    i.nrf_clock_event_clear  nrfx_clock.o
    0x0002a5b0   0x0002a5b0   0x00000040   Code   RO         1548    i.nrf_drv_clock_init  nrf_drv_clock.o
    0x0002a5f0   0x0002a5f0   0x00000034   Code   RO         1552    i.nrf_drv_clock_lfclk_release  nrf_drv_clock.o
    0x0002a624   0x0002a624   0x00000070   Code   RO         2727    i.nrf_drv_spi_init  nrf_drv_spi.o
    0x0002a694   0x0002a694   0x00000016   Code   RO         4490    i.nrf_drv_spi_transfer  app_sdcard.o
    0x0002a6aa   0x0002a6aa   0x00000002   PAD
    0x0002a6ac   0x0002a6ac   0x00000068   Code   RO         1694    i.nrf_drv_uart_init  nrf_drv_uart.o
    0x0002a714   0x0002a714   0x00000020   Code   RO         3367    i.nrf_drv_uart_tx   app_uart_fifo.o
    0x0002a734   0x0002a734   0x0000001a   Code   RO         4029    i.nrf_fprintf       nrf_fprintf.o
    0x0002a74e   0x0002a74e   0x00000018   Code   RO         4030    i.nrf_fprintf_buffer_flush  nrf_fprintf.o
    0x0002a766   0x0002a766   0x000001da   Code   RO         4070    i.nrf_fprintf_fmt   nrf_fprintf_format.o
    0x0002a940   0x0002a940   0x00000024   Code   RO         2380    i.nrf_gpio_cfg      nrfx_uart.o
    0x0002a964   0x0002a964   0x00000024   Code   RO         2569    i.nrf_gpio_cfg      nrfx_uarte.o
    0x0002a988   0x0002a988   0x00000024   Code   RO         2793    i.nrf_gpio_cfg      nrfx_spim.o
    0x0002a9ac   0x0002a9ac   0x00000024   Code   RO         4491    i.nrf_gpio_cfg      app_sdcard.o
    0x0002a9d0   0x0002a9d0   0x00000012   Code   RO         2381    i.nrf_gpio_cfg_default  nrfx_uart.o
    0x0002a9e2   0x0002a9e2   0x00000012   Code   RO         2570    i.nrf_gpio_cfg_default  nrfx_uarte.o
    0x0002a9f4   0x0002a9f4   0x00000012   Code   RO         2382    i.nrf_gpio_cfg_input  nrfx_uart.o
    0x0002aa06   0x0002aa06   0x00000012   Code   RO         2571    i.nrf_gpio_cfg_input  nrfx_uarte.o
    0x0002aa18   0x0002aa18   0x00000014   Code   RO         2383    i.nrf_gpio_cfg_output  nrfx_uart.o
    0x0002aa2c   0x0002aa2c   0x00000014   Code   RO         2572    i.nrf_gpio_cfg_output  nrfx_uarte.o
    0x0002aa40   0x0002aa40   0x00000014   Code   RO         2794    i.nrf_gpio_cfg_output  nrfx_spim.o
    0x0002aa54   0x0002aa54   0x00000022   Code   RO         2031    i.nrf_gpio_cfg_sense_set  nrfx_gpiote.o
    0x0002aa76   0x0002aa76   0x00000002   PAD
    0x0002aa78   0x0002aa78   0x0000002c   Code   RO         2032    i.nrf_gpio_latches_read_and_clear  nrfx_gpiote.o
    0x0002aaa4   0x0002aaa4   0x0000000e   Code   RO         2795    i.nrf_gpio_pin_clear  nrfx_spim.o
    0x0002aab2   0x0002aab2   0x0000000e   Code   RO         2796    i.nrf_gpio_pin_set  nrfx_spim.o
    0x0002aac0   0x0002aac0   0x0000000e   Code   RO         4492    i.nrf_gpio_pin_set  app_sdcard.o
    0x0002aace   0x0002aace   0x00000016   Code   RO          458    i.nrf_gpio_pin_write  boards.o
    0x0002aae4   0x0002aae4   0x00000014   Code   RO         2034    i.nrf_gpiote_event_clear  nrfx_gpiote.o
    0x0002aaf8   0x0002aaf8   0x00000010   Code   RO         2035    i.nrf_gpiote_event_is_set  nrfx_gpiote.o
    0x0002ab08   0x0002ab08   0x0000005c   Code   RO         4828    i.nrf_log_backend_add  nrf_log_frontend.o
    0x0002ab64   0x0002ab64   0x00000002   Code   RO         4685    i.nrf_log_backend_rtt_flush  nrf_log_backend_rtt.o
    0x0002ab66   0x0002ab66   0x00000004   Code   RO         4686    i.nrf_log_backend_rtt_init  nrf_log_backend_rtt.o
    0x0002ab6a   0x0002ab6a   0x00000002   Code   RO         4687    i.nrf_log_backend_rtt_panic_set  nrf_log_backend_rtt.o
    0x0002ab6c   0x0002ab6c   0x00000018   Code   RO         4688    i.nrf_log_backend_rtt_put  nrf_log_backend_rtt.o
    0x0002ab84   0x0002ab84   0x000000c8   Code   RO         4747    i.nrf_log_backend_serial_put  nrf_log_backend_serial.o
    0x0002ac4c   0x0002ac4c   0x00000002   Code   RO         5061    i.nrf_log_backend_uart_flush  nrf_log_backend_uart.o
    0x0002ac4e   0x0002ac4e   0x00000006   Code   RO         5062    i.nrf_log_backend_uart_init  nrf_log_backend_uart.o
    0x0002ac54   0x0002ac54   0x0000002c   Code   RO         5063    i.nrf_log_backend_uart_panic_set  nrf_log_backend_uart.o
    0x0002ac80   0x0002ac80   0x00000018   Code   RO         5064    i.nrf_log_backend_uart_put  nrf_log_backend_uart.o
    0x0002ac98   0x0002ac98   0x00000030   Code   RO         4830    i.nrf_log_color_id_get  nrf_log_frontend.o
    0x0002acc8   0x0002acc8   0x00000034   Code   RO         4781    i.nrf_log_default_backends_init  nrf_log_default_backends.o
    0x0002acfc   0x0002acfc   0x00000238   Code   RO         4831    i.nrf_log_frontend_dequeue  nrf_log_frontend.o
    0x0002af34   0x0002af34   0x00000008   Code   RO         4833    i.nrf_log_frontend_std_0  nrf_log_frontend.o
    0x0002af3c   0x0002af3c   0x0000000e   Code   RO         4834    i.nrf_log_frontend_std_1  nrf_log_frontend.o
    0x0002af4a   0x0002af4a   0x00000010   Code   RO         4835    i.nrf_log_frontend_std_2  nrf_log_frontend.o
    0x0002af5a   0x0002af5a   0x00000002   PAD
    0x0002af5c   0x0002af5c   0x000000b0   Code   RO         5009    i.nrf_log_hexdump_entry_process  nrf_log_str_formatter.o
    0x0002b00c   0x0002b00c   0x00000028   Code   RO         4840    i.nrf_log_init      nrf_log_frontend.o
    0x0002b034   0x0002b034   0x00000014   Code   RO         4841    i.nrf_log_module_cnt_get  nrf_log_frontend.o
    0x0002b048   0x0002b048   0x0000001c   Code   RO         4844    i.nrf_log_module_name_get  nrf_log_frontend.o
    0x0002b064   0x0002b064   0x00000028   Code   RO         4845    i.nrf_log_panic     nrf_log_frontend.o
    0x0002b08c   0x0002b08c   0x000000b6   Code   RO         5010    i.nrf_log_std_entry_process  nrf_log_str_formatter.o
    0x0002b142   0x0002b142   0x00000060   Code   RO         4109    i.nrf_memobj_alloc  nrf_memobj.o
    0x0002b1a2   0x0002b1a2   0x00000032   Code   RO         4110    i.nrf_memobj_free   nrf_memobj.o
    0x0002b1d4   0x0002b1d4   0x00000008   Code   RO         4111    i.nrf_memobj_get    nrf_memobj.o
    0x0002b1dc   0x0002b1dc   0x00000004   Code   RO         4112    i.nrf_memobj_pool_init  nrf_memobj.o
    0x0002b1e0   0x0002b1e0   0x0000001e   Code   RO         4113    i.nrf_memobj_put    nrf_memobj.o
    0x0002b1fe   0x0002b1fe   0x00000010   Code   RO         4114    i.nrf_memobj_read   nrf_memobj.o
    0x0002b20e   0x0002b20e   0x00000010   Code   RO         4115    i.nrf_memobj_write  nrf_memobj.o
    0x0002b21e   0x0002b21e   0x00000002   PAD
    0x0002b220   0x0002b220   0x00000028   Code   RO         4187    i.nrf_pwr_mgmt_init  nrf_pwr_mgmt.o
    0x0002b248   0x0002b248   0x00000004   Code   RO           11    i.nrf_qwr_error_handler  main.o
    0x0002b24c   0x0002b24c   0x0000001c   Code   RO         4264    i.nrf_ringbuf_init  nrf_ringbuf.o
    0x0002b268   0x0002b268   0x00000014   Code   RO         5507    i.nrf_sdh_ble_app_ram_start_get  nrf_sdh_ble.o
    0x0002b27c   0x0002b27c   0x00000130   Code   RO         5508    i.nrf_sdh_ble_default_cfg_set  nrf_sdh_ble.o
    0x0002b3ac   0x0002b3ac   0x00000130   Code   RO         5509    i.nrf_sdh_ble_enable  nrf_sdh_ble.o
    0x0002b4dc   0x0002b4dc   0x00000060   Code   RO         5510    i.nrf_sdh_ble_evts_poll  nrf_sdh_ble.o
    0x0002b53c   0x0002b53c   0x00000074   Code   RO         5389    i.nrf_sdh_enable_request  nrf_sdh.o
    0x0002b5b0   0x0002b5b0   0x00000024   Code   RO         5390    i.nrf_sdh_evts_poll  nrf_sdh.o
    0x0002b5d4   0x0002b5d4   0x0000000c   Code   RO         5391    i.nrf_sdh_is_enabled  nrf_sdh.o
    0x0002b5e0   0x0002b5e0   0x0000003c   Code   RO         5561    i.nrf_sdh_soc_evts_poll  nrf_sdh_soc.o
    0x0002b61c   0x0002b61c   0x0000000a   Code   RO         4322    i.nrf_section_iter_init  nrf_section_iter.o
    0x0002b626   0x0002b626   0x00000024   Code   RO         4323    i.nrf_section_iter_item_set  nrf_section_iter.o
    0x0002b64a   0x0002b64a   0x00000020   Code   RO         4324    i.nrf_section_iter_next  nrf_section_iter.o
    0x0002b66a   0x0002b66a   0x0000000a   Code   RO         2797    i.nrf_spim_event_check  nrfx_spim.o
    0x0002b674   0x0002b674   0x00000038   Code   RO         4413    i.nrf_strerror_find  nrf_strerror.o
    0x0002b6ac   0x0002b6ac   0x00000014   Code   RO         4414    i.nrf_strerror_get  nrf_strerror.o
    0x0002b6c0   0x0002b6c0   0x0000000a   Code   RO         2384    i.nrf_uart_event_check  nrfx_uart.o
    0x0002b6ca   0x0002b6ca   0x0000000c   Code   RO         2385    i.nrf_uart_event_clear  nrfx_uart.o
    0x0002b6d6   0x0002b6d6   0x0000000c   Code   RO         2386    i.nrf_uart_int_enable_check  nrfx_uart.o
    0x0002b6e2   0x0002b6e2   0x0000000a   Code   RO         2573    i.nrf_uarte_event_check  nrfx_uarte.o
    0x0002b6ec   0x0002b6ec   0x0000000c   Code   RO         2574    i.nrf_uarte_event_clear  nrfx_uarte.o
    0x0002b6f8   0x0002b6f8   0x00000010   Code   RO         1555    i.nrf_wdt_started   nrf_drv_clock.o
    0x0002b708   0x0002b708   0x0000002c   Code   RO         1892    i.nrfx_clock_enable  nrfx_clock.o
    0x0002b734   0x0002b734   0x00000020   Code   RO         1895    i.nrfx_clock_init   nrfx_clock.o
    0x0002b754   0x0002b754   0x00000030   Code   RO         1898    i.nrfx_clock_lfclk_stop  nrfx_clock.o
    0x0002b784   0x0002b784   0x00000010   Code   RO         2575    i.nrfx_is_in_ram    nrfx_uarte.o
    0x0002b794   0x0002b794   0x00000010   Code   RO         2798    i.nrfx_is_in_ram    nrfx_spim.o
    0x0002b7a4   0x0002b7a4   0x0000003a   Code   RO         2326    i.nrfx_prs_acquire  nrfx_prs.o
    0x0002b7de   0x0002b7de   0x00000012   Code   RO         2327    i.nrfx_prs_release  nrfx_prs.o
    0x0002b7f0   0x0002b7f0   0x0000016c   Code   RO         2801    i.nrfx_spim_init    nrfx_spim.o
    0x0002b95c   0x0002b95c   0x00000094   Code   RO         2803    i.nrfx_spim_uninit  nrfx_spim.o
    0x0002b9f0   0x0002b9f0   0x00000064   Code   RO         2804    i.nrfx_spim_xfer    nrfx_spim.o
    0x0002ba54   0x0002ba54   0x00000010   Code   RO         2387    i.nrfx_uart_0_irq_handler  nrfx_uart.o
    0x0002ba64   0x0002ba64   0x000000d4   Code   RO         2389    i.nrfx_uart_init    nrfx_uart.o
    0x0002bb38   0x0002bb38   0x000000a8   Code   RO         2395    i.nrfx_uart_tx      nrfx_uart.o
    0x0002bbe0   0x0002bbe0   0x00000020   Code   RO         2397    i.nrfx_uart_tx_in_progress  nrfx_uart.o
    0x0002bc00   0x0002bc00   0x000000c0   Code   RO         2398    i.nrfx_uart_uninit  nrfx_uart.o
    0x0002bcc0   0x0002bcc0   0x00000010   Code   RO         2576    i.nrfx_uarte_0_irq_handler  nrfx_uarte.o
    0x0002bcd0   0x0002bcd0   0x0000006c   Code   RO         2578    i.nrfx_uarte_init   nrfx_uarte.o
    0x0002bd3c   0x0002bd3c   0x000000ac   Code   RO         2582    i.nrfx_uarte_tx     nrfx_uarte.o
    0x0002bde8   0x0002bde8   0x0000001c   Code   RO         2584    i.nrfx_uarte_tx_in_progress  nrfx_uarte.o
    0x0002be04   0x0002be04   0x00000108   Code   RO         2585    i.nrfx_uarte_uninit  nrfx_uarte.o
    0x0002bf0c   0x0002bf0c   0x00000098   Code   RO           12    i.nus_data_handler  main.o
    0x0002bfa4   0x0002bfa4   0x00000018   Code   RO         5981    i.nvmc_config       system_nrf52.o
    0x0002bfbc   0x0002bfbc   0x00000036   Code   RO           13    i.on_adv_evt        main.o
    0x0002bff2   0x0002bff2   0x00000002   PAD
    0x0002bff4   0x0002bff4   0x0000001c   Code   RO           14    i.on_conn_params_evt  main.o
    0x0002c010   0x0002c010   0x0000006a   Code   RO         1485    i.on_connect        ble_nus.o
    0x0002c07a   0x0002c07a   0x00000002   PAD
    0x0002c07c   0x0002c07c   0x000000a8   Code   RO         1348    i.on_connected_evt  nrf_ble_gatt.o
    0x0002c124   0x0002c124   0x000000ac   Code   RO         1349    i.on_exchange_mtu_request_evt  nrf_ble_gatt.o
    0x0002c1d0   0x0002c1d0   0x00000084   Code   RO         1486    i.on_write          ble_nus.o
    0x0002c254   0x0002c254   0x00000012   Code   RO          912    i.phy_is_valid      ble_advertising.o
    0x0002c266   0x0002c266   0x00000002   PAD
    0x0002c268   0x0002c268   0x000000b4   Code   RO         2068    i.port_event_handle  nrfx_gpiote.o
    0x0002c31c   0x0002c31c   0x00000010   Code   RO         2069    i.port_handler_polarity_get  nrfx_gpiote.o
    0x0002c32c   0x0002c32c   0x0000003c   Code   RO         5012    i.postfix_process   nrf_log_str_formatter.o
    0x0002c368   0x0002c368   0x00000098   Code   RO         5013    i.prefix_process    nrf_log_str_formatter.o
    0x0002c400   0x0002c400   0x00000018   Code   RO         2328    i.prs_box_get       nrfx_prs.o
    0x0002c418   0x0002c418   0x000000ea   Code   RO         5718    i.put_fat           ff.o
    0x0002c502   0x0002c502   0x00000074   Code   RO         5721    i.remove_chain      ff.o
    0x0002c576   0x0002c576   0x00000032   Code   RO         2399    i.rx_byte           nrfx_uart.o
    0x0002c5a8   0x0002c5a8   0x00000016   Code   RO         2400    i.rx_done_event     nrfx_uart.o
    0x0002c5be   0x0002c5be   0x00000016   Code   RO         2586    i.rx_done_event     nrfx_uarte.o
    0x0002c5d4   0x0002c5d4   0x00000044   Code   RO           15    i.saadc_init        main.o
    0x0002c618   0x0002c618   0x00000028   Code   RO           16    i.saadc_start       main.o
    0x0002c640   0x0002c640   0x00000058   Code   RO         1556    i.sd_state_evt_handler  nrf_drv_clock.o
    0x0002c698   0x0002c698   0x000000b8   Code   RO         4493    i.sdc_cmd           app_sdcard.o
    0x0002c750   0x0002c750   0x0000009c   Code   RO         4627    i.sdc_handler       nrf_block_dev_sdc.o
    0x0002c7ec   0x0002c7ec   0x0000029c   Code   RO         4494    i.sdc_pt_identification  app_sdcard.o
    0x0002ca88   0x0002ca88   0x00000080   Code   RO         4495    i.sdc_pt_read       app_sdcard.o
    0x0002cb08   0x0002cb08   0x00000160   Code   RO         4496    i.sdc_pt_sub_data_read  app_sdcard.o
    0x0002cc68   0x0002cc68   0x00000208   Code   RO         4497    i.sdc_pt_write      app_sdcard.o
    0x0002ce70   0x0002ce70   0x0000003c   Code   RO         4498    i.sdc_spi_transfer  app_sdcard.o
    0x0002ceac   0x0002ceac   0x00000030   Code   RO         5396    i.sdh_request_observer_notify  nrf_sdh.o
    0x0002cedc   0x0002cedc   0x0000002c   Code   RO         5397    i.sdh_state_observer_notify  nrf_sdh.o
    0x0002cf08   0x0002cf08   0x00000010   Code   RO         1009    i.send_error_evt    ble_conn_params.o
    0x0002cf18   0x0002cf18   0x00000050   Code   RO         4689    i.serial_tx         nrf_log_backend_rtt.o
    0x0002cf68   0x0002cf68   0x00000040   Code   RO         5065    i.serial_tx         nrf_log_backend_uart.o
    0x0002cfa8   0x0002cfa8   0x00000088   Code   RO          799    i.service_data_encode  ble_advdata.o
    0x0002d030   0x0002d030   0x00000030   Code   RO         1283    i.set_security_req  ble_srv_common.o
    0x0002d060   0x0002d060   0x00000018   Code   RO         1557    i.soc_evt_handler   nrf_drv_clock.o
    0x0002d078   0x0002d078   0x00000058   Code   RO         5399    i.softdevices_evt_irq_enable  nrf_sdh.o
    0x0002d0d0   0x0002d0d0   0x000001bc   Code   RO         4499    i.spi_handler       app_sdcard.o
    0x0002d28c   0x0002d28c   0x00000038   Code   RO         2728    i.spim_evt_handler  nrf_drv_spi.o
    0x0002d2c4   0x0002d2c4   0x000000bc   Code   RO         2805    i.spim_xfer         nrfx_spim.o
    0x0002d380   0x0002d380   0x00000028   Code   RO         5722    i.st_clust          ff.o
    0x0002d3a8   0x0002d3a8   0x00000010   Code   RO         5723    i.st_dword          ff.o
    0x0002d3b8   0x0002d3b8   0x00000008   Code   RO         5724    i.st_word           ff.o
    0x0002d3c0   0x0002d3c0   0x00000094   Code   RO         4847    i.std_n             nrf_log_frontend.o
    0x0002d454   0x0002d454   0x00000088   Code   RO         5725    i.sync_fs           ff.o
    0x0002d4dc   0x0002d4dc   0x00000052   Code   RO         5726    i.sync_window       ff.o
    0x0002d52e   0x0002d52e   0x00000002   PAD
    0x0002d530   0x0002d530   0x0000004c   Code   RO           17    i.timer_init        main.o
    0x0002d57c   0x0002d57c   0x00000038   Code   RO         3239    i.timer_req_schedule  app_timer2.o
    0x0002d5b4   0x0002d5b4   0x00000020   Code   RO         2402    i.tx_byte           nrfx_uart.o
    0x0002d5d4   0x0002d5d4   0x0000001a   Code   RO         2403    i.tx_done_event     nrfx_uart.o
    0x0002d5ee   0x0002d5ee   0x0000001a   Code   RO         2587    i.tx_done_event     nrfx_uarte.o
    0x0002d608   0x0002d608   0x00000030   Code   RO         1695    i.uart_evt_handler  nrf_drv_uart.o
    0x0002d638   0x0002d638   0x0000000c   Code   RO         5066    i.uart_evt_handler  nrf_log_backend_uart.o
    0x0002d644   0x0002d644   0x00000050   Code   RO         5067    i.uart_init         nrf_log_backend_uart.o
    0x0002d694   0x0002d694   0x0000012a   Code   RO         2404    i.uart_irq_handler  nrfx_uart.o
    0x0002d7be   0x0002d7be   0x00000002   PAD
    0x0002d7c0   0x0002d7c0   0x00000030   Code   RO         1696    i.uarte_evt_handler  nrf_drv_uart.o
    0x0002d7f0   0x0002d7f0   0x00000112   Code   RO         2588    i.uarte_irq_handler  nrfx_uarte.o
    0x0002d902   0x0002d902   0x0000000a   Code   RO          800    i.uint16_encode     ble_advdata.o
    0x0002d90c   0x0002d90c   0x000000b4   Code   RO         4071    i.unsigned_print    nrf_fprintf_format.o
    0x0002d9c0   0x0002d9c0   0x00000068   Code   RO         1010    i.update_timeout_handler  ble_conn_params.o
    0x0002da28   0x0002da28   0x00000018   Code   RO          913    i.use_whitelist     ble_advertising.o
    0x0002da40   0x0002da40   0x00000024   Code   RO         1444    i.user_mem_reply    nrf_ble_qwr.o
    0x0002da64   0x0002da64   0x00000030   Code   RO          801    i.uuid_list_encode  ble_advdata.o
    0x0002da94   0x0002da94   0x0000009e   Code   RO          802    i.uuid_list_sized_encode  ble_advdata.o
    0x0002db32   0x0002db32   0x00000032   Code   RO         5727    i.validate          ff.o
    0x0002db64   0x0002db64   0x0000003a   Code   RO          576    i.wakeup_button_cfg  bsp.o
    0x0002db9e   0x0002db9e   0x00000002   PAD
    0x0002dba0   0x0002dba0   0x0000001c   Data   RO           20    .constdata          main.o
    0x0002dbbc   0x0002dbbc   0x00000008   Data   RO          459    .constdata          boards.o
    0x0002dbc4   0x0002dbc4   0x0000002c   Data   RO          581    .constdata          bsp.o
    0x0002dbf0   0x0002dbf0   0x00000016   Data   RO         1350    .constdata          nrf_ble_gatt.o
    0x0002dc06   0x0002dc06   0x00000002   PAD
    0x0002dc08   0x0002dc08   0x00000010   Data   RO         1487    .constdata          ble_nus.o
    0x0002dc18   0x0002dc18   0x00000004   Data   RO         2071    .constdata          nrfx_gpiote.o
    0x0002dc1c   0x0002dc1c   0x00000004   Data   RO         2407    .constdata          nrfx_uart.o
    0x0002dc20   0x0002dc20   0x00000004   Data   RO         2591    .constdata          nrfx_uarte.o
    0x0002dc24   0x0002dc24   0x00000010   Data   RO         2730    .constdata          nrf_drv_spi.o
    0x0002dc34   0x0002dc34   0x00000004   Data   RO         2808    .constdata          nrfx_spim.o
    0x0002dc38   0x0002dc38   0x00000014   Data   RO         3242    .constdata          app_timer2.o
    0x0002dc4c   0x0002dc4c   0x00000010   Data   RO         4072    .constdata          nrf_fprintf_format.o
    0x0002dc5c   0x0002dc5c   0x00000018   Data   RO         4192    .constdata          nrf_pwr_mgmt.o
    0x0002dc74   0x0002dc74   0x0000000c   Data   RO         4193    .constdata          nrf_pwr_mgmt.o
    0x0002dc80   0x0002dc80   0x0000013c   Data   RO         4415    .constdata          nrf_strerror.o
    0x0002ddbc   0x0002ddbc   0x00000020   Data   RO         4501    .constdata          app_sdcard.o
    0x0002dddc   0x0002dddc   0x00000018   Data   RO         4628    .constdata          nrf_block_dev_sdc.o
    0x0002ddf4   0x0002ddf4   0x00000048   Data   RO         4629    .constdata          nrf_block_dev_sdc.o
    0x0002de3c   0x0002de3c   0x0000000c   Data   RO         4691    .constdata          nrf_log_backend_rtt.o
    0x0002de48   0x0002de48   0x00000008   PAD
    0x0002de50   0x0002de50   0x00000006   Data   RO         4692    .constdata          nrf_log_backend_rtt.o
    0x0002de56   0x0002de56   0x00000002   PAD
    0x0002de58   0x0002de58   0x0000000c   Data   RO         4852    .constdata          nrf_log_frontend.o
    0x0002de64   0x0002de64   0x0000000c   Data   RO         5069    .constdata          nrf_log_backend_uart.o
    0x0002de70   0x0002de70   0x00000020   Data   RO         5070    .constdata          nrf_log_backend_uart.o
    0x0002de90   0x0002de90   0x00000010   Data   RO         5400    .constdata          nrf_sdh.o
    0x0002dea0   0x0002dea0   0x00000028   Data   RO         5401    .constdata          nrf_sdh.o
    0x0002dec8   0x0002dec8   0x00000010   Data   RO         5402    .constdata          nrf_sdh.o
    0x0002ded8   0x0002ded8   0x00000010   Data   RO         5403    .constdata          nrf_sdh.o
    0x0002dee8   0x0002dee8   0x00000020   Data   RO         5511    .constdata          nrf_sdh_ble.o
    0x0002df08   0x0002df08   0x00000010   Data   RO         5512    .constdata          nrf_sdh_ble.o
